:020000040000FA
:200000000208540200800402003F00020008B922FFFFFF02008014FFFFFFFF0200801CFFAA
:20002000FFFFFF020080244447532D31323234542020202020204C56332E30EB7002E7229C
:2000400089828A831410E704F593E022F593E49322BB0002F722BB8000500989828A838BC1
:20006000931593F022BC000BBE0029EF8DF084FFADF022E4CCF875F008EF2FFFEE33FEEC9A
:2000800033FCEE9DEC984005FCEE9DFE0FD5F0E9E4CEFD22EDF8F5F0EE008420D21CFEADD5
:2000A000F075F008EF2FFFED33FD4007985006D5F0F222C398FD0FD5F0EA22A3F8E0C5F033
:2000C00025F0F0E582158270021583E0C838F0E822BB0006F709A7F01922BB8000500D8985
:2000E000828A838B931593F0E5F0A3F022E88FF0A4CC8BF0A42CFCE98EF0A42CFC8AF0ED79
:20010000A42CFCEA8EF0A4CDA8F08BF0A42DCC3825F0FDE98FF0A42CCD35F0FCEB8EF0A40D
:20012000FEA9F0EB8FF0A4CFC5F02ECD39FEE43CFCEAA42DCE35F0FDE43CFC22EB9FF5F0F0
:20014000EA9E42F0E99D42F0E89C45F022E8600FEFC333FFEE33FEED33FDEC33FCD8F122D5
:20016000BB0006E9F802000332BB8000500C89828A838B9315930200017B22ECF0A3EDF035
:20018000A3EEF0A3EFF022EB700C87F009E608B5F019DFF6801589828A831410E70FF59383
:2001A000E0F5F0A3E608B5F002DFF5806AF593E493F5F0A3E608B5F05EDFF4805ACB701311
:2001C00088828C838B9387F009E493A3B5F048DFF580441410E71F88848C858B9589828ACD
:2001E00083F593758620E0F5F0E493A3A3B5F024DFF4DEF2801E88848C858B9589828A83F8
:20020000F593758620E493F5F0E493A3A3B5F004DFF3DEF17586007FFFB5F0020F22400245
:200220007F012202000187809488F0EF60010E4E60F0ED60EE1410E7EECB701288828C8370
:20024000F59387F009E0A3B5F0CDDFF680C91410E71E88848C858B9589828A83F593758682
:2002600020E0F5F0E0A3A3B5F0AADFF5DEF380A488848C858B9589828A83F593758620E47F
:2002800093F5F0E0A3A3B5F08BDFF4DEF28085EB7008E709F608DFFA801B89828A831410E7
:2002A000E70AF593E0A3F608DFFA8009F593E493A3F608DFF9ECFAA9F0EDFB2288F0EF601A
:2002C000010E4E60F088F0ED60C51410E7E7CB700E88828C838B93E709F0A3DFFA80D614AF
:2002E00010E71C88848C858B9589828A83F593758620E0F0A3A3DFFADEF875860080B68875
:20030000848C858B9589828A83F593758620E493F0A3A3DFF9DEF77586008099C5F0F8A3AF
:20032000E028F0C5F0F8E582158270021583E038F022ECF608EDF608EEF608EFF62290008E
:200340007004E0F54090007005E0F541854082854183E020E7077E007F00C2D72289428A6E
:20036000435407F54512000539E02402F54450020545120003E0053AE53A7002053BE54050
:200380002544F540E541354530E604C2E6242DF5411200040090007004E540F090007005A2
:2003A000E541F0AE45AF44D2D72290007010E020E61EA3EDF0A3E9F0A3EAF0EC5407D2E6EA
:2003C00090007010F00538E53870020539D2D7227C007D00C2D72290007010E0A2E6B32247
:2003E00075F001800375F0041200040078407F06900070921200052190007090E5F0F02217
:2004000090007090E0540770F7221200046D90007008742DF0900070107508101200045861
:20042000E490007004F090007006F0742D90007005F090007007F0751D10751C10751E008B
:20044000751F2D75832D758200E4F0753800753900753A00753B0022E4A808F0A3D8FC22F2
:20046000120005171200040A120004AB22900004A175080A79707860120005287518C075CD
:2004800019A8751A00751B647510C07511A87512007513017514FF7515FF7516FF7517006E
:2004A00022000B78667788C0A800649000706AE0440CF0229000706AE054F3F02290007017
:2004C0006AE04401F0229000706AE054FEF0229000706AE04402F0229000706AE054FDF0A0
:2004E000229000706AE04440F0229000706AE054BFF02290007000E04410F0229000700045
:20050000E054EFF02290007000E04420F02290007000E05420F0229000700AF000000000F0
:2005200022E6F008A3DFFA2289A0E493A3F208B800030989A0D508F222A3E58330E6037569
:20054000832D22754300754200754100754000754508754400120003E5754308754200758E
:200560004108754000754508754400120003E51200040090000000750910750800750B00D7
:20058000750A0012000638400B9000706CE04408F0D2D722C2D7227543007542007541000E
:2005A000754000754508754400120003E5754308754200754108754000754508754400129A
:2005C0000003E51200040090000000750910750800750B00750A00120006384051754310DA
:2005E000754200754110754000754508754400120003E575431875420075411875400075D5
:200600004508754400120003E51200040090001000750910750800750B10750A00120006F2
:2006200038400B9000706CE04418F0D2D722C2D722E6F008A3DFFA22A90B89A0A80AE49397
:20064000F5F0A3E265F0701008B800030989A01200067D50E9C2D722D2D722A90B89A0A88D
:200660000AE0F5F0A3E265F0701008B800030989A01200067D50EAC2D722D2D722E50860BA
:200680000A14F50845097007D2D72215091508C2D7229000700B7418F09000700C7420F0A2
:2006A00075A06022120006927824E2E2B408157400F21200072912000721120007071200B4
:2006C000070E802E22120006927816E2E2703708E2E2B4013178281200079C5029120007F9
:2006E0003912000779120007411200078178177402F27800E2E2FC4480F208E2E2FD7918FC
:200700007A20120003AA22781AE4F208F222782680F7E2E2F5F0E3E3F2E5F0F30809DAF2BF
:20072000227A04781C792080E9790878027A0680E1E2E2F30809DAF922780879027A0680EF
:20074000F0780879227A0680E8E4F309F3227A08E480037A04E4F309DAFC22E0F3A309E013
:20076000F3227A04E0F3A309DAFA227A0280027A04E2E2F0A308DAF922900070607A068041
:20078000E3781879227A0A8089E0F5F0E2E265F0700708A3DAF3D2D722C2D7229000706605
:2007A0007A0480E59000200AE0FEA3E08E8375820075814F73220D0A205446333331465556
:2007C0003A333956463038302031364B2D626173656420426C616E6B20436865636B696E64
:2007E00067002E2E2E5B6661696C5D0A002E2E2E5B6F6B5D0A000D0A205446333331465581
:200800003A6465766963655B53535420333956463038305D000D0A20544633333146553A7F
:20082000536563746F722D62617365642832353620736563746F72732920466C61736820DD
:2008400045726173652028314D29002E2E2E5B6F6B5D2E0075C7AA75C755759D02787FE409
:20086000F6D8FD900000007F007E607D01E4F0A3DFFCDEFADDF875814F12000517D20D12DF
:200880000004B41200040A12001DD412001DF0120013EBEF7004020008A5020008B312006D
:2008A0001D36EF700EC20D120004AB1200000702000C7BD20D02008000300D040200800C16
:2008C000C0E0C0D075D00012001DACD0D0D0E0320D0A544633333146553A52657620257542
:2008E0000A54616966617465636820496E632E000D0A2849503D200025752E00257529003D
:200900000D0A284D41433D200025782E00257829000D0A54463333313A2054465450206475
:200920006F6E652E204A756D7020746F20307825782E0A000D0A436865636B204368656363
:200940006B53756D3D00307825782E2E2E4F4B21210D0A00307825782E2E2E4661696C218C
:20096000210D0A001B5B324A000D0A436865636B204D6167696320436F64652E2E2E004FE3
:200980004B2121004661696C212100496C6C6567616C206669726D77617265002E000D0A90
:2009A00020496E76616C6964206669726D776172652021000D0A20466C6173682065727204
:2009C0006F722021004387049000555574AAF090002AAA7455F09000555574A0F08F828EE5
:2009E000838D93E52EF05387FB229000262FEEF0A3EFF0E4784EF608F6D390002630E0944A
:200A0000009000262FE094005003010C7A90002620E0FF94094003010B36EF705E90002659
:200A20002FE0FEA3E0FFD39400EE94004031784EE6FC08E67B012448F974203CFA1200007A
:200A40003B643A601A90002630E024FFF09000262FE034FFF0784F06E61870C10680BEEF53
:200A60004E7003010C7A784B7601900026207401F0784F06E618704F06804C90002620E0A7
:200A8000784BF6784BE6C39409504E90002630E094009000262FE09400403E784E0806E60B
:200AA000188606700106147B012448F974203EFA1200003BFF784BE6062423F582E4342663
:200AC000F583759300EFF090002630E024FFF09000262FE034FFF080AA784BE6900026204D
:200AE000F0C394095003010C7A9000261A7426F0A37423F0120018D1EF64014E70069000A5
:200B00002620F022120018D1EF64044E7003010C2B7D027F01120018D59000261CEFF07D06
:200B2000067C007F037E00120018D990002614EEF0A3EFF0807E9000261DE0FFA3E0900043
:200B40002614CFF0A3EFF090002621E06066D390002630E094009000262FE09400405590F2
:200B600000261A7426F0A37421F0784E0806E6188606700106147B012448F974203EFA12DB
:200B800000003B90002622F090002630E024FFF09000262FE034FFF07D017C00E4FFFE12A4
:200BA0000018D912001541E490002621F09000261CE014F09000261A7420F0A37448F0A335
:200BC000E0FF784C760008A607D3784DE6940018E694004049D390002630E0940190002636
:200BE0002FE094004038784EE6FE08E6FF2401FDE43EFC120018D912001541784F74022635
:200C0000F618E436F618E6161870011690002630E024FEF09000262FE034FFF080AB784D53
:200C2000E69000261CF0E61846700890002620F00109F99000262FE07004A3E064017026D0
:200C4000784E0806E6188606700106147B012448F974203EFA1200003B90002621F0E49076
:200C600000262FF0A3F090002614E0FFA3E09000261DCFF0A3EFF00109F922900070FFE058
:200C8000784AF67E087FD0E6540FFD7C0012000E721200113C7E087FF0E4FDFC12000E72B0
:200CA000E4784AF6784AE6FDC39403501E7E087FF874042DF582E43420F583759300E0FD7D
:200CC0007C0012000E72784A0680D97E087FFC90002007E0FD7C0012000E727E097F00E458
:200CE000FDFC12000E72E4784AF6784AE6FDC39405501E7E097F0974122DF582E43420F5F8
:200D000083759300E0FD7C0012000E72784A0680D97E097F0D90002017E0FD7C0012000EE9
:200D2000727B017A2079181200033E90002608EEF0A3EFF0D39424EE940040E59000202621
:200D4000E0B4081FA3E0B4061A90002609E024F0F090002608E034FFF0120006C5784AA6D8
:200D60000780BE90002026E0B408B6A3E0B400B19000202AE0FFA3E090002608CFF0A3EFD3
:200D8000F090002034E0FCA3E0FDA3E0FEA3E0FF900020001200017BE4784AF6784AE6FF9F
:200DA0007C007B012420F9EC3420FA1200003BFE740C2FF582E43420F583759300EEF006B7
:200DC000E6B406D890002028E064456003010D219000202EE0543F6003010D2190002031E4
:200DE000E0B4010E120006A4E490002608F0A3F0805190002031E0B411499000203EE07091
:200E000004A3E06445701690002609E024E4F090002608E034FFF012000FDA802690002073
:200E20003EE064FC7004A3E064036003010D2190002609E024E4F090002608E034FFF012DA
:200E400000164D9000264DE07003010D2112001E169000200A741FF0A374FCF07E097F110D
:200E6000FD7C1F12000E72C2A9C2AF120007A4010D2190002638EEF0A3EFF0A3ECF0A3ED23
:200E8000F090002638E475F001120000BB85F082F583759300E4939000263DF07003010F09
:200EA000D9E064256003010FBA9000263C740AF090002638E475F001120000BB85F082F572
:200EC00083759300E49324DB7003010FBA800090002639E024FFF090002638E034FFF090F1
:200EE000002638E475F001120000BB85F082F583759300E4939000263DF0E0249D60142473
:200F0000EE601924FD6003010FBA9000263C7410F080099000263BE0FF010FD29000263E87
:200F2000740AF09000263AE07002A3E0605A9000263CE0FBFD7C009000263AE0FEA3E0FF2E
:200F400012000065AA059000263AE0FEA3E0FFEBFD7C00120000659000263AEEF0A3EFF0F0
:200F6000D3EA64809489EA40052457FF80032430FF9000263EE014F0244EF582E43426F540
:200F800083759300EFF0809B9000263EE0B40A047F30803E9000263EE0C3940A4003010E42
:200FA00081E0FF04F0744E2FF582E43426F583759300E0FF12001E2880DA9000263DE0FF54
:200FC00012001E289000263DE0640A6003010E817F0D12001E28010E812290002044E0FE1D
:200FE000A3E0FFEE600301113BEF24FD606404600301113B12001C509000203CE0FFA3E07D
:2010000090002643CFF0A3EFF09000203EE0FEA3E0FF90002641EEF0A3EFF090002044E419
:20102000F0A37404F0E4A3F0A3F09000203CEEF0A3EFF090002643E0FFA3E09000203ECF47
:20104000F0A3EFF090002608E4F0A37404F0020012949000203EE0FEA3E0FF90002641E0B4
:201060006E7003A3E06F60030111339000263FE0FEA3E0FF90002046E0B50608A3E0B507C8
:201080000301112F90002640E02401FF9000263FE03400FE90002046E06E7003A3E06F6002
:2010A000030111339000203CE0FFA3E090002643CFF0A3EFF07E097F9CE4FDFC12000E724F
:2010C000C390002609E09404FF90002608E09400FE120009EA9000262EE0702B90002617B6
:2010E000E0C3941450067E097F9E80047E097FB4E4FDFC12000E727F047E0012001BE4905C
:2011000000264D7401F02290002640E004F070079000263FE004F0C390002609E094049041
:20112000002608E0940250079000264D7401F002001D72E490002608F0A3F022D2A9D2AF78
:20114000E49000262FF0A3F09000262FE0FEA3E0FFC39402EE9400505BEF2404FFE43EFE42
:2011600012001A7D90002631EEF0A3EFF0E0FD90002630E025E0FB9000262FE033FA740472
:201180002BF58274203AF583759300EDF090002631E0FF74052BF58274203AF58375930053
:2011A000EFF090002630E004F0709D9000262FE004F08094E49000262FF0A3F09000262F8B
:2011C000E0FEA3E0FFC39403EE9400505412001A7D90002631EEF0A3EFF0E0FD900026307C
:2011E000E025E0FB9000262FE033FA74122BF58274203AF583759300EDF090002631E0FF04
:2012000074132BF58274203AF583759300EFF090002630E004F070A49000262FE004F08071
:201220009BE4784BF6784BE6FF2404F582E43420F583759300E0FEEF2466FDE434708D828C
:20124000F583759300EEF006E6B404D9E4784BF6784BE6FF2412F582E43420F58375930009
:20126000E0FEEF2460FDE434708D82F583759300EEF006E6B406D99000706CE054FDF0908F
:20128000007001743FF0900070007410F0900070DAE4F02290002609E02408FE900026086F
:2012A000E0340090002040F0A3CEF0E4A3F0A3F090002000E0FCA3E0FDA3E0FEA3E0FF9030
:2012C0000020381200017B90002004E0FCA3E0FDA3E0FEA3E0FF900020341200017B900013
:2012E0002609E0241CF090002608E03400F0900020287445F0E4A3F09000202E7440F0E48F
:20130000A3F0A37410F0A304F090002608E0FFA3E09000202ACFF0A3EFF090002009E004B4
:20132000F0700790002008E004F090002008E09000202CF090002009E09000202DF0E4907C
:20134000002032F0A3F0900020187490F090002609E02412F090002608E03400F0C3A3E02F
:20136000944090002608E094005006E4F0A37440F090002018E054F8FE90002608E04EFF19
:20138000A3E090002018CFF0A3EFF0E4FF740C2FF582E43420F583759300E0FEEF7C007B3C
:2013A00001241AF9EC3420FAEE120000510FEFB406DBE4FF74122FF582E43420F583759310
:2013C00000E0FE74202FF582E43420F583759300EEF00FEFB406DD900020267408F0A3E401
:2013E000F07B017A207918020003AAE4FFFEFDFC9000262F1200017BE490002633F07E0916
:201400007F64FDFC12000E727E097F69E4FDFC12000E727FFC7EFF7D0F7C00900026341284
:2014200000017B9000262FE0F8A3E0F9A3E0FAA3E0FBC000C001C002C003A3E0FFE4FDFE95
:20144000A3A3E0F9A3E0FAA3E02FFFEE3AFEED39FDE42FFFE43EFEED3481FDA907AA06AB1A
:20146000051200003BFFD003D002D001D000EB4FFFEAFEE9FDE8FC9000262F1200017B90E7
:2014800000262FE0FCA3E0FDA3E0FEA3E0FF78081200014D9000262F1200017B900026335C
:2014A000E004F0E0C3940350030114239000262FE0F8A3E0F9A3E0FAA3E0FBC000C001C01E
:2014C00002C003A3E0FFE4FDFEA3A3E0F9A3E0FAA3E02FFFEE3AFEED39FDE42FFFE43EFE1E
:2014E000ED3481FDA907AA06AB051200003BFFD003D002D001D000EB4FFFEAFEE9FDE8FCC0
:201500009000262F1200017B7F557EAA7D557CAA9000262FE0F8A3E0F9A3E0FAA3E0FBC36D
:201520001200013C700D7E097F7FFDFC12000E727F01227E097F84E4FDFC12000E727F00B5
:201540002290002618EEF0A3EFF090002614E475F001120000BBAFF090002631F0A3EFF062
:2015600090002619E0FF9000262CF090002046E07004A3E0640160030115FC90002631E07D
:20158000FCA3E0FDC39427EC9400403CD3ED943AEC9400503390002617E004F08D828C8305
:2015A000759300E4936F6006E49000262DF090002617E0B414129000262DE07004A3F0804F
:2015C000079000262E7401F090002616E0702DA3E0641470279000262EE06020E4F52F1282
:2015E0000005971200173912001810EF70069000262EF022900026167401F022900026311E
:20160000E0FEA3E04E7002052F9000262EE06401703A90002616E0640170319000262CE02E
:20162000FDF46028E52F7011C3EE9440401E90002631E0FEA3E0FF800F90002631E0FEA37B
:20164000E0FF9000262CE0FD12001B76227FE07E5A7D947C0190002054E0F8A3E0F9A3E087
:20166000FAA3E0FBC31200013C600301173890002046E0FEA3E0FF64014E6007EF4E60031D
:20168000011738E490002052F0A3F090002050E0FEA3E0FFEE6003011738EF24FB600B24F3
:2016A000FB600924096003011738802D78127C207D017B017A2079487E007F06120002297E
:2016C000EF707590002608E4F0A37428F090002050E4F0A3740BF0800E12001CA390002080
:2016E00050E4F0A3740CF078487C207D017B017A2079127E007F06120002BC90002044E48D
:20170000F0A37402F0A3E4F0A304F09000204EE4F0A304F09000203EE0FEA3E0FF9000205B
:201720003CE0FDA3E0A3CDF0A3EDF09000203CEEF0A3EFF012001294227E077FF6E4FDFC30
:2017400012000E727E087F15E4FDFC12000E72E4F52FF523752408AE23AF24E4FCFDFB7AB7
:2017600010F9F8120000ED8F288E278D268C25A2AFE433F522C2AF4387049000555574AA83
:20178000F090002AAA7455F0900055557480F074AAF090002AAA7455F0E47FFF7EFFFDFC1B
:2017A000AB28AA27A926A825D31200013C401BE42528FFE43527FEE5263401FDA907AA0661
:2017C000AB05743012000051800C8528828527837593007430F05387FBE52224FF92AFAEDE
:2017E00023AF24E4FCFDFB7A10F9F8120000ED120019FB0524E52470020523C3E52394014F
:2018000050030117577E087F4BE4FDFC02000E727E077FB6E4FDFC12000E72E4752502F5B9
:2018200024F523F522E47F3FFEFDFCAB25AA24A923A822D31200013C40030118C3E4F52648
:20184000F527E4FF7E40FDFCAB25AA24A923A822120000ED8F2B8E2A8D298C28E4FCFDE501
:201860002B2527F52BE52A3526F52AED3529F529EC3528F528E4252BFFE4352AFEE52934C3
:2018800081FDA907AA06AB051200003BF4600D7E077FE2E4FD12000E727F00220527E527DA
:2018A00070020526C3E52694404097E5252401F525E43524F524E43523F523E43522F522CD
:2018C0000118257E077FEDE4FDFC12000E727F01227D087F077C007E0090002631ECF0A35D
:2018E000EDF0E4A3F0A3F0AD07AC06C390002632E09D90002631E09C40629000261AE0FEC0
:20190000A3E08E837593002DF582E5833CF583759300E0F990002634E0C4F8540FC868F081
:2019200090002633E0C454F048F0E9D39439500BE9C39430FFE49400FE8013C3E99441FFC2
:20194000E49400CF240ACF3400FE90002633E04EF0A3E04FF00DBD00010C808F9000263379
:20196000E0FEA3E0FF2290002635EEF0A3EFF09000265C7408F0F5C84402F0F5C87F327E3D
:201980000012001E159000265CE04404F0F5C87F647E0012001E1512001E079000265A74BA
:2019A00008F0A3E4F09000265AE0FCA3E0FD4C6043A3E054FAF090002635E0FEA3E0FFEC65
:2019C0005EFEED5F4E60089000265CE04404F09000265CE012001E0F12001E119000265CFB
:2019E000E04401F0F5C89000265AE0C313F0A3E013F080B19000265CE0FF22900026361297
:201A000000017B752901E4F52CF52D90002636A3E0FDA3E0FEA3E02400FFE43EFEED34812F
:201A2000FDA907AA06AB051200003BF52A532A40E529604090002636A3E0FDA3E0FEA3E052
:201A40002400FFE43EFEED3481FDA907AA06AB051200003BF52B532B40E52AB52B03E4F59E
:201A600029852B2A052DE52D7002052CB4FFC1E52CB4FFBCE5297F0060027F0122C2AFEE98
:201A80004408FE120019669000265CEFF0E490002633F0A3F09000265A7480F0A3E4F0902F
:201AA00000265AE07002A3E060379000265CE054FA12001E0E12001E07AFC8EF30E3149068
:201AC00000265AE0FEA3E0FF90002633E04EF0A3E04FF09000265AE0C313F0A3E013F080A1
:201AE000BE9000265CE054F8F0F5C87F907E0112001E15D2AF90002633E0FEA3E0FF2290EE
:201B000000262FEBF0A3EAF0A3E9F0E490002637F0A3F09000263574FFF5F0120000BB45F3
:201B2000F0604690002632E0FBA3E0FAA3E0F91200003BFF9000262FE0FBA3E0FAA3E0F94E
:201B400090002637E475F001120000BBFCE925F0F9EA3CFAEF1200005160B890002633E437
:201B600075F0011200031C80AA9000262FE0FBA3E0FAA3E0F92290002633EEF0A3EFF0A3DD
:201B8000EDF0AF2FE4FCFDFEFBFA7901F8120000ED8F268E258D248C2390002633E0FEA317
:201BA000E0FFE4FCFDE5262FF526E5253EF525ED3524F524EC3523F523A3E0F52EA2AFE41C
:201BC00033F522C2AFAF26AE25AD24AC23120009C5AF26AE25AD24AC23120019FBE5222489
:201BE000FF92AF22900070007429F090002044E4F0A37405F0A3EEF0A3EFF064044E7020D9
:201C0000900026327481F0A37409F0A3748BF0A3E4F0A37411F07B017A20794812001AFFC4
:201C200090002641E0FFA3E09000203CCFF0A3EFF090002643E0FFA3E09000203ECFF0A373
:201C4000EFF090002608E4F0A37415F002001294E49000263FF0A3F090002000E0FCA3E0E4
:201C6000FDA3E0FEA3E0FF900026451200017BE490002641F0A3F0A3F0A3F09000264DF064
:201C80009000262EF090002617F090002616F09000262D04F0900070007421F0900070DAC1
:201CA000E4F0227B017A20796CE475F004120000D1740229F9E43AFAE475F008120000D11F
:201CC000740229F9E43AFA90002004E0FCA3E0FDA3E0FEA3E0FF12000160740429F9E43A16
:201CE000FEC3E99444FFEE942090002608F0A3EFF0229000262FEEF0A3EFF0E4F523D3ED6E
:201D00009400EC9400402C9000262FE0FEA3E0AA06F97B811200003B2523F523ED1D700130
:201D20001C90002630E004F070D49000262FE004F080CBAF23227E097F34E4FDFC12000E5A
:201D400072E4F522FD7C80FF7E8012001CF28F22E522B4FF0E7E097F46FD7C0012000E7230
:201D60007F01227E097F54AD227C0012000E727F002290002044E4F0A37404F0900026411F
:201D8000E0FFA3E09000203CCFF0A3EFF090002643E0FFA3E09000203ECFF0A3EFF090009A
:201DA0002608E4F0A37404F002001294C0D0C2A9C2AFE5492401F549E43548F548E4354773
:201DC000F547E43546F546758C5D758A3DD2AFD2A9D0D022E58954F04401F589758C5D758D
:201DE0008A3DE4F549F548F547F546D2B9D28C227598504387805389CF438920758DF37593
:201E00008CF3D28ED299229000265CE04401F0F5C87FF47E01229000706CE054E7F022AF16
:201E200049AE48AD47AC46223099FDC2998F9922FFFFFFFFFFFFFFFFFFFFFFFFFFFFFFFF00
:201E4000FFFFFFFFFFFFFFFFFFFFFFFFFFFFFFFFFFFFFFFFFFFFFFFFFFFFFFFFFFFFFFFFA2
:201E6000FFFFFFFFFFFFFFFFFFFFFFFFFFFFFFFFFFFFFFFFFFFFFFFFFFFFFFFFFFFFFFFF82
:201E8000FFFFFFFFFFFFFFFFFFFFFFFFFFFFFFFFFFFFFFFFFFFFFFFFFFFFFFFFFFFFFFFF62
:201EA000FFFFFFFFFFFFFFFFFFFFFFFFFFFFFFFFFFFFFFFFFFFFFFFFFFFFFFFFFFFFFFFF42
:201EC000FFFFFFFFFFFFFFFFFFFFFFFFFFFFFFFFFFFFFFFFFFFFFFFFFFFFFFFFFFFFFFFF22
:201EE000FFFFFFFFFFFFFFFFFFFFFFFFFFFFFFFFFFFFFFFFFFFFFFFFFFFFFFFFFFFFFFFF02
:201F0000FFFFFFFFFFFFFFFFFFFFFFFFFFFFFFFFFFFFFFFFFFFFFFFFFFFFFFFFFFFFFFFFE1
:201F2000FFFFFFFFFFFFFFFFFFFFFFFFFFFFFFFFFFFFFFFFFFFFFFFFFFFFFFFFFFFFFFFFC1
:201F4000FFFFFFFFFFFFFFFFFFFFFFFFFFFFFFFFFFFFFFFFFFFFFFFFFFFFFFFFFFFFFFFFA1
:201F6000FFFFFFFFFFFFFFFFFFFFFFFFFFFFFFFFFFFFFFFFFFFFFFFFFFFFFFFFFFFFFFFF81
:201F8000FFFFFFFFFFFFFFFFFFFFFFFFFFFFFFFFFFFFFFFFFFFFFFFFFFFFFFFFFFFFFFFF61
:201FA00075C7AA75C755759D02787FE4F6D8FD900000007F007E607D01E4F0A3DFFCDEFA5B
:201FC000DDF875814F12000517C20D120004B41200040A12001DD412001DF0C20D120004F9
:201FE000AB02000C7BFFFFFFFFFFFFFFFFFFFFFFFFFFFFFFFFFFFFFFFFFFFFFF0200085466
:20200000020020C0C5F0F8A3E028F0C5F0F8E582158270021583E038F022EB9FF5F0EA9EC0
:2020200042F0E99D42F0E89C45F022E8600FECC313FCED13FDEE13FEEF13FFD8F122E86096
:202040000FEFC333FFEE33FEED33FDEC33FCD8F122BB0006E9F8020020B4BB8000500C89B3
:20206000828A838B9315930200206C22ECF0A3EDF0A3EEF0A3EFF022D093D083D082E4935B
:202080007012740193700DA3A393F8740193F5828883E4737402936C70127403936D700C9D
:2020A0007404936E70067405936F60DDA3A3A3A3A3A380CAECF608EDF608EEF608EFF62295
:2020C00002002FF6E490002005F0A3F0E0FF12003492E490002004F090002004E0FF04F0F7
:2020E000EFC3940A5069E47F807E80FDFC9000200F1200206C90002006E0FFC00790002094
:202100000FE0FCA3E0FDA3E0FEA3E0FF900020161200206CD0077D147C00120032D790005E
:202120002006E0FF7B017A20790F7D147C00120033E5E47F807E80FDFC9000200FE0F8A3B1
:20214000E0F9A3E0FAA3E0FBC31200201A708990002004E0B40A0280FEE47F81FEFDFC9066
:2021600000200F1200206C90002006E0FFC0079000200FE0FCA3E0FDA3E0FEA3E0FF900088
:2021800020161200206CD0077D177C00120032D7E4FF7E04FDFC9000200F1200206C90001E
:2021A0002006E0FFC0079000200FE0FCA3E0FDA3E0FEA3E0FF900020161200206CD0077D7D
:2021C000187C00120032D7E490002004F090002004E0FF245AF582E43420F583759300E0A8
:2021E000FE74092FF582E43420F583759300EEF090002004E004F0E0B406D2E4900020049C
:20220000F090002004E0FBC39403506DE0FD25E02409F582E43420F583759300E0FEED25FA
:20222000E0240AF582E43420F583759300E0FDEDFFE4FCFD9000200F1200206C90002006A8
:20224000E0FFC007EB2419FDE433FCC004C0059000200FE0FCA3E0FDA3E0FEA3E0FF900069
:2022600020161200206CD005D004D007120032D790002004E004F08088E47F747E88FDFC89
:202280009000200F1200206C90002006E0FFC0079000200FE0FCA3E0FDA3E0FEA3E0FF90D7
:2022A0000020161200206CD0077D1C7C00120032D7E47F807E19FDFC9000200F1200206C73
:2022C00090002006E0FFC0079000200FE0FCA3E0FDA3E0FEA3E0FF900020161200206CD050
:2022E000077D1D7C00120032D7E47F2C7E01FDFC9000200F1200206C90002006E0FFC007E6
:202300009000200FE0FCA3E0FDA3E0FEA3E0FF900020161200206CD0077D1E7C0012003209
:20232000D7E4FFFEFDFC9000200F1200206C90002006E0FFC0079000200FE0FCA3E0FDA375
:20234000E0FEA3E0FF900020161200206CD0077D267C00120032D7E47FFF7EFFFDFC900040
:20236000200F1200206CE490002004F090002004E0FEC39424503D90002006E0FFC007EE24
:202380002427FDE433FCC004C0059000200FE0FCA3E0FDA3E0FEA3E0FF9000201612002043
:2023A0006CD005D004D007120032D790002004E004F080B8E47FFFFEFDFC9000200F12002C
:2023C000206C90002006E0FFC0079000200FE0FCA3E0FDA3E0FEA3E0FF90002016120020FF
:2023E0006CD0077D4B7C00120032D7E47FFF7EFFFDFC9000200F1200206C90002006E0FF71
:20240000C0079000200FE0FCA3E0FDA3E0FEA3E0FF900020161200206CD0077D4C7C001245
:202420000032D7E47FFF7E01FDFC9000200F1200206C90002006E0FFC0079000200FE0FC65
:20244000A3E0FDA3E0FEA3E0FF900020161200206CD0077D4D7C00120032D7E47FFF7EFF7E
:20246000FDFC9000200F1200206C90002006E0FFC0079000200FE0FCA3E0FDA3E0FEA3E08B
:20248000FF900020161200206CD0077D4E7C00120032D7E47FA07EC0FDFC9000200F120095
:2024A000206C90002006E0FFC0079000200FE0FCA3E0FDA3E0FEA3E0FF900020161200201E
:2024C0006CD0077D687C00120032D7E47F417EFAFDFC9000200F1200206CE490002004F043
:2024E00090002004E0FEC39402503D90002006E0FFC007EE2469FDE433FCC004C005900064
:20250000200FE0FCA3E0FDA3E0FEA3E0FF900020161200206CD005D004D007120032D7909E
:20252000002004E004F080B8E47F417EFAFDFC9000200F1200206CE490002004F0900020C1
:2025400004E0FEC39402503D90002006E0FFC007EE246BFDE433FCC004C0059000200FE0A2
:20256000FCA3E0FDA3E0FEA3E0FF900020161200206CD005D004D007120032D79000200429
:20258000E004F080B8E47F107E20FDFC9000200F1200206C90002006E0FFC0079000200FAD
:2025A000E0FCA3E0FDA3E0FEA3E0FF900020161200206CD0077D6D7C00120032D7E47F0499
:2025C0007E08FDFC9000200F1200206C90002006E0FFC0079000200FE0FCA3E0FDA3E0FE27
:2025E000A3E0FF900020161200206CD0077D6E7C00120032D7E47F107E20FDFC9000200FD3
:202600001200206C90002006E0FFC0079000200FE0FCA3E0FDA3E0FEA3E0FF9000201612CA
:2026200000206CD0077D6F7C00120032D7E47F047E08FDFC9000200F1200206C90002006BB
:20264000E0FFC0079000200FE0FCA3E0FDA3E0FEA3E0FF900020161200206CD0077D707C12
:2026600000120032D7E490002004F090002004E0FBC39404400301271DE47FFF7E01FDFC6B
:202680009000200F1200206CEB75F002A42471FDE435F0FCC004C00590002006E0FFC0076B
:2026A0009000200FE0FCA3E0FDA3E0FEA3E0FF900020161200206CD007D005D004120032D4
:2026C000D7E47FFF7EFFFDFC9000200F1200206C90002004E075F002A42471FFE435F0CFE3
:2026E0002401FDE43FFCC004C00590002006E0FFC0079000200FE0FCA3E0FDA3E0FEA3E095
:20270000FF900020161200206CD007D005D004120032D790002004E004F001266BE47F0836
:202720007E08FDFC9000200F1200206C90002006E0FFC0079000200FE0FCA3E0FDA3E0FEC5
:20274000A3E0FF900020161200206CD0077D797C00120032D7E47F1E7E14FDFC9000200F64
:202760001200206C90002006E0FFC0079000200FE0FCA3E0FDA3E0FEA3E0FF900020161269
:2027800000206CD0077D7A7C00120032D7E4FFFEFDFC9000200F1200206C90002006E0FF7C
:2027A000C0079000200FE0FCA3E0FDA3E0FEA3E0FF900020161200206CD0077D7B7C001273
:2027C0000032D7E47F207E40FDFC9000200F1200206C90002006E0FFC0079000200FE0FC62
:2027E000A3E0FDA3E0FEA3E0FF900020161200206CD0077D817C00120032D7E47F507EFA5B
:20280000FDFC9000200F1200206C90002006E0FFC0079000200FE0FCA3E0FDA3E0FEA3E0E7
:20282000FF900020161200206CD0077D827C00120032D7E4FF7E40FDFC9000200F1200203D
:202840006C90002006E0FFC0079000200FE0FCA3E0FDA3E0FEA3E0FF900020161200206C2E
:20286000D0077D8C7C00120032D7E47F11FEFDFC9000200F1200206C90002006E0FFC007BD
:202880009000200FE0FCA3E0FDA3E0FEA3E0FF900020161200206CD0077D957C001200320D
:2028A000D7E47F337E22FDFC9000200F1200206C90002006E0FFC0079000200FE0FCA3E03B
:2028C000FDA3E0FEA3E0FF900020161200206CD0077D967C00120032D7E47F557E44FDFCA0
:2028E0009000200F1200206C90002006E0FFC0079000200FE0FCA3E0FDA3E0FEA3E0FF9071
:202900000020161200206CD0077D977C00120032D7E490002007F0A3F090002007E0FAA30F
:20292000E0FBC39419EA648094804003012BF9E47F837E04FDFC9000200F1200206C9000B4
:202940002006E0FFC007EBAE027803C333CE33CED8F92400FDEE3401FCC004C00590002086
:202960000FE0FCA3E0FDA3E0FEA3E0FF900020161200206CD005D004D007120032D790005A
:202980002007E0FAA3E0FB64184A6003012A547F817E16FDFC9000200F1200206C90002076
:2029A00006E0FFC007EBAE027803C333CE33CED8F92402FDEE3401FCC004C0059000200F35
:2029C000E0FCA3E0FDA3E0FEA3E0FF900020161200206CD005D004D007120032D7E47F80B6
:2029E0007E36FDFC9000200F1200206C90002006E0FFC007A3E0FEA3E07803C333CE33CE2D
:202A0000D8F92401FDEE3401FCC004C0059000200FE0FCA3E0FDA3E0FEA3E0FF9000201637
:202A20001200206CD005D004D007120032D7E4FFFEFDFC9000200F1200206C90002006E090
:202A4000FFC007A3E0FEA3E07803C333CE33CED8F9012B1AE47FF17E17FDFC9000200F12A2
:202A600000206C90002006E0FFC007A3E0FEA3E07803C333CE33CED8F92402FDEE3401FC17
:202A8000C004C0059000200FE0FCA3E0FDA3E0FEA3E0FF900020161200206CD005D004D0B2
:202AA00007120032D7E47F807ED6FDFC9000200F1200206C90002006E0FFC007A3E0FEA3E7
:202AC000E07803C333CE33CED8F92401FDEE3401FCC004C0059000200FE0FCA3E0FDA3E09D
:202AE000FEA3E0FF900020161200206CD005D004D007120032D7E47F01FEFDFC9000200F3D
:202B00001200206C90002006E0FFC007A3E0FEA3E07803C333CE33CED8F92403FDEE34015F
:202B2000FCC004C0059000200FE0FCA3E0FDA3E0FEA3E0FF900020161200206CD005D004E5
:202B4000D007120032D7E4FFFEFDFC9000200F1200206C90002006E0FFC007A3E0FEA3E0EC
:202B60007803C333CE33CED8F92404FDEE3401FCC004C0059000200FE0FCA3E0FDA3E0FEDB
:202B8000A3E0FF900020161200206CD005D004D007120032D7E47F017E10FDFC9000200F0A
:202BA0001200206C90002006E0FFC007A3E0FEA3E07803C333CE33CED8F92405FDEE3401BD
:202BC000FCC004C0059000200FE0FCA3E0FDA3E0FEA3E0FF900020161200206CD005D00445
:202BE000D007120032D790002008E004F0700790002007E004F0012919229000201EEFF043
:202C00007B017A2079427D107C0012002EEB90002042A3A3A3E05480FFEF60037F0022909E
:202C200000201FA3A3A3E05407FFE4FEFDFC120020782C91000000012C420000000500007C
:202C40002C8E9000204EE0FCA3E0FDA3E0FEA3E0FF9000202D1200206C9000201EE0FF7DB8
:202C6000037C001200339E9000204AE0FCA3E0FDA3E0FEA3E0FF9000202D1200206C90008E
:202C8000201EE0FF7D027C001200339E80037F002290002023E0FCA3E0FDA3E0FEA3E0FFE3
:202CA0009000202D1200206C9000201EE0FF7D017C001200339E9000201FE0FCA3E0FDA341
:202CC000E0FEA3E0FF9000202D1200206C9000201EE0FFE4FDFC1200339E9000201EE0FFFF
:202CE0007B017A2079427D107C0012002EEB90002042A3A3A3E05480FFEF70DE9000201F35
:202D0000A3A3A3E05478FFE4FEFDFC78031200202B120020782D43000000002D57000000CE
:202D2000012D6B000000032D6B000000042D6B000000052D6B000000062D6B000000070081
:202D4000002D819000201EE0FF7B017A2079527D047C0012002EEB9000201EE0FF7B017A6C
:202D600020794E7D037C0012002EEB9000201EE0FF7B017A20794A7D027C0012002EEB8019
:202D8000037F00227F012290002021EFF07B017A2079427D107C0012002EEB90002042A3A3
:202DA000A3A3E05480FFEF60037F002290002022A3A3A3E05407FFE4FEFDFC120020782D80
:202DC000D8000000022DD8000000042DD80000000600002DD57F002290002022A3A3A3E0C7
:202DE0005478FFE4FEFDFC78031200202B120020782E19000000002E36000000012E53007E
:202E00000000032E53000000042E53000000062E530000000700002E7A90002052E0FCA3F2
:202E2000E0FDA3E0FEA3E0FF9000202D1200206C7D04120033969000204EE0FCA3E0FDA3DE
:202E4000E0FEA3E0FF9000202D1200206C7D03120033969000204AE0FCA3E0FDA3E0FEA3C2
:202E6000E0FF9000202D1200206C90002021E0FF7D027C001200339E80037F002290002096
:202E800026E0FCA3E0FDA3E0FEA3E0FF9000202D1200206C90002021E0FF7D017C00120076
:202EA000339E90002022E0FCA3E0FDA3E0FEA3E0FF9000202D1200206C90002021E0FFE401
:202EC000FDFC1200339E90002021E0FF7B017A2079427D107C0012002EEB90002042A3A329
:202EE000A3E05480FFEF70DE7F01229000202AEFF0A3ECF0A3EDF0A3EBF0A3EAF0A3E9F06E
:202F0000E4A3F0A3F0E4FFFEFDFC9000203E1200206C9000202BE0FCA3E0FD9000202AE050
:202F2000FF120031F29000202AE0FFE4FD1200348CE0FF0D120034DFE0FF120032CAE0FF14
:202F4000E4FD120034DFE4FFFEFC900020371200206CE490002032F0120034AC12003267B6
:202F600090002032E004F0E0C3942040EB90002037E0FCA3E0FDA3E0FEA3E0FF9000202DF6
:202F8000E0FBA3E0FAA3E0F912002051E4FFFEFDFC900020371200206CE490002032F012B3
:202FA0000034AC1200326790002032E004F0E0C3940940EB90002037A3A3E0FEA3E0FBEEEE
:202FC000FAE4F9F89000202BE0FEA3E0FFE4FCFDC31200201A601E90002030E475F0011241
:202FE000002004FED3741E95F0EE6480F87480984003012F0522E490002000F0A3F090002E
:203000002000E0FEA3E0FFC39402EE9400505BEF2404FFE43EFE1200317090002002EEF031
:20302000A3EFF0E0FD90002001E025E0FB90002000E033FA74562BF58274203AF583759329
:2030400000EDF090002002E0FF74572BF58274203AF583759300EFF090002001E004F07073
:203060009D90002000E004F08094E490002000F0A3F090002000E0FEA3E0FFC39403EE9418
:203080000050541200317090002002EEF0A3EFF0E0FD90002001E025E0FB90002000E03396
:2030A000FA745A2BF58274203AF583759300EDF090002002E0FF745B2BF58274203AF58333
:2030C000759300EFF090002001E004F070A490002000E004F0809B020020C490002006EE47
:2030E000F0A3EFF0900020647408F0F5C84402F0F5C87F327E00120034D290002064E044AF
:2031000004F0F5C87F647E00120034D2120034C4900020627408F0A3E4F090002062E0FC98
:20312000A3E0FD4C6043A3E054FAF090002006E0FEA3E0FFEC5EFEED5F4E600890002064EB
:20314000E04404F090002064E0120034CC120034CE90002064E04401F0F5C890002062E065
:20316000C313F0A3E013F080B190002064E0FF22C2AFEE4408FE120030DB90002064EFF004
:20318000E490002004F0A3F0900020627480F0A3E4F090002062E07002A3E0603790002079
:2031A00064E054FA120034CB120034C4AFC8EF30E31490002062E0FEA3E0FF90002004E0CF
:2031C0004EF0A3E04FF090002062E0C313F0A3E013F080BE90002064E054F8F0F5C87F9077
:2031E0007E01120034D2D2AF90002004E0FEA3E0FF229000203CECF0A3EDF0AB07E4FA1297
:20320000003477120032CA9000203EE0FCA3E0FDA3E0FEA3E0FF78011200202B9000203EE4
:203220001200206C0AEAB420D69000203CE0FEA3E0FFE4FCFDA31200206CE4FA120034774D
:20324000120032CA9000203EE0FCA3E0FDA3E0FEA3E0FF78011200202B9000203E1200201D
:203260006C0AEAB409D622E4FCFDFE900020331200206C90002033E0FCA3E0FDA3E0FEA37A
:20328000E0FF90002032E0F9F81200203EA31200206C90002037E0FCA3E0FDA3E0FEA3E0A4
:2032A000FF90002033E0F8A3E0F9A3E0FAA3E0FBEF4BFFEE4AFEED49FDEC48FC9000203724
:2032C0001200206C9000202AE0FFAE077D01120034D91D020034D990002013EFF0A3ECF0F8
:2032E000A3EDF0C3EC94015027A3E0FCA3E0FDA3E0FEA3E0FF9000202D1200206C90002066
:2033000014E0FCA3E0FD90002013E0FF0200339E90002016E0FCA3E0FDA3E0FEA3E0FF9013
:2033200000201D1200206C90002014E0FCA3E0FD90002013E0FF120034332290002019ECA0
:20334000F0A3EDF0A3EBF0A3EAF0A3E9F0C007E47F21FEFDFC9000201F1200206C90002027
:2033600019E0FEA3E0FFE4FCFD900020231200206CD00712002BFA9000204AE0FCA3E0FD22
:20338000A3E0FEA3E0FF9000201BE0FBA3E0FAA3E0F90200205190002021E0FF7C0090005C
:2033A000202AEFF0C007C004C0059000202DE0FCA3E0FDA3E0FEA3E0FF9000203E12002038
:2033C0006CD005D004D007120031F29000202AE0FFE4FD1200348CE0FF0D120034E5E0FF6A
:2033E0001D020034E590002013EFF090002016EBF0A3EAF0A3E9F090002014ECF0A3EDF039
:20340000C3EC940190002013E0FF5013A3E0FCA3E0FDA3E0FBA3E0FAA3E0F902002EEBA32F
:20342000E0FCA3E0FDA3E0FBA3E0FAA3E0F91200333B22AB05AA04A9079000201DE0FCA3BD
:20344000E0FDA3E0FEA3E0FF9000204A1200206CAF01C007E47F22FEFDFC9000202212001D
:20346000206CAE02AF03E4FCFD900020261200206CD00702002D879000203EE0FCA3A3E090
:20348000FEA3E05401FFA907AF03AD01ED24FF929122AE07E4FD1200348C0D120034D31D47
:2034A000120034D9120034DF020034E59000202AE0FFA290E4339000203BF09000203BE005
:2034C0005401FF2290002064E04401F0F5C87FF47E0122ED24FF929022ED24FF929222EDE5
:2034E00024FF929522ED24FF929322FFFFFFFFFFFFFFFFFFFFFFFFFFFFFFFFFFFFFFFFFF1E
:20350000FFFFFFFFFFFFFFFFFFFFFFFFFFFFFFFFFFFFFFFFFFFFFFFFFFFFFFFFFFFFFFFFCB
:20352000FFFFFFFFFFFFFFFFFFFFFFFFFFFFFFFFFFFFFFFFFFFFFFFFFFFFFFFFFFFFFFFFAB
:20354000FFFFFFFFFFFFFFFFFFFFFFFFFFFFFFFFFFFFFFFFFFFFFFFFFFFFFFFFFFFFFFFF8B
:20356000FFFFFFFFFFFFFFFFFFFFFFFFFFFFFFFFFFFFFFFFFFFFFFFFFFFFFFFFFFFFFFFF6B
:203F0000120020C022FFFFFFFFFFFFFFFFFFFFFFFFFFFFFFFFFFFFFFFFFFFFFFFFFFFFFFA8
:203F2000FFFFFFFFFFFFFFFFFFFFFFFFFFFFFFFFFFFFFFFFFFFFFFFFFFFFFFFFFFFFFFFFA1
:203F4000FFFFFFFFFFFFFFFFFFFFFFFFFFFFFFFFFFFFFFFFFFFFFFFFFFFFFFFFFFFFFFFF81
:203F6000FFFFFFFFFFFFFFFFFFFFFFFFFFFFFFFFFFFFFFFFFFFFFFFFFFFFFFFFFFFFFFFF61
:203F8000FFFFFFFFFFFFFFFFFFFFFFFFFFFFFFFFFFFFFFFFFFFFFFFFFFFFFFFFFFFFFFFF41
:208000000200DBE26D643500257800320202593D020000000202D7783098FDAF99C2987EF8
:20802000002222220200800BEB7008E709F608DFFA801B89828A831410E70AF593E0A3F65A
:2080400008DFFA8009F593E493A3F608DFF9ECFAA9F0EDFB2288F0EF60010E4E60F088F0C9
:20806000ED60C51410E7E7CB700E88828C838B93E709F0A3DFFA80D61410E72A89828A837D
:20808000F593ECFAE0A3C8C582C8CCC583CCCBC593CBF0A3C8C582C8CCC583CCCBC593CB12
:2080A000DFE2DEE080AA89828A83F593ECFAE493A3C8C582C8CCC583CCCBC593CBF0A3C877
:2080C000C582C8CCC583CCCBC593CBDFE1DEDF02008050EB7002E72289828A831410E704E7
:2080E000F593E022F593E49322F8EB7006E7C828F3E82289828A831410E708F593E0C82825
:20810000F0E822F593E49322BB000327F722F8EB89828A831410E706F593E028F022F59310
:20812000E4932822BB0002F722BB8000500989828A838B931593F022EF8DF0A4A8F0CF8C21
:20814000F0A428CE8DF0A42EFE22C2D5EC30E709B2D5E4C39DFDE49CFCEE30E716B2D5E4B9
:20816000C39FFFE49EFE120088D1C3E49DFDE49CFC8004120088D130D507C3E49FFFE49E34
:20818000FE22C5F0F8A3E028F0C5F0F8E582158270021583E038F022A3F8E0C5F025F0F063
:2081A000E582158270021583E0C838F0E822EB7007E7F5F009E7192289828A831410E70859
:2081C000F593E0F5F0A3E022F593E493F5F074019322F8EB700C09E5F027C7F5F019E83757
:2081E000C72289828A831410E707F593E802008198F593E4740193F5F0E49322BB000B0920
:20820000C5F027F7C5F01937F722F8EB89828A831410E707F593E802008182F5937401935B
:2082200025F0F5F0E4933822BB0006F709A7F01922BB8000500D89828A838B931593F0E595
:20824000F0A3F022E88FF0A4CC8BF0A42CFCE98EF0A42CFC8AF0EDA42CFCEA8EF0A4CDA874
:20826000F08BF0A42DCC3825F0FDE98FF0A42CCD35F0FCEB8EF0A4FEA9F0EB8FF0A4CFC540
:20828000F02ECD39FEE43CFCEAA42DCE35F0FDE43CFC2275F008758200EF2FFFEE33FECD4A
:2082A00033CDCC33CCC58233C5829BED9AEC99E58298400CF582EE9BFEED9AFDEC99FC0F2E
:2082C000D5F0D6E4CEFBE4CDFAE4CCF9A88222B800C1B90059BA002DEC8BF084CFCECDFCF3
:2082E000E5F0CBF97818EF2FFFEE33FEED33FDEC33FCEB33FB10D703994004EB99FB0FD89B
:20830000E5E4F9FA227818EF2FFFEE33FEED33FDEC33FCC933C910D7059BE99A4007EC9BDE
:20832000FCE99AF90FD8E0E4C9FAE4CCFB2275F010EF2FFFEE33FEED33FDCC33CCC833C82E
:2083400010D7079BEC9AE899400AED9BFDEC9AFCE899F80FD5F0DAE4CDFBE4CCFAE4C8F91A
:2083600022CFF4CFCEF4CECDF4CDCCF4CC22EB9FF5F0EA9E42F0E99D42F0E89C45F022E8D9
:20838000600FECC313FCED13FDEE13FEEF13FFD8F122E8600FEFC333FFEE33FEED33FDEC65
:2083A00033FCD8F122EB7006E9F80200893589828A831410E706F59302008941F59302009A
:2083C000894DBB0006E9F8020089A6BB8000500C89828A838B9315930200844C22EB70062A
:2083E000E9F80200898F89828A831410E706F59302008420F5930200894DEB7006E9F80287
:2084000000895D89828A831410E706F5930200896AF593020089767401FF3395E0FEFDFC34
:20842000A3A3A3E02FFFF0E582158270021583E03EFEF0E582158270021583E03DFDF0E54A
:2084400082158270021583E03CFCF022ECF0A3EDF0A3EEF0A3EFF022A42582F582E5F03582
:2084600083F58322EB7006E9F8020089B289828A831410E706F593020089C4F59302008A4C
:2084800004BB001CD093D0F0D0E0F8D0E0C9FBD0E0FAD0E0CBC8C0E0C0F0C093020089BBEC
:2084A000BB80005022D093D0F0D0E0F8D0E0C9F582D0E0CAF583D0E0CB14C8C0E0C0F0C0FB
:2084C000938893020089FBD093D083D082D0E0D0E0D0E0E473D093D083D082F8E493701200
:2084E000740193700DA3A393F8740193F5828883E4737402936860EFA3A3A380DFD093D00A
:2085000083D082F8E4937012740193700DA3A393F8740193F5828883E473740293B5F006AA
:208520007403936860E9A3A3A3A380D8D093D083D082E4937012740193700DA3A393F874D1
:208540000193F5828883E4737402936C70127403936D700C7404936E70067405936F60DD1D
:20856000A3A3A3A3A3A380CA8B938A838982159353937FE473EB700C87F009E608B5F0418A
:20858000603F80F489828A831410E70FF593E0F5F0A3E608B5F02A602880F3F593E493F5FA
:2085A000F0A3E608B5F01A601880F2CB701588828C838B9387F009E493A3B5F004600280E5
:2085C000F380611410E72E89828A83F593ECFAE0F5F0A3C8C582C8CCC583CCCBC593CBE417
:2085E00093A3C8C582C8CCC583CCCBC593CBB5F033603180DA89828A83F593ECFAE493F5EB
:20860000F0A3C8C582C8CCC583CCCBC593CBE493A3C8C582C8CCC583CCCBC593CBB5F004BA
:20862000600280D97F00F845F0600EE863F0806480D395F01F40027F01220200857502006D
:2086400085ABED60F51410E7F5CB701488828C83F59387F009E0A3B5F0CA60C880F480C466
:208660001410E72D89828A83F593ECFAE0F5F0A3C8C582C8CCC583CCCBC593CBE0A3C8C51F
:2086800082C8CCC583CCCBC593CBB5F097609580DB89828A83F593ECFAE493F5F0A3C8C524
:2086A00082C8CCC583CCCBC593CBE0A3C8C582C8CCC583CCCBC593CBB5F0A360A180DAEBEC
:2086C0007008E709F60870FA801B89828A831410E70AF593E0A3F60870FA8009F593E49307
:2086E000A3F60870F9ECFAA9F0EDFB2288F0ED60CE1410E7F0CB700E88828C83F593E7097F
:20870000F0A370FA80DF1410E72889828A83F593ECFAE0A3C8C582C8CCC583CCCBC593CB1C
:20872000F0A3C8C582C8CCC583CCCBC593CB70E280B589828A83F593ECFAE493A3C8C582CB
:20874000C8CCC583CCCBC593CBF0A3C8C582C8CCC583CCCBC593CB70E1808CEB700C87F010
:2087600009E608B5F019DFF6801589828A831410E711F593E0F5F0A3E608B5F002DFF5024B
:2087800000880CF593E493F5F0A3E608B5F07DDFF48079CB701388828C838B9387F009E4F9
:2087A00093A3B5F067DFF580631410E73089828A83F593ECFAE0F5F0A3C8C582C8CCC583AC
:2087C000CCCBC593CBE493A3C8C582C8CCC583CCCBC593CBB5F035DFDCDEDA802F89828A8F
:2087E00083F593ECFAE493F5F0A3C8C582C8CCC583CCCBC593CBE493A3C8C582C8CCC583DF
:20880000CCCBC593CBB5F004DFDBDED97FFFB5F0020F2240027F01220200875B020087934A
:2088200088F0EF60010E4E60EEED60EC1410E7ECCB701288828C83F59387F009E0A3B5F000
:20884000CBDFF680C71410E72F89828A83F593ECFAE0F5F0A3C8C582C8CCC583CCCBC5932F
:20886000CBE0A3C8C582C8CCC583CCCBC593CBB5F09ADFDDDEDB809489828A83F593ECFAB7
:20888000E493F5F0A3C8C582C8CCC583CCCBC593CBE0A3C8C582C8CCC583CCCBC593CBB557
:2088A000F004DFDCDEDA0200880CEF4E6022EF60010EEDBB0007F709DFFCA9F022BB80001E
:2088C000500E89828A838B931593F0A3DFFCDEFA22BC000BBE0029EF8DF084FFADF022E4B4
:2088E000CCF875F008EF2FFFEE33FEEC33FCEE9DEC984005FCEE9DFE0FD5F0E9E4CEFD2289
:20890000EDF8F5F0EE008420D21CFEADF075F008EF2FFFED33FD4007985006D5F0F222C3FA
:2089200098FD0FD5F0EA22C3E49FFFE49EFEE49DFDE49CFC22E6FC08E6FD08E6FE08E6FF3B
:2089400022E0FCA3E0FDA3E0FEA3E0FF22E493FC740193FD740293FE740393FF22E6FB08E1
:20896000E6F908E6FA08E6CBF822E0F8A3E0F9A3E0FAA3E0FB22E493F8740193F974029373
:20898000FA740393FB227401FF3395E0FEFDFC080808E62FFFF618E63EFEF618E63DFDF623
:2089A00018E63CFCF622ECF608EDF608EEF608EFF622E6FB08E6FA08E6F922EBF608EAF606
:2089C00008E9F622E0FBA3E0FAA3E0F922F8E0FBA3A3E0F925F0F0E582158270021583E0B9
:2089E000FA38F022F8E0FBA3A3E025F0F9F0E582158270021583E038FAF022EBF0A3EAF0B8
:208A0000A3E9F022E493FB740193FA740293F922706F72743D00706F72743D253032640031
:208A200073706565643D0073706565643D2564007365745F666C6F773D007365745F666CF4
:208A40006F773D2564007365745F716F733D007365745F716F733D2564006367695F736501
:208A600074706F72743D256400506F72742053657474696E67004D65646961207479706592
:208A8000206973206368616E6765642E3C62723E43757272656E7420737065656420736568
:208AA0007474696E67206973206E6F74207375697461626C652E00766C616E5F69643D0062
:208AC000766C616E5F69643D256400646573633D0026007663623D007663623D2530326416
:208AE000006367695F736574766C616E3D256400564C414E2053657474696E6700546865D1
:208B000020766C616E2067726F757020706F7274206D7573742073657420746F2074686599
:208B20002073616D65207472756E6B2073657474696E67006E756D3D006E756D3D2564005A
:208B40007663623D2564006367695F64656C766C616E0076747970653D0076747970653DB2
:208B600025640044656661756C74007379733D006C6F633D006C6F67696E3D005379737487
:208B8000656D2053657474696E6700496E76616C6964206C6F67696E2074696D656F7574DE
:208BA0002076616C7565006367695F7379730069703D00496E76616C69642049502061640C
:208BC0006472657373006D6B3D00496E76616C6964207375626E6574206D61736B0067773D
:208BE0003D00496E76616C69642067617465776179204950004950207375626E6574206DCF
:208C000075737420657175616C20746F2067617465776179207375626E6574006F6C645F5C
:208C2000706173733D006E65775F706173733D0072656E65775F706173733D004368616EB5
:208C400067652050617373776F72640070617373776F7264206C656E6774682063616E6E00
:208C60002774206265207A65726F006367695F70617373006F6C642070617373776F726477
:208C80002069732077726F6E67006E65772070617373776F726420697320696E636F6E7308
:208CA000697374656E74007425643D0025303264005472756E6B2053657474696E67005492
:208CC00068652073656C6563746564207472756E6B20706F72742073657474696E67206D7A
:208CE0007573742073657420746F207468652073616D652056414C4E2047726F75700063A1
:208D000067695F7472756E6B006D6F64653D006D6F64653D2530326400736E696666657254
:208D20003D00736E69666665723D2530326400736F757263653D00736F757263653D2530F0
:208D4000326400547261702053657474696E6700496E76616C6964205472617020495000B1
:208D60006367695F74726170006669623D00636F703D00257325256400647669643D005043
:208D80005649442053657474696E6700496E76616C6964205649442076616C756500636721
:208DA000695F7076696400647072693D00496E76616C6964205072696F726974792076610C
:208DC0006C7565007669643D005649442053657474696E67006367695F61646476696400EE
:208DE0005468652056494420697320657869737420696E20564944207461626C650070254F
:208E0000643D002564007461675F69643D007461675F69643D256400546865206465666184
:208E2000756C7420766964206F6620706F727420253032642069732025642C20736F206939
:208E4000742063616E6E277420626520756E73656C65637465642E00276367695F736574DD
:208E60007669643D2564270054686520766964206973207468652064656661756C74207646
:208E80006964206F6620706F727420253032642C20736F2069742063616E6E2774206265B3
:208EA0002064656C657465642E006367695F7365747669643D25640052656D6F76652056C2
:208EC0004C414E007061737377643D00716F73747970653D00716F73747970653D256400BB
:208EE00070253032643D0053797374656D20626F6F747570004C6F67696E20696E76616C69
:208F000069642070617373776F72642066726F6D2025642E25642E25642E256400506F721E
:208F20007420256420666962657220696E73657274656400506F727420256420666962656A
:208F4000722072656D6F76656400506F7274202564206669626572206C696E6B2075700044
:208F6000506F7274202564206669626572206C696E6B20646F776E00506F72742025642067
:208F800066696265722072656365697665206572726F7200506F7274202564206669626578
:208FA00072207472616E736D6974206572726F7200506F727420256420636F70706572204C
:208FC00072656365697665206572726F7200506F727420256420636F707065722074726106
:208FE0006E736D6974206572726F72004447532D313232345400282564290002029E1FFF3A
:209000000180C200000F3C74723E3C746820636F6C7370616E3D343E25730A3C74723E0ABB
:20902000203C74643E3C623E42797465730A203C746420636F6C7370616E3D333E256C75D9
:209040000A0A003C74723E0A203C74643E3C623E25730A203C74643E256C750A203C7464EC
:209060003E3C623E25730A203C74643E256C750A0A008403E38403EB8403EE8403F1766306
:209080006200203C74643E0A203C73656C656374206E616D653D25733E0A203C6F70746920
:2090A0006F6E2076616C75653D25643E25730A000A3C7472206865696768743D33303E0A43
:2090C000203C746420616C69676E3D63656E7465723E3C623E25730A203C74643E3C623E69
:2090E0000A008423F784240584241384242684243A84245120203C696E707574207479708E
:20910000653D636865636B626F78206E616D653D25732076616C75653D25642025733E20B7
:2091200025733C62723E0A00696E6465782E68746D006C6566742E68746D00746F702E68A5
:20914000746D0062756C6C65742E67696600666F726D2E637373006C6F676F2E6769660002
:209160006D6F64656C2E676966003C68746D6C3E0A3C626F6479206267636F6C6F723D23EF
:20918000433643414344206C6566746D617267696E3D313E0A3C7461626C653E0A3C74729E
:2091A0003E3C746420616C69676E3D63656E7465723E3C696D67207372633D6D6F64656C07
:2091C0002E6769663E0A3C74723E3C74643E3C666F6E742073697A653D333E3C623E536521
:2091E0007475700A3C74723E3C74643E3C696D67207372633D62756C6C65742E6769663E12
:20920000203C6120687265663D6367695F706F7274207461726765743D6D61696E3E506FB2
:2092200072740A3C74723E3C74643E3C696D67207372633D62756C6C65742E6769663E2024
:209240003C6120687265663D6367695F766C616E207461726765743D6D61696E3E564C4182
:209260004E0A3C74723E3C74643E3C696D67207372633D62756C6C65742E6769663E203C40
:209280006120687265663D6367695F7472756E6B207461726765743D6D61696E3E547275A3
:2092A0006E6B696E670A3C74723E3C74643E3C696D67207372633D62756C6C65742E676937
:2092C000663E203C6120687265663D6367695F6D6972726F72207461726765743D6D6169E3
:2092E0006E3E4D6972726F720A3C74723E3C74643E3C666F6E742073697A653D333E3C6271
:209300003E4D61696E74656E616E63650A3C74723E3C74643E3C696D67207372633D6275FB
:209320006C6C65742E6769663E203C6120687265663D6367695F64657669636520746172B2
:209340006765743D6D61696E3E5374617475730A3C74723E3C74643E3C696D67207372638C
:209360003D62756C6C65742E6769663E203C6120687265663D6367695F7374617469737429
:20938000207461726765743D6D61696E3E537461746973746963730A3C74723E3C74643E1F
:2093A0003C696D67207372633D62756C6C65742E6769663E203C6120687265663D63676973
:2093C0005F737973207461726765743D6D61696E3E53797374656D0A3C74723E3C74643EC7
:2093E0003C696D67207372633D62756C6C65742E6769663E203C6120687265663D63676933
:209400005F74726170207461726765743D6D61696E3E547261700A3C74723E3C74643E3CE0
:20942000696D67207372633D62756C6C65742E6769663E203C6120687265663D6367695FCF
:2094400070617373207461726765743D6D61696E3E50617373776F72640A3C74723E3C7421
:20946000643E3C696D67207372633D62756C6C65742E6769663E203C6120687265663D63E0
:2094800067695F6261636B7570207461726765743D6D61696E3E4261636B757020536574BE
:2094A00074696E670A3C74723E3C74643E3C696D67207372633D62756C6C65742E67696634
:2094C0003E203C6120687265663D6367695F7265736574207461726765743D6D61696E3E13
:2094E00052657365742053657474696E670A3C74723E3C746420616C69676E3D63656E74DB
:2095000065723E3C6120687265663D6367695F6C6F676F7574207461726765743D6D616950
:209520006E3E3C666F6E742073697A653D333E3C62723E3C623E4C6F676F75740A3C2F7476
:2095400061626C653E0A3C2F68746D6C3E0068310A7B0A20636F6C6F723A20233039633BE6
:209560000A20666F6E742D7765696768743A20626F6C643B0A20666F6E742D73697A653A1C
:2095800020313670783B0A20666F6E742D66616D696C793A20417269616C3B0A7D0A626FB1
:2095A00064790A7B0A206261636B67726F756E643A20234646464646463B0A20666F6E74C2
:2095C0002D73697A653A20313270783B0A20666F6E742D66616D696C793A20417269616CF0
:2095E0003B0A206D617267696E3A203670783B0A7D0A74680A7B0A20636F6C6F723A20231D
:209600003030383038303B0A20666F6E742D73697A653A20313670783B0A20666F6E742D24
:2096200066616D696C793A20417269616C3B0A7D0A74640A7B0A20666F6E742D73697A6573
:209640003A20313270783B0A20666F6E742D66616D696C793A20417269616C3B0A7D0A612A
:209660000A7B0A20666F6E742D636F6C6F723A20233030303046463B0A20666F6E742D66C0
:20968000616D696C793A20417269616C3B0A7D0A0047494638396107000700C400004A00DB
:2096A0008A9E00526C00736B0073B90040800065C70036340099630079CB0033800066C843
:2096C00000365B007E3D0093B9003F49008A5B007FC400383600977F006779006ACA003476
:2096E0004C0088B20045AC004841008F550083590080CB00343A00959B0053CC003321F955
:209700000400000000002C0000000007000700000527E0D1598C96491DE25DD804585EF488
:209720005584005DC9372B003C68746D6C3E0A3C534352495054204C414E47554147453DDD
:209740004A6176615363726970743E0A66756E6374696F6E206C6F6164696E6728290A7B90
:209760000A20202020646F63756D656E742E746F70692E6973697A652E77696474683D73C6
:20978000637265656E2E7769647468202A20302E39393939203B0A7D0A3C2F73637269704A
:2097A000743E0A3C626F6479206F6E6C6F61643D6C6F6164696E672829206267636F6C6F64
:2097C000723D272346464646464627206C6566746D617267696E3D3020746F706D617267F5
:2097E000696E3D30206D617267696E77696474683D30206D617267696E6865696768743DA6
:20980000303E0A3C666F726D206E616D653D746F70693E0A3C7461626C652077696474685A
:209820003D313030252076616C69676E3D746F7020626F726465723D302063656C6C737056
:209840006163696E673D302063656C6C70616464696E673D303E0A3C74723E0A3C746420AF
:2098600076616C69676E3D27746F70273E3C696D67207372633D276C6F676F2E67696627CA
:20988000206E616D653D6973697A652077696474683D273130323427206865696768743D3E
:2098A000273735273E0A3C2F7461626C653E0A3C2F666F726D3E0A3C2F68746D6C3E003CEA
:2098C00068746D6C3E0A3C7469746C653E4447532D31323234543C2F7469746C653E0A3CB6
:2098E0006672616D6573657420726F77733D273037352C2A27206672616D6573706163696E
:209900006E673D3020626F726465723D30206672616D65626F726465723D6E6F3E0A203C93
:209920006672616D65206E616D653D746F70207372633D746F702E68746D207363726F6C19
:209940006C696E673D6E6F3E0A203C6672616D6573657420636F6C733D273135302C2A2700
:2099600020626F726465723D30206672616D6573706163696E673D30206672616D65626F63
:20998000726465723D6E6F3E0A20203C6672616D65206E616D653D6C656674207372633DE3
:2099A0006C6566742E68746D206E6F726573697A653E0A20203C6672616D65206E616D6566
:2099C0003D6D61696E207372633D6367695F6C6F67696E206E6F726573697A653E0A203C22
:2099E0002F6672616D657365743E0A3C2F6672616D657365743E0A3C2F68746D6C3E00FF32
:209A0000D8FFE000104A46494600010201012C012C0000FFDB0043000604040504040605BF
:209A2000050506060607090E0909080809120D0D0A0E1512161615121414171A211C17183E
:209A40001F1914141D271D1F2223252525161C292C28242B21242524FFDB004301060606B6
:209A600009080911090911241814182424242424242424242424242424242424242424243C
:209A80002424242424242424242424242424242424242424242424242424242424FFC000F3
:209AA0001108004B032003012200021101031101FFC4001C000100020301010100000000E8
:209AC0000000000000000607030405020801FFC400541000010302030208050F08070803FA
:209AE00000000002000304010506111207131721223132425492141641515208152333535B
:209B000061627172818291A1B1C1343544637393D1E1244345556483D225367475A2A3B33A
:209B2000C2B2C3F0FFC4001B01010003010101010000000000000000000002030405010602
:209B400007FFC4003B11000103020405010504090501000000000200010304110512213143
:209B60001314415152320615224261168191A13334536271B1C1D1F023242572E1F1FFDAB6
:209B8000000C03010002110311003F00D3BC638BD46984DB6F86911F4568F0817DED41DDEB
:209BA0005CDBF7E72717397D90C4166D17E7473C977F8948F840BEF690EEAFDAE3FBED3F60
:209BC0004A0EEA93616D87DD31459E3DCDABBDBE3EF875EE78CC8695E6D597356ABA52FD48
:209BE0004F770B7B3BD9788ED51DBE6D6EE603F5D5652A8A512B3BEAB58D25690B18B3D988
:209C0000D41BC7FBED7F490EEA78FF007DED41DD5387BD4E37EA33BC8F77B63E5967412DCA
:209C200074A17CF95556378B44DB0DC5DB65CE394796CD7221AF97DFA79E9556C32C12FC66
:209C400020AB9E3AB85AF25D99D75ABB40BE76A0EE278FF7DED21DD51CA29D60BD925DF1D2
:209C6000BDB0A7C49B6F8C15320007CABACB2F2E54A57894A418A31CC6D6655425512BE422
:209C80008DDDDD723C7FBEF690EEA78FF7DED41DD538AFA9C712529F9DAD5DE73FD2ABDCCD
:209CA0005987BC53BC95A9CB8449CFB634272B18AB5A375AF56B9D29C792AE3969E47CA19A
:209CC000ABAB6686AE26BC97665B54C7F7DAFE921DD4F1FEFBDA43BAB3ECFB014BC7F77216
:209CE00086CBD58D1D81D721FA8E7A69CD4A529E5AD54CF689B108B84B0E48BDDBAE8F3A8E
:209D0000317493CDC91A57552B5A0F1569979F990E6A70368DF77528A9EA8E379836505EBB
:209D2000102FBDA83BA9C205F7B5077546C4A843AA8BF569E10765938F277523F1FEFBDA32
:209D400083BA9C205F7B507754729967C6BA363B0DC712CF1816A8852A4D46A5A69D5A5350
:209D6000CB5AD78A8A24118B5C9AC832CA4F6177BBAE970817DED21DD4E102FBDA83BAA6D7
:209D8000965F53BE239B513BA4B896E6BCA23ECAE7D54E4FFD4AAFB84708372950C5DDE7A6
:209DA00083BC6D6BE6D5A6B966AA8CE091DC435B2D32C7531333C976675DCF1FEFBDA43BB0
:209DC000A9E3FDF7B48775475B1D4423E9712D8991DA8CDB24DBBA88F9C7D1F8FCCAFE1CA1
:209DE0007D966E3CBE4BB5C205F7B507753840BEF6A0EEA8E649927043B2733279291F0803
:209E000017DED41DD4E102FBDA83BAA3992649C10EC9CCC9E4A47C205F7B507753840BEF25
:209E20006A0EEA8E649927043B2733279291F0817DED41DD4E102FBDA83BAA3992649C1080
:209E4000EC9CCC9E4A47C205F7B507753840BEF6A0EEA8E649927043B2733279291F081783
:209E6000DED41DD4E102FBDA83BAA3992649C10EC9CCC9E4A47C205F7B507753840BEF6A72
:209E80000EEA8E649927043B2733279291F0817DED41DD4E102FBDA83BAA3992649C10EC9E
:209EA0009CCC9E4A47C205F7B507753840BEF6A0EEA8E649927043B2733279291F0817DE31
:209EC000D41DD4E102FBDA83BAA3992649C10EC9CCC9E4A47C205F7B507753840BEF6A0EE2
:209EE000EA8E649927083B2733279291F0817DED41DD4E102FBDA83BAA3992649C20EC9C9C
:209F0000CC9E4A47C205F7B507753840BEF6A0EEA8E649927043B2733279291F0817DED498
:209F20001DD4E102FBDA83BAA3992649C10EC9CCC9E4A47C205F7B507753840BEF6A0EEA6B
:209F40008E649927083B2731279291F0817DED41DD4E102FBDA83BAA3889C20EC9C793C91D
:209F600048FC7FBEF6A0EEA70817DED41DD519271B0E9100AC0F5D2131D392CD3E92810487
:209F800063BB3298C9397A5DDD4B7840BEF6A0EEAFDF1FEFBDA83BAA13E31C1D5A5A23747E
:209FA000BD16C6B5590674D7FF0026B45C1CF37B1568AB2929C7776570C3585B33A98F0874
:209FC00017DED41DD4F1FEFBDA43BAA2EDDAF1449E53565DD8FEB9CA516D378471649E90EF
:209FE000418DF28EB5FB9525574C3F55A870FAD2FA2EF78FF7DED21DD5FBE3FDF3B5077548
:20A00000729BD9DE2377DB6EB19B1FD5B5525B4DEC9E5BBEDB7A975F92D528A92AFA7F15CC
:20A0200078E13585B92D8F1FEF7DA83BABCF08D781FD301666763B18BDBE55C5EFF332FC39
:20A040001741BD8E5A7AD11E2F94ED55458847D015C383CDD645C72DA65D47A53D91584B1A
:20A060006A9701FED1654A19D90D99BFECA64BE5664BA0DECB6D43FD930FBAA3EF16F05755
:20A080008E107D6475052DACCE1FED26963E1766D39AE205F24558CDECD6DA3D1B644FDD69
:20A0A000516E3780628F461C61FF002A8A3CF7EEB290E11DE47556F0BD70EACA32F92D5535
:20A0C000385BBAF54DD2FF0022AADA1C12C8FF0050C8FD1A2CC3835AF720EEA8F3EFE2CA4F
:20A0E000CF750F9BAA7F85BBC7F88FDC55385BBC7F88FDC555C5E2787A0BD789E1E8A87335
:20A10000CFE2CA5EEA0F2754DF0B578FF11FB8AA70B576F4E47EE2AAE4F13C3D15E7C4D64F
:20A12000BD004E79FC5947DD21E4EA9DE172E7D67CC7E53554E17A775A700FCA156F160BBB
:20A1400064BFAA02FA34585CC0714BA51592FF002A8A7CF978B28FBA1BCDD5563B599C5F49
:20A16000DA6D2F43B569E5FDA2CAB21ED9CDBDDE95BA217F9545AAE6CBED45D2B644FDD5B5
:20A1800014BDE1FBACA1EE77FDA3A828ED3AE65D1B8B2B2708D782FD31952C7B64B6573A18
:20A1A00056A8DF4472FB968B9B1BB2F56098FC976BFC5487100EA0AB2C1A4E922E18ED0AFA
:20A1C000F65D1940BDF8FF007CED41DD5BAF6C66DDFD5F8735FB37EBF8AD17B63E63ED1793
:20A1E00069CDFCACAAAC1C422EA2A92C22A3A489C205F7B507753C7FBEF690EEAD57B65B45
:20A200007863DA2F465FB663F9AD37300E2963A3320BBEF69AD3F0568D6D3F8D952585D6D3
:20A220000EC575D6E102FBDA43BA9C205F7B50775701CC378B98E95BA3BBF25DA7E2B51E23
:20A2400066FB13F29B14BD3E937CBFB95C3534C4B3151568F4752AE102FBDA83BA9E3FDF55
:20A260007B50775438EEFB8FCA61CB63DF71AAD11BBEDBDDE48C90D5F095825016D659C8AA
:20A280002AC7767532AE3EBED3F4A0EEAFCE102FBDA43BAA2E329973A2E817D2596842AE1F
:20A2A000E147D9953C6987777523E102FBDA83BA9C205F7B50775471325EF083B2F39893E3
:20A2C000C948F840BEF6A0EEA70817DED41DD51CC9324E08764E664F2523E102FBDA83BA66
:20A2E0009C205F7B5077547324C93841D939993C948F840BEF6A0EEA70817DED41DD51CC54
:20A300009324E08764E664F2523E102FBDA83BA9C205F7B5077547324C93841D939893C9F8
:20A32000493C7EBEF6A0EEAE6DFF001BDEE4DB1E6CE56912E7D3C4B9B5E2AAD0BD7E6F35F5
:20A3400019231107766538A6908C59DF4520BF7E727573BC8BA37EFCE4EAE7791583B32A99
:20A3600024F53ABD3D4CDED7883E531FFBAD8F555910E04B7E9FEF20FF00C66B5FD4CDEDEE
:20A380007883E531FF00BAD8F5567FB8B6DFF9987FE335F3953FAE3FF9D17D7D1BFF00C783
:20A3A000B7F9D57BF537E3B3BC580B0CDC1DD536DA39C722E7723D7C9F46BC5F1695B3EA56
:20A3C00085C194BB61C1C4711ACE6DABDB74F39C7AD795DDAF2BBCA07EA74C272EE3890286
:20A3E000FF00A89A896E121D63FD63841968FAAB9D55CFB5DC491B0BECF2F73A41066718F3
:20A40000E3B405D671CA691A7DAA13FF00A150CF1BAB69FF00DC51BB4CCBE5281065DC1A6E
:20A42000DE448921F11E2A936D54BEE53DD8C419D0B69769F0962446136DEC85C0A86AC92C
:20A44000B2F3F3AC981FD5096BC1985E159E2E1278C586E9ADCACBA52AF395E91D791E5AD2
:20A46000ADFC0FB4D9BB4ADB55A65BB17C0A230CBC11E36AD7BBCDB2D455AE54E3AFC4B798
:20A48000CD5324804CE366B2E441451C720989DDEEDA595DBB44326B00E2236C884C6DB2CC
:20A4A0006B4A8F3D3D8C97C4969A3AE535996A5F6D6D1FFDC0C47FF2C93FF8C97C7D80B034
:20A4C000ECFC533D9B55B1B0394E0D4A9A8B211A5299D6B5AACF85E51B913D9996EC684868
:20A4E000B288B6AEAD1D8C1E34658B996158769741D20175C9E454D254CF9B4D73F2AEFE4F
:20A50000D2B03E2EB9E0CBB5E31862707461B35798B65ADADD47DE52B4CAA645CA3F9D7132
:20A520007639689187B6B32AD321C127634775A72AD95749569A55B5B662D3B2EC475FF0FB
:20A5400085F7D146B0ED50CE3D6CA586C79A91D8BA5DACAA5D92EC930CE34C3CDDC5EBBC74
:20A56000D7DD0AE87D86868DD1B3E7D39D695CF894DB16EC630BD625B1A6A547B1C261DABC
:20A58000EFDD32A6F2454B2A50759579F8972BD4AD5D583EE9FF001BFF00D62B47D56C4798
:20A5A000E2FE1E0122A50A69D6B4A7BC0A124F2F1F2313A9C749072D9C85AFFF00AAC085DB
:20A5C000B16C13122EE4AD14935D3955E79C3A997D55A7D8BE79BBC4AE13DA4C9B2C092FA5
:20A5E00036DB134006A2795482A62541AE4BEACC299F8AF68CEB9D7C098CEB5F2FB1D17C61
:20A60000A9B422AF0EB74FF8F67EE052A39E429098DEEA3885244310980D9EEDB2FAFF00D8
:20A620002E2F997CB5B3AD95BFB40C557FB84F71E8F67627BE02E37966F39AEBC91CFCDEFF
:20A640005AAFA9694E2A556BC38912231BA86CB4CB3AAB5D0D0D2839D6BC7CDEFAC314E519
:20A6600015F26EEBA7514C1365CFAB32A231FECFF673B3B84CC9B9CEBC3AF482D2CC669DF5
:20A680006F5B997978C78A94F3AA5DC95E16E1137AF46AA90091675F9EBE55D9DB0D8F1568
:20A6A000C7DA04B77143BBDDF954A1BC1ED44C52BC9A079B2F2D17123B146474AFA0A0CE57
:20A6C0004198DEEBE531368C0F280D9654445D25C7444445E2222222222222222222222220
:20A6E0002222222222222F5111117888888BD44CEA95210E92C2F4F8CC74DF0A7D250231CD
:20A700001DD7A2045B32CD9A2E69E208752D2D113E5E8B635AAD867D7B9C3AA1D8E590F97E
:20A7200008F914FB55255710EE4B5474139EC2B6B8D17B6708E2C97A757824412F8753AF5C
:20A74000D8BA91F657364E9F0BBC483F38B234059CB148876D56F8F02A82F568B8A4F34D89
:20A76000749D015A8F5EE0B1C927C3579878D4F61EC82D62424719E93FB576B5522B7ECD24
:20A780006DF13DA2DD19BFA3FC5662C55FE515B23F67DBE7254EB778AC92D3120CB925FA8F
:20A7A000B6EAB699838966FB4594D91F49F2D2AF68F83C0474E9011F82BA0CE17647A42BDE
:20A7C00039625292DB1E094E3BB5D510CE09C532FDB9F891BE48D4D7422ECAE6BFF965DEFC
:20A7E00059FC164681457AB7618E3D55B0DDB638F55662A994B725AE3A1A70D81952F0F654
:20A800003B6CD5A9D6A5C92FD73B5FC176A0ECAED318B535698E25E910E75FB55A44CB2C44
:20A82000091168111E55489716463AC2F10885CBB46D43EE799FFF001A557822726D775674
:20A84000914317A9D9971E2E0969AE8B00DFC915D06F0980F49384CC25FDEBFF0061DFF461
:20A86000A7099853FBD7FEC3BFE95EF2D2F8BA87394FE6DF8B2DC6F0CB23D205B0387E2899
:20A88000F556E41B844B94719309F07D83E636F8E8B8F2B1F61C8939C82EDC7FA4039A2A27
:20A8A00002C387CBF37246AAB18CC9ECCDB2B0A78C199DCB475D21B4C71EA2CC36F647AA6E
:20A8C000B60484BA2BF5455AB10C5687AABD6E43D05ED11178DD8FA2BD6915FA88888B1495
:20A8E000870988EE3A3D20122A7CD4503E11AE1D8E37DBFC573EB3108296CD33EEBA787E1B
:20A9000013515CC4F035ECAC1455F708D70ECB1BEDFE29C235C3B2C6FB7F8ACBF6828FBBEC
:20A92000FE0B7FD96AEECDF8AB05142AD38EA5DC2E4CC67588CD81969A90E79F37C6A64D08
:20A9400096F4752DF495B1D5039C6FA6CB995D87CB446D1CADABEABDA222D6B02222222257
:20A9600022222FCD229BBA7A2BF511178DC87A0BC94768BA8B2A222D6282C9755632B5C728
:20A980002EAADD4445CC72C71CBAAB5DCC371CBAABB6888A30F61164BAAB973367706589BB
:20A9A0000BB063383F09AA129DA22595492B63B642D5A6DC0DE7EE6550FB971646C6596B0F
:20A9C00057834CB8B1E6D2E67F7ABD348AF24C81751486421D9D40A102DC597CF3236637C5
:20A9E000E8C5FD1AEA0E0FA2F35C7F62E6BD85716C3FD1A3C91A7A2EE55FB57D24E4164B98
:20AA0000A42B5DCB2C777AAAE1AD947E65964C369CF715F33BC57689F95D96737A79EA2362
:20AA2000AA9F62C237C89AB4B846C97A2E0D68BE927B0CB05D115CB9D816249121762B2EDB
:20AA4000097A434AAD238A4A3BB5D62930280BD2F6544B7323BBD0740BE92CFAA9E7564DA7
:20AA6000C363F667F57FB381B22EB339857EC5C199B1B06FF239D3A37CA2D745A07166F9A2
:20AA8000856293D9F2F909451174656CEF13422FE8D3234B0FD70D42BF8AE5C8B6E23B7EBC
:20AAA000AF09B2BCE08F39B0543FB29C6B5C788445D6CB0498454874BAF79553E75A15BD45
:20AAC000C76CB4BE0F305E8BC1515B2C4C8CFF0041D025A46602D9D961929E40F50BB2CDF5
:20AAE000E55A17AFCDE6B7FCAB42F5F901A4BE875E41FA41FE2A417EFCE4EAE7791746FDE1
:20AB0000F9C9D5A4CB64EBCDB63D232A0FD6A43E96513F5BABFB64C585367F6C92770C659C
:20AB200063297345A375BACC6C68CE9A57939EAE3E92CDB5797823699608D690DA161D825F
:20AB40004CC9191ACA6347AB2A10E596BA7A4A8BC4F80255B8C01A7D9B816FE546318C2E0D
:20AB60006A0723E55733A5469C54A167AA8B956FD9FC995125CC71B763B4C32DBA264C3972
:20AB8000503D6E088F2A94C873E55695AFA2B87252E73E3315EEBE961ADC91F0086CCBE93F
:20ABA000FC2F8A7673B3FC2B1ED91F1658CD98A199B8129B3378ABCE7A46B5AD6B55406DE2
:20ABC000B76B34DA65DE3DB6D1BD6EC708B50D4F93590E578B5D69E4A529C545CD6F65B77D
:20ABE00019777B9C06DB74A3DB0E4B4FCDA3655686ACD0AB5CCB2E2CF4F166BF5BD9EDD2DD
:20AC00003561D22DBE74C7244609042D447736F554B4D3A3C79D033A569C491D20E7CCE5ED
:20AC20007529B103E1E411B36CB8B160B60C88D455BFB1DB0E1FC3D73878A2EB8B2C910CEE
:20AC40005B3D108A480B81AB31E5E65C5C5C6ABD670EDE1E86F4B6AD1707234723A3AF0CB5
:20AC600063A83750A665A8B2CA997957A0C1D3AED87245E982028F1A4B71DD0E3D43AF98B5
:20AC8000FE2CF2A2E8D400947905EDD171A94CC666321BF55F4D623C71816F961B8DA0F11C
:20ACA000B61F67C3A3391F5F87B55D3AC6A39E5ABDF55F6C9B0F606D9CCE7AE32768387A0B
:20ACC000E320DBDD054253600DD2B5CEB5E9D78F8952337671748F36E2C330644B0B7C938D
:20ACE00088F48618326F589E9E7CBCB55B375D99DF6C937C024DB65139526C049B6CEA2EC6
:20AD000019E7A283C5C75AE454FA355CC0A36667663D1D76E4C4189D8C835656E604BA58EB
:20AD2000385AC4B8B24E2AB1C68147DC8F1C1C96DD0E467A796399743E17954FB1D62EC120
:20AD400038AB095D6C6DE38C3AC3B3582685D29ED56835F267CA5F2DC2C137597516E1DAC5
:20AD6000A749236EAE88B2C19D4828751A971539A854CBE3592D9B3B9F76784FC19D62394D
:20AD8000B4E3A125D68E8D9501B70F2A165E5DD1D29F12F65A36776272D9461C45845C1871
:20ADA0007475786C06F186F07E0D786E98AEC6D3B2E493B46CA60054469C9A6742AD2B4C7D
:20ADC000F2CD6AFAA12EB85B19E198AF5AF17D81E916B749FF00066E6038E3DAA941D2342D
:20ADE0001AD6B9AA558C1F73951DD38F6D9AEB6D35478CC182AD01BAE75A156B9715393C85
:20AE0000EB62D1B389572B1DC6FE22F0C4855A056ADB067A8EB4AD7C9C5411A53945E4D4AF
:20AE20002A4546C25C4CCA2188668B85957D4785769B82C70BDAA8F628B3453188C8137229
:20AE40002636D98950294AD2A255A5552D89ECB63BEED98AE51319E1E2832AA139C7CA4896
:20AE600068674108EEF567911572E2A66ABF9382EEA3B9072D5700379A279A1260E9571B5E
:20AE8000A53554878B8E94A71E6B259B039BEFDC5B96F85B7D6D6B7B237ED9E63EC82DE967
:20AEA000D234AD73D468147909C84B7513C438A0C063B7F45F5E1ED3303B6391E30C3E3F1C
:20AEC0001DC1AFF52A5B0B6D120ECAF1B4CB43B88E0DFB0CDD1E3960FC33DE7ADE4665CF89
:20AEE000A73A7C74A7C6AAABAECF6E71E5CF6A90DD96DDBCB4BF2633666D0D39E95A965C8F
:20AF000059D3CEB1B5832EB1E912A76B9B4A4CE38F5AB05ECF4E7E47172BE6510C3C7BAB8E
:20AF200065C55F47CBAB2FA87185FF006658E6CE56EB962DB0506BCB69CF0E6A8E325E4243
:20AF40001CEABE78C4F68B661E9E312DF886DF7C021D5BE865AA834F2675E3A67F15572D98
:20AF6000ED9F4D066E2ECD8AF4176030DC92664B5503704DD06E9952B4F86B5DEC3170B155
:20AF8000B8D8CF832E11383ADBA3ED54350D7CB4CE9CCB45242F116512BB2C588548540632
:20AFA000671B3F759511175D7091111111111111111111117E6A144B2FDC938D6072745688
:20AFC0003DB1F01FA4B59CC416F0E48BBBC2F440735594803BBAB469E42F48BAE864992D80
:20AFE00026E5DCA58EA85659CE8F9089AD34FB56E3386F16CBE8C38F104BDD1DCC87EA54AD
:20B00000157443F32D91E13527F2D97EE5979579275B0E9100AE9C7D99DE24E9F0BBC69135
:20B02000F2D196BF1AAEB43D904122D524E64BF79C778BEAA2CA58A07465B63C0652F59592
:20B040009439EBBC063A72416B0DF01FE4C68D22497EADBA92B7ADBB31B6442D4C5B233771
:20B06000F08873FBD48A2E0D068748B40D8FA22392CC58A49D196D8F01887D657545B3077C
:20B08000124E1D4C594DA12E627CB25D06702E2697EDB3234612E7DD8D4EAAF68F85D91EBF
:20B0A00092DE66C71DAEAACC55B297CCB7C785D307CAA8F8BB24A3E42532E13A4F9C756861
:20B0C000A7D8A416DD93D9E316A1B60395F3BDCBAFDAADA6EDECB5D115985901E88ACE52B7
:20B0E000116EEB60C201B0B282C1C0ECC61D2D30CB23F0474AEB47C2603D2527451535C88F
:20B10000670FC76BAAB71BB6C76BAAB6D1116218ED0F44564D22BF5111111111111463681E
:20B120009880AC186DE264B4C995EC0D7C1CF9EBF3514A38DE43606EAAA9A56881CDF6653B
:20B140005CED13193D7EB9396F86E9FADD1CB45047FAF3A73957CFEF2C76DD9EC896C8B8D4
:20B16000FBFBB32EA08E7A7E7CD73706DAFD72BC0910EA067975F8FC8AD6BD5B6E3E2EB848
:20B18000D5A340CC7748EF7568DDD3CB5A57CEBAF3CBC0718227B7775C0A5A76AA62A99D9E
:20B1A000AFD9941F82F3ED8F7EEBF9AE15CB085D60CB7196A2BD21A1E8BBA72D4B76ED1F77
:20B1C00016D9A393F2EF12C5B1211E4CC3AD4AB5F9D61C372AED7BBC32C3B739C4C096B7C1
:20B1E000753E7CD4F273F955A05308BC99D9D9659429CCC61689C49D4CB09CE0C1785F7D56
:20B2000074DF3224E6AA80F19E65C54A53E6A2D3C3B6BC3979B914DB4B1388E3B8275392A8
:20B220005C5AEBF3F3AE2ED1EF032EE4DDB58F6A89D3F84E57F82C37298EE1BC3ECD9D8378
:20B24000DDC8963BD9043CF957C9F82A46172167BD88BF92D2552212385AE11FF356348DB2
:20B26000A261DB47B03B30DF7479C638EBFB799616F6B9871C7044BC31B1AF589AE2FB2B6C
:20B280005507C238359BA4519331A3737BD00D551A65E7AE4BA58AB06DA6C9639133C17793
:20B2A000274E4B75DE9972EBCDCF555706998F87ABBECB4F1EB5E3E3FC2CDBDB552EB86DE6
:20B2C0003AC36FB83904BC2DE75A2D35265AA5699F9A9C6A452AED120C3F0D9AF84660476F
:20B2E0008C9E2A534E7E4F8D51782EDA572BD0BEE7282396F6A45D63F27F15DCC5D8A2C992
:20B300007479B8DE0B2EE251F934217F76DE7E7A654AEA4928C388D1874DD21C464E094B55
:20B3200025B5F4B29848DAC61A60B4B6ECB7FE136C717FD592F2DED730E11692F0B6FE119D
:20B3400035FC2AABB8F31A8CCE91C23BC11E56A735957EBA8AE4DEA6429F31B72DF0FC1870
:20B3600037741A80FA6AE0A18C9ED67FE3765925C52716BDDAFDACEAFC1BA44BCD95C99060
:20B380005F07587593C8C78BCFE75528F487529B6118276DC37E085D564C8FE3AE75AA841A
:20B3A0008F28B4AFCE7DAB66E3064D77FE8BF60F6209CA9E423D1DED7FCD49196EC243EC73
:20B3C0008FB225F26AB26E70EFBBB3DDAAD7670993A3A85D3EEAF5E279FBA9F717AC159634
:20B3E000FD007E5FDD41CF0FBFEB327E7FD974AD306D32660F813ACB8E80EBE48D79B9BF7F
:20B4000015D2BF5FA761DDD9370D97A39F2687AAB98D7CD55CFC3F6176D73B7E2465A874BB
:20B42000747DFA57F0528B8416A74171A7F94043C7A975628A67A576B301FD365C69E6A65C
:20B440000AB67BBC81FBD7BFF45C5C3F8D06EF20A349681874B94DE92E22F3AD7BB6D03C5A
:20B4600012738C42601F683935322E957CB9283C810625382C3BBC002E418F16A59AD6CB9B
:20B480002FCC6DB7CB925CDF0AABE70719AA361A662B15FD4BEB8FD9FA289CAA9C6E36BE98
:20B4A0005D7FFAAC8C3F7A95748FBF92C03025D011E3A953CEA3ECED1243AF362E4364406E
:20B4C0008846A5AABC9A2935AE1EE99D4AA964449E6C4BA2442355D5C5AA6A295A208CB569
:20B4E0007BDFEBB2E2E0547495AF39C81A35ACDAE9BA984ADA33DBE21890D9DD7909C2AE12
:20B5000065F52F2CED225017B2C16487F5655A7DF9AEA41B1B4FB23EC4023F268B838CAC40
:20B52000ED5B463B8220246443C9EB285605753C6F3F1AF6E9652A0930DAA99A9B816BF5E5
:20B54000BA9B59EF516F3177EC727AB502E71AA8BC5DA23AECA6DB7E2B2DB445CB3D55E43C
:20B56000D16BE057887C21BEAEA15156477AF36DFA4422A9AAC56A3830480F672BDFEEB2AC
:20B58000D34382D235454C520DD82D6FA5D9D4C256D19EDE1783436443C84E156B5FB17453
:20B5A00030FE36A5D250C492C032E9F42A25C459791618F86D9930F4EE00474FA2B9717046
:20B5C000ACAB7CE6DDDEEAD05ABA2B570B128A512CD987AECB0F13079E03161C84DB6FAB35
:20B5E000AEF5F31C47B5C828CC31E12E874F95908FBCB923B449A5D1B733DEAA89BC44EC25
:20B60000A71C2E5113845F3E6BB4CDC2F023EC704087F655FE2B9E189D454486F9DC59B616
:20B62000666BAEB4B83D2D2C40DC362276D5DCACBAD1F6907BCD3260F23CA4D9718FCD558A
:20B64000269188213169F5CB56A63489534F48B3E6A2ADEE0DDC2739BE760EECB4E9F6317C
:20B66000AD17519832E5E19288227ADA735D00BFFDEFAD54B5F597901EE566BB3BB5961A84
:20B68000EC2E82D118D86EECCECCF7D16D39B469445EC16E647CDA8AB5FBB25E4B681736F9
:20B6A000B94E416447E49D3F151B8EE4BB6BC442D189746A242B70B104E21D24D32425CF4F
:20B6C000A9AAAE7C788CC4D9A59098BB65D17525C26984D86084487BE6D54AACB8F02E122D
:20B6E0009B8D262EE48F92062598E6BA588313316165BF62DFBEEF4004B2E2A796B5503B7F
:20B700006DE196A5364FC38C23A8796DB59547DF5DAC696D9127C1E5B026F0037A0C478E4A
:20B72000A3E55D28B109DE8CCE32CC4DF4D597267C2A983108E3943203FD747FBD3844B835
:20B740003A5EC5059F93C755E7842B8345ECD059F93C7451F87709B6F6F76DB5C9D5D61506
:20B7600099EBE4B7474BAC4721F84D2E68E232E4CC72BB17FD745D62C260E2650805C7BEF6
:20B780006D54EB0EE2C66FBA9B26B70F872AA3AB3A153DE5DF55E613BA32EDC374515961DF
:20B7A000D21E236C72D5E5C9580DF457D561752F3C0C6E599FBAF8AC6691A9EA5C1872B758
:20B7C0006DD7AD22BC93205D215ED17417296A396F65DEAAD37B0FC777AABAE888A293B033
:20B7E0005C5923A5C681C1F44873515BA6C86CB2F95E020D97A4CE615FFA55AABF348A5DDB
:20B80000784225BB2A1A76C82446D456FB9CB6BCC0E72E9FC5472ED81316331C9A118D2C0D
:20B820006BE8968AFDABE9828ED174856BB9698EEF555C35320B5B32CA543013E671D57C67
:20B84000FB7EFCE4EAD28EE51A7DB70BA204255F9AAB76FDF9C9D5CEF22FA91F4B2F8337A3
:20B86000F8DD4F6EDB47B4C9BE3526BEBA4B8FBF9A7575F6DB0763B521B30DD374A1D75009
:20B880008EBD7C654FA2B8D23185AE8121A8AD4E703D69620B64F005088DB90DB95A964533
:20B8A0005CA9510FAFEB51826A84BF77145946904765B5EB88B7536958FAC6E4F9729B6E98
:20B8C000E7F95DC6547A1B4DD3578633A0A87CBAE5A0B9B2CF553D15CDF1CA20D823C016EF
:20B8E000A58BA10E3C732D14C8AADCA75DAF979B231F9D46B7144DDD102905BEE42AF22B05
:20B90000AB2A7E21B7DEADB75BD54DD89528B706986CDE63D901C944E866343A98B9EC992D
:20B9200069D3D5D5AB2517C378C5BB15BA3B558C72729BBF90C965A1E8E4DE830CFCF5F2DB
:20B94000717173A8D947125E85BA08AF429728B8BECBC3AD727636DD4CAE3B4787363DD26F
:20B9600091C24447DE973DD60BC11A7778D4AAF189954B36CB4F1574EA581CC716D1B85DBA
:20B9800026B2D4E3F0F841A41C100F079819504E95A157508D3571E54E97454537344DD8C6
:20B9A000AF0694457A55C44A673B1F5A2E53E736E47B9C4B73AFC6951E91F455D6C9B270E7
:20B9C000C9BE3AD29A48DF72B42CF93E625E38448CE621B75DCE218F83C59CDB8C0B43563A
:20B9E000F7AF9C921A506B5E30A6F833CD43F7344DD8A3D28FF9F823571A96F8E96796F5ED
:20BA0000CDE99165D63CF1A3AE5B858036BC245B211A83953A1B42352E4E9CF93C9E3A2EE3
:20BA20001C4BC351B0E4BB7EECCA43B323C90AE9A68C9B17A859F1FEB0573B405179A93436
:20BA40003D220526845BF2FC956F524EF9ACA6B271FDB2B325BCCB170CA6BB3E63BBC10FBF
:20BA600061764304D8B61CAE3112AF19F167E8F171F0B0E6202B1C6BB69A9D244B8948EC32
:20BA8000908D0C44F7CD9D6A59FC1025C327A2F59D0EF2F0E5CE0B5D292D77944618C5AD8A
:20BAA0007D14CA694DEECDAA97DBF1B6E6C2FC694EC9A5CB7B29EA48F0607EB237ED881D44
:20BAC0000C8CA950E21E953567A976ED18E2D73713C07868F4739F798B709652B4035174FF
:20BAE000090E96EB9D731F64AF1D72CA8397BEAAE3BF5B3B4817C95E46ECD3FED10E5BBFD7
:20BB0000B362A5F82AA40875F8AD75AA33A8D3E0753F6B1BDA2243ADB1A098FC666DE319FC
:20BB2000975D60286F3A32E927961AF210AF43888BCFEF2D1C658B59C4921AAC371DDC6FDC
:20BB40009E93565D88DB3BB71DA8D4A9A84ABAFA34E5574FC4A26DFAE4F97B058E717CA6BA
:20BB6000B2FBD6CB765C50EFB5D9777FB4769FC556D2411BDF36AAD7A7A99072E5D1661AB2
:20BB80002FDA568B2B383715C9E93B0637BDC67F82DC6366B7B7CBFA4DDF48FEA5AFE2AC32
:20BBA0002C4A21FAAA8704A82DF45CFCD63290D0F49D01FA4A44CEC87785FD26E771787D1A
:20BBC00011C817522EC7AD14E9C379FF00DABB5AAA0B156F945680F67CFE6250072F105BF4
:20BBE000E7921DE587D7E8E65A5A6E43BFB36EB5570C3D98DB18D3A2D91072FD550BEF5D00
:20BC0000C8B8341AE4B6D0363E888E4A92C524E8CB5C780C7F315D512DBB7797F9258E63A7
:20BC200083E910E5F7ADA670FE2D97CA1831E30FEB9DE3FB15F8CE1301E92DA6F0DC71EAEA
:20BC4000AA0B109CBAAD51E114C3F2DD50F1F6778824F2A4DD41AF82D36BA517642D39F948
:20BC60005CE9CF97CAD14FB15E4DD9E3B5D55B030591EAACE53C85B92D71D2401B0AA86DBA
:20BC8000FB23B3B14FCD80E57CEF72EBF6A9241C071E3088B51596447D11A514F85901EAF6
:20BCA0002F5A455775A3288ECCA2F1F0980F496F3386E3B5D55DB445EAD06ED31DAEAAD81F
:20BCC00018AD0F445674445F82D88F557EA22222222222222222222222222222222222221D
:20BCE0002222AE36B965B95CAB05F88D1C8619131306F8EA35AE5C797CCAC7589E645F1D50
:20BD000024AC825788D8DBA2A2A6069E378DDECCEBE7688DDDED6FEF22B33A3BBD1AE96EDC
:20BD2000B4FC174E989B18E9D3E1571D3FB2FE4AE672C2C916AD2BCF8BECADE58866D5C12C
:20BD40009D728707706B04AECCA8F799C437D787C2465C821E6DF674A0FD7C4A6563B19E07
:20BD600019B2CA9BBA3912847564D8D6BA8FAA34CBC99AB006C2C897456E370C1A6F488A06
:20BD8000A65AD73660B59BB2D14F858C6EE59AE4FD5FA2A370DD8E6DC2F9BF9CC3C2205B33
:20BDA000D32786B4D479FBFEFACD8D30FDD86F4F49AC379E8C7A7766D8E74CA94A79B99580
:20BDC000A5892CF29DB3CCF5B4B4CC26CB764259573F7AAAA56EE58B2DB2B53FEBA3C43C32
:20BDE0009DD4ADE3805F3556C8272949E46766B6965CDABA68E9E3685D9DEEF7BB2DAB2E4E
:20BE000020C576F6DB8D0A199080E9A6F22F469F1AD1C5D78BC5CA5371AED301F7191E3656
:20BE20009B1A501B2AF938B9EABA1E3062B963BB6209B79F275B71ABF79712D8C378265B10
:20BE4000B3066DCBA5AB5D1BD5991579F3256710227790D9AFF4DD50D0C9333431B93B7730
:20BE60007D999742DB619B0707CA184D194D75BD5511E7E55694AE5F10A87DB46E964B8046
:20BE8000BE36B789D0E4E87983F2ABE2DB6F1623E925E5EB2B2E96A5CF8EB5C5899C6F7582
:20BEA000D99F0B6371712B65D9563E3162676DEF3A36908C223C464D1D4F3AF3691AD57188
:20BEC000708D864CCBC0BB25879B06397EC835A6A3F273ABA06CAD02F4DD9DA69CD49CEE2A
:20BEE000507001B5D1F0CCF209C86EF6EEB0B30F716B78447944D97DCAAF287284B94C3C35
:20BF000025F26AAE4D3C9D2B4645A5A7CB512F9CC4B0A6AD71272B597D86118D961C242267
:20BF200037BAAC4665D87A2FCE1F9246BD7875E7B4DC7F7A6AC8F58DA4F58DA583ECF97EF4
:20BF4000D9D74BED40FEC07FCFB940ECB70BA8DD23EF5F9C4D6AE58911E5F3E6BB98BAF57E
:20BF60002DF67D6F84C3DA0BDB5D11AE45F069F8A910D95A12D4B61C822E8E95B430C308D3
:20BF80000A0691F5EAB0C98D01D48D43C2DF0ECDD3F8AADEC367392F6F1D68C447984961D4
:20BFA000BD58E45B657B1B464D1F280847A3EF2B323DADA60B56959244307C7492ACB01898
:20BFC0005E9DA2BD9DB5BF55607B4F50D5253135D9F4CBD2CA3B84EF8F498BE0D2DA317550
:20BFE000A1E2321AF2A8ABF6C77AE08FA45A55B4DDAC18E50AAAE3C7786533A9A31F641E9F
:20C0000090D7CEB998D539B3411BBB95AFAFE0BB3ECED544EF5130B30DD99EDF8AE90DD336
:20C0200011411DDB6FC9111EB69CFEDC96ACC72EB77704A4F84BE43CDA87922AC2836D697B
:20C04000F8E3A856C0D9595B8F01E26852965ECB9B1FB4FC37B8422C5DD946F09DADD88DED
:20C060009139D22E55544E3C390D4A6778C3C3EC94E90D7CEADC6618303C915AEF5AC1F740
:20C080003512D35183472846025660FCD64A5F682584A590C6EF26FF0044B48FF4715B84DF
:20C0A000C8175179659160748ACABAECDA59702FADD5618830ECB837079C61A371832230DE
:20C0C00021E71CFC8BCB37CBAB03BBF030734F589A3CFECAAB2A44507FA42B4CACAD2E1FFE
:20C0E000B9B2191C1238DFA2FA46F687891885444C79767755CCA9176B93DBCDD3CDF56878
:20C100002D8D407ED5DE1B6CEF17F74C3EF0CA12D752176B4D5EF66A50365696E370C1A13D
:20C12000D222AD830A60CCE66EEEFA5D51538E94991A38C4585EF6EEAAB1917688F7B20C5E
:20C14000970BD1786B55B1EBB5D4B92317FED55584F5A5974B56958FD656952183480D615F
:20C1600098ACB51FB4111BDCA01BAAD63DA65CB903BC68DB122E5910E4A498821DD499657C
:20C18000F84EC9D023A5C69B2AD3E7C94A9BB3B225AB42DA28A04DEEF4AB22C1A28A228D54
:20C1A00089EE5D5679FDA29659C26216B0ECDD35556C7B85D636A1DD3CE7ED06B5AAF5228F
:20C1C000E17596C934518F4973E96AAAC42B2B445A93D656953EE693264E33D968FB4316DE
:20C1E0006E2701B3281E1DB5CA6AE0DBEE346DE8E6D5EFF12B2A3EADC8EA5AECDADA60B5DC
:20C20000695B83C95D2A1A20A38F861AF55C8C4B1292BE5E349A3EDA2FD4445B9739111119
:20C22000111111111111117CED7EC1F8D06738E390EDD97934BFFC972FC57C61D8E0FEFFBA
:20C2400000F92FA22E519A32E53742F8D69781C7F710FA96CE727EEB9CD85533FCAA84F167
:20C260005F17F6383FBFFE49E2BE30EC707F7BFC95F7E071FDC43EA4F038FEE21F52F39D2A
:20C280009FC93DD34DE2A86F1571876583FBDFE49E29E2EF72823FE6D7F82BE7C0E3FB8875
:20C2A0007D49E08C7B90A97373F9297BA69BC551038371697611FA55590702E293E94C82FA
:20C2C000DFD1AD55EA3118F7215EC62B1EE62A05593792F070FA6F05458ECEF12974AED141
:20C2E00087E4B555E8766B7E2E95E03E8B4AF818AC7B98AC83158F73150E6E5F2570E1F45D
:20C30000FE0CA891D95DCCFDB2F4F7D16A8B337B2374BDB2F1712FAA8AF418AC7B98AC8305
:20C3200019AF73A283D448FB93A9B5242DB0B2A34763AC97B64CB8B9F4B25B8CEC6ED5FD26
:20C3400063525DFDA3E6AEA18CD7B9D17E8B61E88FD4A0F293EEEA6D4E0DB332A89BD90589
:20C360009BFBB00BE56755D08BB2DB531D0B5441FF002A8AD0101F447EA411A79A8999FB4C
:20C38000A9B462DB3281B38062B5ED70E30FC96A8BA0CE0F01EA80A97A2F17B651A6F09B70
:20C3A0004B61BC331C7AABBA88BD5CA6EC31C7AAB606D71C7AAB751178B00C1647AAB20BC0
:20C3C000203D45ED1117E6915FA88888888888888888888888888888888888888888888878
:20C3E0008888888888888888888888888888888888888888888888888BF08750E95CF916D7
:20C40000765F2D4BA2888B94361696D47B6B4C74456DA22591111111111111111111111165
:20C4200011111111111111683D6B07DCD44B7D17965EB3BB2C4CB22C0E91595117ABC44414
:20C4400044444444444444444444444444444444444444444444444444444444444444445C
:20C46000444445FFD9002A67FFD8FFE000104A46494600010201004800480000FFDB0043F0
:20C48000000101010101010101010101010101010201010101010201010102020202020275
:20C4A000020202030304030303030302020304030304040404040203050504040504040410
:20C4C00004FFDB0043010101010101010201010204030203040404040404040404040404F2
:20C4E0000404040404040404040404040404040404040404040404040404040404040404BC
:20C50000040404040404FFC0001108002C005503011100021101031101FFC4001E0000018A
:20C52000030501010000000000000000000006000407010305090A0802FFC400491000009E
:20C5400004040302070B070B0500000000000304050600010708021314091511162324339B
:20C56000439317253134353645515354630A1221447375A318192646485255839194B361E5
:20C58000647174B5FFC4001A010002030101000000000000000000000000010203040506A3
:20C5A000FFC400291101000103020405050100000000000000000304131401020511258379
:20C5C0000612243133152123324352FFDA000C03010002110311003F00E968A1232744903C
:20C5E000458398824E7294B0CBC339CE3D3B9E38274B6A01E0B38A368F8A145591124FAE20
:20C60000E5AF5EB91C7060BF103CEE64BDEE063B185900F3B94B83DC0CF6306403E2F461A3
:20C62000D267D1C62219667C3D097783F50859676915AFB694DBC6665944A8A584FA78248E
:20C640002619E1F9D28D3B37EDDFFAA1E50DC488A005004797174B5FF596D06EF2975274EF
:20C66000B30B5556A45ADD4161530472AAC55BC6551C4B0D2574E442C128191812E5B34EE1
:20C68000192DCE07182082F6B192AD346256CDAB8996F55F53A4F66350A86DAEAE545A4207
:20C6A000E059D9E2B75C192DA7AD712ED5C6FAEE8A788994273A8361330ADE15BA73C08EA8
:20C6C000656CB9554C34D870CF6329854849E2E1EEF7D5B501546B23BD4735AA53F6EE1BF8
:20C6E000463E45D8C7AF5521E14CA89B05C2D0198CD3465B4C46E2B6079329C1564D942187
:20C70000835B855BE61961BEC332818400F12694C5AF3211741D18BCBBB1854E69F0ACE256
:20C72000F4813EA26A5238FC4DF4756155A84CB693BF41251A2DCE861F3FC5C53312269E5A
:20C74000ABA5AD55F4760ED0A2CD4B7B7F5E598AE374CCDA8745DA8FDADE8E7C81E045644C
:20C76000375216D7D492D4DD68248E24370E04AB889B40D9D4F2C6C64A4DC2148B61906A19
:20C7800065CD766ED39F3D069AE9AFB2EA3DB856940BA3B133ED6B67AFA489D05B55404EE6
:20C7A0005BBACAB359D94EB7338DCE469EAE3548B1EA1102EFE18C10492821E09457C7696C
:20C7C000A62DE05B5B10A0818D90431281B5CB5D74E7A69F63454DED9C9746FCB53B8FA6D3
:20C7E000B7754D29D568AD2B37DED6AE54C5D65AAC49F23B9D25414697F746582269443208
:20C80000181288182690E90C247F985B2CBE7932E44303091C0381B657E535269286DA6600
:20C82000331B29EDC67B1508A34DA6828C57213915353CBE909132DF0810410A3A74ACD2DC
:20C84000A0252652B2772A3941E37DD520D103C41E29E1C529CA72F5C5A4B70030715EDD9E
:20C86000B4DAAB9C934EA918A866DF26508BB9C0466AB435C57446BA11756398042EAA3972
:20C8800035750D102A676E3DB19703BDF4E6B69CFB74C42240FF00E9C739A11838B6DDD28E
:20C8A00031BCDFA1750D4FEFB7926B7BFC1A9868A3839B6A01CAE636D8586F65A9AA661423
:20C8C0003F0B7643BC60C55DB41518D79A76FAC44FFBC15D51C5A3FE77348578001436B9C7
:20C8E000DD30FE26D7A7C4BEED640DC8FF00787A15D063F9D56F214C5E68B4928DC8FA356E
:20C90000828FC8F6E08B1030E2B5FF005D92D794AB2B9C97DDC9A968BFE02D0C97D9FB4B5F
:20C920002BAD35E6AE4A96D77EB7C635A93A8B568E1455EC8FF8E05DB43BA49DD1F6A7D98D
:20C9400033A85CBA96E04AA2AAA30DCAAA25BDD35FACF03EDBEBFD9171E3745C4245365E35
:20C96000BC6FAFB35F4D56DD41A68F46F547A76F22639F693E1A46F78202F0258D982067D6
:20C98000245F8464A9903F911D48A6BACCD326DBEA5958C824D20BBD6123F18A95319A85B9
:20C9A00069955D3293CB2CD3935BD0F0C9AAAA217F0E35BCB4DAAEA070F95F180E3935BF2C
:20C9C0002B542E7DD4AF34D242C9E40E29B43BDDC8EF4703F7716BF9B971FC574637B7FC38
:20C9E00028C6D00658BEC7E93E45398B4FF53EC8070A8AAE93F04184932ED7BD07FAC796D8
:20CA0000074A445514FE5114B6CB338C59C0FDB8EA7D2FC28E0F139FC497FA352C5DD95DB7
:20CA2000DE194FE1B961EB355376A238FCAD2A4BC8F154F695482083DF94E4D3871FE9C8D0
:20CA4000CCC2A2EF23E114E63E39CEBA5E6DD742A1A9E3F6FAE450F64B8853F00B9D125966
:20CA6000BBC1B50AF55D8249D7A85C9320E6622EF12E9ED13CE13A7943F4777B05A231C536
:20CA8000400874DEF26C1E43E2C7472E4737199419EE51751352EABA6A965CF0E95A8DD62C
:20CAA000DF6928BA8E8236E16B1ECAF2DA6151B9CA9AB743D2F43F51162ABF5973E34ECD1E
:20CAC0002FF43C6351A78D41778E2339977675898A068721652294A86B861F8CD946023674
:20CAE0005C03AA84B47BBFAED4EA8703A8CF89FAEB08FA2BC3541D9BD79AFA2C7D351EC2BB
:20CB0000AF15495CFB6C32C4D55E6D9D3102C73468BE3007158801999DBCFD23D2E77B683B
:20CB2000B63CC55E9522B7F60B6D5057FD900DA1E59CC9137B55169A68B95D474AABDA466B
:20CB4000D6275F5697445ED6C56616B16FD54C8252354AA66C25222F345495D2CE32494639
:20CB6000941C6AEAD93AD2FC88BC91E0BA28EC50C7F8999EA366AD21E916DAEF0444A75326
:20CB800029DE8E65B4F06A2F91DE884E34D3A0E98E123857AD0450A2EA986F0681EA6FC91D
:20CBA00095A08F9A98E87BD32BD373D2F642B2DEF36AD395DA1215493CCE29FC377D718457
:20CBC000AEB0307A308418BE66565E66774A27271256ABC286EFC997B2C4804B71DAEC6EA4
:20CBE0003DD073D242B5105A8C92A6BFEB862923A205DA8D0F12417D39B3B605ECBB66841D
:20CC000060B2F9DB97AA24CC09CE483BEAD9345283FB3F2426911FF1627848DF7A619BB289
:20CC2000EF64F53AF372CF5BE747EBCD39AA2BB5CBAECAE5797D429E5C4BE9E5929C5AD669
:20CC4000BFB3C98FE6D58BDAD951FDED4A8F2338CFFF00707001458B3011BE99D3D7695B1D
:20CC600053CC9A2546DA79016401C5EA668C9193D9178B3051BC241EE09EBD0953BA307F18
:20CC8000DB17CA8BB0A146E83D46AF3E943F5854BB78B31A1442269D8E53939CCCAE2A0B07
:20CCA000C3E19633A24E5C3FD62CB71FF94581146147C73106104171CFC38C4C73C78E72C5
:20CCC00097FAC4C2983162C18B0CF0CE729CF83C1FF339401900944DE0C329611B14A5EA4A
:20CCE00094E7C1F44E179768571A81BC529CF10D8E7C129F070E29FAA0F2833C6606C53958
:20CD0000CA62629FD3E1E19F0F86185ACC13F7A7007CF0CFD73FEB38029C339F867C300216
:20CD2000801400A005007FFFD90008C24124AA0151248A694C6F7645446C696E4B537769A6
:20CD400054634800412F070142277E000A422786000042277A000042277C000042277600D5
:20CD6000004227880000422780FFFF4227788000422770000042277200004227740000C128
:20CD80001F42204500004220470000420024000052294F84000084000C84001D84002F8408
:20CDA000001D84002F4C2B0D840A2D840A35840A38840A3B60302540841F21841F28841FEB
:20CDC00035841F35841F37841F3E841F4B841F4B841F4D841F54841F61841F61841F618438
:20CDE0001F61841F61841F6158263483F30383F30B83F31583F31F83F32883F33183F336EE
:20CE000083F33E46262883F33683F34346262E83F34A83F34E46262283F35183F358604084
:20CE2000238200081018202830380A121A220C141C240E161E262E01020304050607090BEF
:20CE40000D0F11131517191B1D1F21232527292A2B2C2D2F31323334353637393A3B3C3DCD
:20CE60003E3F4C289484283784283E84284284284949288B84284E84285984286B462DED0B
:20CE8000842C0C842C13492C83841C59841C61841C66432145000000625612FB83DCF063FB
:20CEA00067695F64756D79000000000000000000000000832C9A6367695F6C6F67696E0090
:20CEC00000000000000000000000839C646367695F706F7274000000000000000000000078
:20CEE000008275176367695F736574706F7274000000000000000000839AA66367695F76B6
:20CF00006C616E000000000000000000000000831E8E6367695F736574766C616E00000018
:20CF200000000000000082FC1A6367695F64656C766C616E0000000000000000008390EFDF
:20CF40006367695F70766964000000000000000000000000828AAB6367695F766964000000
:20CF6000000000000000000000000082E90A6367695F61646476696400000000000000003E
:20CF80000000825AA76367695F64657669636500000000000000000000824DB36367695FF8
:20CFA00064657461696C0000000000000000000082CEFF6367695F73746174697374000011
:20CFC00000000000000000830E866367695F7472756E6B000000000000000000000082A151
:20CFE000FC6367695F6D6972726F7200000000000000000000835FE66367695F70617373F7
:20D000000000000000000000000000008296EE6367695F7379730000000000000000000019
:20D0200000000082910B6367695F7472617000000000000000000000000083CDF663676910
:20D040005F6261636B7570000000000000000000008364A86367695F62616B5F64617461B3
:20D06000000000000000000083A2F66367695F72657365740000000000000000000000835D
:20D08000D9746367695F716F73000000000000000000000000008396F66367695F7170627A
:20D0A000617365000000000000000000008395046367695F7164736370000000000000006E
:20D0C000000000008398DC6367695F713170000000000000000000000000000000000000B5
:20D0E000000000000000000000000000000000000000422EA2000042178C0000421672006F
:20D100000046166C818EE7818EF5521774818F1D818F34818F4A818F60818F78818F9446C3
:20D120001786818FB1818FCE42156200004219C7000100E52524A1F582E43426F5837593D3
:20D1400000E00525229000269E301704900026A1E475F001120089CD020080D32010E57F12
:20D160002ED2108018EF540F2490D43440D4FF30140BEF24BFB41A0050032461FFE52660B5
:20D180000215260529E529700205283017119000269EE475F001120089CDEF020081240281
:20D1A00000DD717403D2178003E4C217F5259000269E120089FBE4F526F528F529E52660D8
:20D1C000087F201200D17D80F47527FFC211C210C212C213C215C216C2181200D145FF70CB
:20D1E0000E3017067F001200D18EAF29AE2822B42563C2D5C2141200D145FF24D0B40A0092
:20D20000501A75F00A782630D50508B6FF0106C6A426F620D5047002D21380D824CFB41ADA
:20D2200000EF5004C2E5D2140200D3BBD21180C4D21080BED21280BAD2D580B8D21580B231
:20D240007F201200D17D2012077401B5260040F01200D133FF1200D17D0200D1BDD218D255
:20D2600016808F1200D133FB1200D133FA1200D133F94A4B700679927AD47B8120123DE5A5
:20D280002660397E00E9C0E02EF9EAC0E03400FA120080D3F9D0E0FAD0E0C960060EEE65A1
:20D2A0002770E2C2D5EBC0E0EAC0E0E9C0E0EE1200D403D0E0F9D0E0FAD0E0FB120080D386
:20D2C000FF6096EBC0E0EAC0E0E9C0E01200D17DD0E02401F9D0E03400FAD0E0FBE52704F4
:20D2E00060DAD527D70200D2597BFF7AD379FFD2128089791080027908C216C2188008D230
:20D30000D5790A8004790AC2D5E527047002F527E4FAFDFEFF1200D133FC7B0820111612B3
:20D3200000D133FD7B1030100C1200D133FE1200D133FF7B20EC3382D592D55013C3E4303A
:20D3400010069FFFE49EFEE42011039DFDE49CFCE4CBF8C211EC700CCFCECDCCE824F8F857
:20D3600070F38017C3EF33FFEE33FEED33FDEC33FCEB33FB994002FB0FD8E9EB301105F890
:20D38000D0E0C448B211C0E00AEC4D4E4F78207B0070C2EAB5270040BCC0E01200D405D02C
:20D3A000F0D0E0201104C4C0E0C4B211C0F01200D166D0F0D5F0EA0200D1BD120084D5D278
:20D3C0006353D2F358D2304CD22C42D2F74FD2FF44D2FF49D24643D30555D2E946D2E9451C
:20D3E000D2E947D4AF50D2342DD2382ED25F2BD23C23D25D20D49B2AD1F2480000D2553F07
:20D400003F3F00790AA2D5201314301509B910020404B9080104A2D5201602500104201230
:20D420006D9212B526005036C0E07F2030131A7F30A2127216721550101200D45EC212C232
:20D4400016C215C2187F308010301503E9C0E01200D17D301503D0E0F9D0E0B526CA30150A
:20D46000197F30B9100D1200D17D7F583014077F788003B908041200D17D3012067F2D02F7
:20D4800000D17D7F202018F77F2B2016F222921280CC286E756C6C2900D2111200D1333057
:20D4A00011F7C211782630D50108F60200D1F21200D1337F4960087F4310E7027F5814C07E
:20D4C000E0EF1200D16E743A1200D16ED0E0600DC0E0C41200D166D0E01200D166D2137510
:20D4E00026040200D2F3E52A301C0104F8232824A1F582E43425F583759300229000259E2A
:20D50000301C04900025A1E475F001120089CD020080D360E6C52E7002152D14C52E201C2E
:20D5200005FF0200DDF19000259E74FFF5F0020089E4FF0202DA81E52B6006D52B037F00A7
:20D5400022201C101200DD99EF6008052EE52E7002052D229000259E120089C4120080D35B
:20D56000FF60E59000259EE475F001120089CD80D71200D541EFC0E01200D532D0E040F15A
:20D580008091D21C8002C21C9000259E120089FBE4F52CF52AF52DF52E752B00C21BC21982
:20D5A000C21AC21D1200D4FCFF7005AF2C7E0022B425321200D4FCFF24D0B40A00500C7570
:20D5C000F00AC52BA4252BF52B80E824CFB41A00EF5002C2E50200D81CD21A80D6D2198099
:20D5E000D2D21D80CEEF1200D53250091200D571EF600F80A4EFC0E01200D541D0E06F60AB
:20D6000098EF70040200D68C1200D513809D1200D541EF6077E52B7008052B80041200D583
:20D6200041EF6017201D111200D4E6E475F001120089CDEF12008124D52BE2201D04052A7F
:20D64000052C80AF1200D537EFC0E01200D532D0E050051200D513E4FF201D111200D4E6A8
:20D66000E475F001120089CDEF12008124EF70D4201D04052A052C0200D5F3E52B6002053D
:20D680002B1200D5711200D537EF70BD301C05E41200D513E52C60030200D5AB7EFF7FFFAD
:20D6A00022201D1474FFFCFDFEFF1200D4E6120089C4120083C2052A0200D599D0E080CC71
:20D6C0007900800A7910800679088002790AD21EE52B6002052BE9C0E01200D571EF60DC14
:20D6E0001200D541BF2D04D21B8003BF2B0B1200D571EF60C71200D537D0E0B40A028034FD
:20D70000B40802802FBF302870027408C21EC0E01200D537D0E0BF78028003BF5816052B30
:20D72000D52B028007D52B04D21E800B7410801B7002740ABF000BEFF8E4FCFDFEFF020045
:20D74000D7C4C0E0EF1200D513D0E0F9E4FCFDFEFFE9C0E0ECC0E0EDC0E0EEC0E0EFC0E063
:20D760001200D537EFF8D0E0FFD0E0FED0E0FDD0E0FCD0F0E8604DB461004007B47B0050BE
:20D7800002C2E524D0503DFA24F6500724F95034240AFAEAB5F000502BCFA9F0A42FFF9255
:20D7A000D5E9C5F0CEA4A2D53EFE92D5E9C5F0CDA4A2D53DFD92D5E9C5F0CCA4A2D53CFC86
:20D7C000C21E808DE8C0E0201D30201E09052C301B04120089271200D4E6120089C4052A84
:20D7E00020190C201A0FEE8FF012008228800B120083C28005EF12008124D0E01200D513BB
:20D800000200D599201D131200D4E6120089C4052AE52D852EF01200822880E4120084D5AE
:20D82000D67B53D6C458D5DD4CD5D942D5B348D6C84FD6CC44D60E43D6C049D6CC55D6A14D
:20D8400046D6A145D6A147D5E12AD8044E0000D5E590007004E0F54090007005E0F541858B
:20D860004082854183E020E7077E007F00C2D72289428A435407F5451200DA4CE02402F597
:20D8800044500205451200D8F3053AE53A7002053BE5402544F540E541354530E604C2E696
:20D8A0002430F5411200D91390007004E540F090007005E541F0AE45AF44D2D722900070FB
:20D8C00010E020E61EA3EDF0A3E9F0A3EAF0EC5407D2E690007010F00538E53870020539B2
:20D8E000D2D7227C007D00C2D72290007010E0A2E6B32275F001800375F0041200D9137894
:20D90000407F06900070921200DA3490007090E5F0F02290007090E0540770F7221200D9DA
:20D9200080900070087430F0900070107508101200D96BE490007004F090007006F0743066
:20D9400090007005F090007007F0751D10751C10751E00751F30758330758200E4F07538A1
:20D9600000753900753A00753B0022E4A808F0A3D8FC221200DA2A1200D91D1200D9BE2272
:20D980009000D9B475080A797078601200DA3B7518C07519A8751A00751B647510C075112A
:20D9A000A87512007513017514FF7515FF7516FF75170022000B78667788C0A80064900022
:20D9C000706AE0440CF0229000706AE054F3F0229000706AE04401F0229000706AE054FE4B
:20D9E000F0229000706AE04402F0229000706AE054FDF0229000706AE04440F022900070E6
:20DA00006AE054BFF02290007000E04410F02290007000E054EFF02290007000E04420F0E8
:20DA20002290007000E05420F0229000700AF00000000022E6F008A3DFFA2289A0E493A383
:20DA4000F208B800030989A0D508F222A3E58330E603758330224745542000696E64657868
:20DA60002E68746D00706F73745F75726C3D002E006367695F6C6F676F757400636F6E667A
:20DA800069672E62696E006367695F62616B5F64617461006367695F006367695F6C6F6730
:20DAA000696E004C6F67696E004F6E6C79206F6E6520757365722063616E206C6F67696E28
:20DAC000006367695F6465766963650077726F6E672070617373776F7264006C6F67696E6B
:20DAE0002074696D656F7574006367695F706F7274006367695F716F73006367695F717050
:20DB000062617365006367695F713170006367695F7164736370006367695F64656C766C70
:20DB2000616E006367695F766C616E006367695F7472756E6B006367695F6D6972726F72E0
:20DB4000006367695F737973006367695F70617373006367695F74726170006367695F733D
:20DB600065747674797065006367695F70766964006367695F736574766964006367695F9C
:20DB8000766964006367695F616464766964006367695F64656C766964006367695F7265D1
:20DBA000736574006367695F636C7273746174006367695F73746174697374006367695F5A
:20DBC000616464766C616E006367695F736574766C616E006367695F7365747669643D2559
:20DBE000640075C7AA75C755759D0275C7AA75C75575C600787FE4F6D8FD75814FD20D02B8
:20DC000000DC2D020202F0E493A3F85407240CC8C333C4540F4420C8834004F4568001467F
:20DC2000F6DFE4800C01020408102040809000CD2CE47E019360CCA3FF543F30E509541F2F
:20DC4000FEE493A360010ECF54E0B4E026E493FBA3E493FAA3E493F9A3E493C083C0821236
:20DC6000008124D082D083A309E970010ADFEADEE880BE54C025E0602B408CE493A3FAE415
:20DC800093A3F8E493A3C8C582C8CAC583CA759300F0759300A3C8C582C8CAC583CADFE371
:20DCA000DEE1808DE493A3F8E493A34003F68001F208DFF40200DC3168656C6C6F3F3F3F05
:20DCC0000068696869232323006D616320777269746500676F206C6F6164657200636C6F12
:20DCE0007365746D006D61632072656164002573006D6163006D6F64656C207265616400E8
:20DD00006D6F64656C3A004447532D313232345400667776657220726561640066777665F2
:20DD2000723A00322E30302E303600726263686B004661696C004F6B000A454550524F4DD1
:20DD40002052656D61696E65642053697A653A2025640A00496E69742066696E697368653C
:20DD6000642E0A000A4D414320496C6C6567616C00EFB40A08740D1200DD7D740A30981159
:20DD8000A899B8130CC2983098FDA899C298B811F63099FDC299F5992210210D1200801839
:20DDA000BF0D027F0A0200DD7190002F0DE0FF22E4FFFE120080D3600C0FEF70010E09E9CE
:20DDC00070F10A80EE224447532D3132323454000012233445FE44656661756C74006164EA
:20DDE0006D696E002573004447532D31323234540090002F0DEFF0D22122EF6402600301A6
:20DE0000DFAB90001AAEF0A3F090001AABE0FBA3E0FAA3E02415F9E43AFA120080D3FFB40B
:20DE2000073090001AABA3E0FAA3E02416F9E43AFA740112008108D39405500301EF5C9060
:20DE4000001AABA3E0FAA3E02415F9E43AFAE401EF58EFB4052290001AABE0FBA3E0FAA36D
:20DE6000E02416F9E43AFA740112008108D39405500301EF5C01DFA490001AABE0FBA3E025
:20DE8000FAA3E02415F9E43AFA120080D3FF700301EF5C20E40301DF5090001AABA3E0FA8F
:20DEA000A3E02416F9E43AFA74FF12008108600301EF5C1202A3B890001AABE0FBA3E0FABB
:20DEC000A3E02417F9E43AFA7401120080E9B4052090001AABE0FBA3E0FAA3E02415F9E464
:20DEE0003AFAE412008124900019C97480F001EAE090001AABE0FBA3E0FAA3E02415F9E4EC
:20DF00003AFA120080D3540F14700301E64024FE603014700301EA5124FE700301EA5124ED
:20DF2000FE700301EA512406600301EF5C900019BEE0FBA3E0FAA3E0240DF9E43AFAE401F2
:20DF4000E653900019C97404F01202D23101EBF390001AABE0FBA3E0FAA3E02415F9E43A38
:20DF6000FA120080D3540F6403600301EF5C90001AABA3E0FAA3E02416F9E43AFA74FF12A4
:20DF8000008108600301EF5C90001AABA3E0FAA3E02417F9E43AFA7401120080E9640560EF
:20DFA0000301EF5C1202A3B801DED1900024A3E0FBA3E0FAA3E0F990001AAEE0FEA3E0FF10
:20DFC000E92FF9EA3EFAE41200812490001AAB7401F0A37419F0A374D4F0900024A3E0FB8C
:20DFE000A3E0FAA3E0F9900019B8EBF0A3EAF0A3E9F0240EF9E43AFA900019C4EBF0A3EADB
:20E00000F0A3E9F0900019B8E0FBA3E0FAA3E0240CF9E43AFA120081AEFFAEF0BE0807BFAD
:20E02000060402025AEC900019B8E0FBA3E0FAA3E0240CF9E43AFA120081AE7004E5F06421
:20E0400008600301E7B0900019C4E0FBA3E0FAA3E02402F9E43AFA120081AEFFAEF09000D0
:20E060001AAEEEF0A3EFF0D394DCEE9405400301E7B0900019C4E0FBA3E0FAA3E0F9120080
:20E0800080D3B44511E92406F9E43AFA120081AEE5F0543F600301E7B01202DAD9900019EB
:20E0A000C4E0FBA3E0FAA3E02410F9E43AFA120083FAC31200836E6025900019C4E0FBA3B7
:20E0C000E0FAA3E02410F9E43AFA120083A574FFFBFAF9F8C31200836E600301E7B0120236
:20E0E0006F56EFF47002EEF4600301E7B0900019C4E0FBA3E0FAA3E0240CF9E43AFA12008E
:20E1000083A5900019B8E0FBA3E0FAA3E02406F9E43AFA1202540A900019C4E0FBA3E0FA29
:20E12000A3E02409F9E43AFA120080D3B40149120080D3FF90001AABE0FBA3E0FAA3E02403
:20E1400014F9E43AFAEF12008124900019C4E0FBA3E0FAA3E0240CF9E43AFA120083A590A1
:20E16000001AABE0FBA3E0FAA3E02404F9E43AFA120083C20202C48A900019C4E0FBA3E052
:20E18000FAA3E02409F9E43AFA120080D36411600301E280900019C4A3E0FAA3E02414F986
:20E1A000E43AFA900019C1EBF0A3EAF0A3E9F0900024A3E0FBA3E0FAA3E0F91202BD23905A
:20E1C0000019C4E0FBA3E0FAA3E02409F9E43AFA120080D3FF90001AABE0FBA3E0FAA3E0B5
:20E1E0002414F9E43AFAEF12008124900019C1E0FBA3E0FAA3E02402F9E43AFA120081AE73
:20E20000FF90001AABE0FBA3E0FAA3E0F9E5F08FF012008228900019C1E0FBA3E0FAA3E081
:20E22000F9120081AEFF90001AABE0FBA3E0FAA3E02402F9E43AFAE5F08FF012008228909E
:20E240000019C4E0FBA3E0FAA3E0240CF9E43AFA120083A590001AABE0FBA3E0FAA3E02437
:20E2600004F9E43AFA120083C290001AABE0FBA3E0FAA3E0F9120081AEFFAEF00202D8A3AC
:20E28000900019C4E0FBA3E0FAA3E02409F9E43AFA120080D36406600301E7B0900019C4C1
:20E2A000E0FBA3E0FAA3E02414F9E43AFA900019BEEBF0A3EAF0A3E9F01202DBF390001974
:20E2C000BEE0FBA3E0FAA3E02402F9E43AFA120081AE6F7003EE65F0600301E7B090002E4F
:20E2E00058E4F0A304F090002E58E0FEA3E0FFC39405EE9400400301E3C47C007D2B1200E6
:20E30000813874D42FF974193EFA7B0190001AABEBF0A3EAF0A3E9F02415F9E43AFA12000E
:20E3200080D3700301E3B1900019BEE0FBA3E0FAA3E02402F9E43AFA120081AEFFAEF0909B
:20E34000001AABE0FBA3E0FAA3E0F9120081AE6F7003EE65F0705AE92402F9E43AFA1200C2
:20E3600081AEFFAEF0900019BEE0FBA3E0FAA3E0F9120081AEB50739E5F0B5063490001AF2
:20E38000ABE0FBA3E0FAA3E02404F9E43AFA120083A5900019C4E0FBA3E0FAA3E0240CF913
:20E3A000E43AFA120083FAC31200836E700301E75690002E59E004F0700790002E58E004E3
:20E3C000F001E2E6900019BEE0FBA3E0FAA3E0240DF9E43AFA120080D36402600301E7B03A
:20E3E00090002E58E4F0A304F090002E58E0FEA3E0FFC39405EE9400502D900019E975F0D4
:20E400002BEF12008458EE75F02BA42583F583759300E0605E90002E59E004F070CB900056
:20E420002E58E004F080C290002E58E4F0A304F090002E58E0FEA3E0FFC39405EE9400501B
:20E440002F900019E975F02BEF12008458EE75F02BA42583F583759300E0640760159000F4
:20E460002E59E004F070C990002E58E004F080C001E7B090002E58E0FEA3E0FF7C007D2BAC
:20E480001200813874D42FF974193EFA90001AAB7401F0A3EAF0A3E9F0900019C4E0FBA3DE
:20E4A000E0FAA3E02409F9E43AFA120080D3FF90001AABE0FBA3E0FAA3E02414F9E43AFAE4
:20E4C000EF1200812490001AABE0FBA3E0FAA3E02416F9E43AFA74021200812490001AAB99
:20E4E000E0FBA3E0FAA3E02417F9E43AFAE412008124900019BEE0FBA3E0FAA3E02402F9F9
:20E50000E43AFA120081AEFF90001AABE0FBA3E0FAA3E0F9E5F08FF012008228900019BE03
:20E52000E0FBA3E0FAA3E0F9120081AEFF90001AABE0FBA3E0FAA3E02402F9E43AFAE5F08B
:20E540008FF012008228900019C4E0FBA3E0FAA3E0240CF9E43AFA120083A590001AABE088
:20E56000FBA3E0FAA3E02404F9E43AFA120083C290001AABE0FBA3E0FAA3E02415F9E43A90
:20E58000FA741112008124900019D0E0FCA3E0FDA3E0FEA3E0FF90001AABE0FBA3E0FAA31D
:20E5A000E0240CF9E43AFA120083C2EF2401FFE43EFEE43DFDE43CFC90001AABE0FBA3E0C3
:20E5C000FAA3E02410F9E43AFA120083C2900019BEE0FBA3E0FAA3E02404F9E43AFA120095
:20E5E00083A5EF2401FFE43EFEE43DFDE43CFC90001AABE0FBA3E0FAA3E02408F9E43AFA19
:20E60000120083C290001AABE0FBA3E0FAA3E02422F9E43AFAC003C002C00190001AABA3DE
:20E62000E0FAA3E02420F9E43AFA90002DA8EBF0A3EAF0A3E9F0D001D002D0031202C9BCE0
:20E64000900019BEE0FBA3E0FAA3E0240DF9E43AFA741012008124900019BEE0FBA3E0FA3C
:20E66000A3E0240DF9E43AFA120080D3440212008124900019BEE0FBA3E0FAA3E02414F900
:20E68000E43AFA90002E5AEBF0A3EAF0A3E9F074021200812490002E5AE0FBA3E0FAA3E056
:20E6A0002401F9E43AFA74041200812490002E5AE0FBA3E0FAA3E02402F9E43AFA74051240
:20E6C00000812490002E5AE0FBA3E0FAA3E02403F9E43AFA74781200812490002E5AE0FBD4
:20E6E000A3E0FAA3E02404F9E43AFA74011200812490002E5AE0FBA3E0FAA3E02405F9E4BC
:20E700003AFA74011200812490002E5AE0FBA3E0FAA3E02406F9E43AFA74041200812490AC
:20E72000002E5AE0FBA3E0FAA3E02407F9E43AFA74021200812490001AAEE4F0A37430F0AA
:20E74000900019BEE0FBA3E0FAA3E0240CF9E43AFA747001EE77E4900019C9F0900019BE3F
:20E76000E0FBA3E0FAA3E0240DF9E43AFA120080D330E22490001AABE0FBA3E0FAA3E0248D
:20E7800015F9E43AFAE412008124900019C97420F01202D23101ED39900019BEE0FBA3E0BF
:20E7A000FAA3E0240DF9E43AFA120080D320E40301ED39900019BEE0FBA3E0FAA3E0240C95
:20E7C000F9E43AFA120080D3C4540F75F004A4FFAEF090002E58EEF0A3EFF02414FFE43E23
:20E7E000FEC390001AAFE09FFF90001AAEE09EFEF0A3EFF0D39400EE9400403490001AAB89
:20E80000E0FBA3E0FAA3E02408F9E43AFA120083A5900019BEE0FBA3E0FAA3E02404F9E45F
:20E820003AFA120083FAC31200836E600301EE4390001AABE0FBA3E0FAA3E02410F9E43A3F
:20E84000FA120083A5900019BEE0FBA3E0FAA3E02408F9E43AFA120083FAC31200836E7040
:20E860006690001AABE0FBA3E0FAA3E02410F9E43AFA120083A590001AABA3E0FAA3E0240A
:20E880000CF9E43AFA120083C290001AABE0FBA3E0FAA3E02415F9E43AFA120080D3FF30F6
:20E8A000E425900019C97401F0EF54EF1200812490001AABE0FBA3E0FAA3E02416F9E43A0E
:20E8C000FA74021200812490001AABE0FBA3E0FAA3E02415F9E43AFA120080D3540F14B407
:20E8E0000800400301EE3F9000E8F675F004A4C58325F0C583730200E9160200E9320200EC
:20E90000E9B50200EC540200ED3C0200EE0A0200EE430200EC39900019C9E030E0117403AE
:20E9200012008124900019C97440F01202D23101ED39900019C9E030E078900019BEE0FBB0
:20E94000A3E0FAA3E0240DF9E43AFA120080D36412705F90001AABE0FBA3E0FAA3E0241562
:20E96000F9E43AFA740312008124900019BEE0FBA3E0FAA3E02404F9E43AFA120083A59013
:20E98000001AABE0FBA3E0FAA3E02408F9E43AFA120083C2120083A5EF2401FFE43EFEE4F2
:20E9A0003DFDE43CFC120083C274421202D22401EAC101ED39900019BEE0FBA3E0FAA3E0D5
:20E9C000240DF9E43AFA120080D320E00301EA5490001AAFE02401FF90001AAEE03400FE87
:20E9E000E4FCFD90001AABE0FBA3E0FAA3E02408F9E43AFA120083C274101202D224900058
:20EA00001AABE0FBA3E0FAA3E02410F9E43AFA120083A5EF2401FFE43EFEE43DFDE43CFC6A
:20EA2000120083C290001AABE0FBA3E0FAA3E02415F9E43AFA74181200812490001AABE08D
:20EA4000FBA3E0FAA3E02417F9E43AFAE41200812401EB4DD390001AAFE0940090001AAEA3
:20EA6000E094004045900019C9E04402F090001AABE0FBA3E0FAA3E02408F9E43AFAC003E5
:20EA8000C002C001120083FA90001AAEE0FEA3E0FFE4FCFDEB2FFFEA3EFEED39FDEC38FC4D
:20EAA000D001D002D003120083C2900019C9E05403700301EC361202D231EF4E700301EE94
:20EAC00043900019C9E0FF30E52C90001AABE0FBA3E0FAA3E02415F9E43AFAE4120081244C
:20EAE000900019BEE0FBA3E0FAA3E0240DF9E43AFA741401EE56EF30E46990001AABE0FB29
:20EB0000A3E0FAA3E02410F9E43AFA120083A5EF2401FFE43EFEE43DFDE43CFC120083C2B2
:20EB200090001AABE0FBA3E0FAA3E02415F9E43AFA74141200812490001AABE0FBA3E0FA6F
:20EB4000A3E02417F9E43AFAE412008124900019BEE0FBA3E0FAA3E0240DF9E43AFA741142
:20EB600001EE56D390001AAFE0940090001AAEE09400407790001AABE0FBA3E0FAA3E024D9
:20EB800015F9E43AFA120080D320E45F120080D344101200812490001AABE0FBA3E0FAA3C7
:20EBA000E02417F9E43AFAE41200812490001AABE0FBA3E0FAA3E02410F9E43AFAC003C096
:20EBC00002C001120083FA90001AAEE0FEA3E0FFE4FCFDEB2FFFEA3EFEED39FDEC38FCD0FC
:20EBE00001D002D003120083C28008E490001AAEF0A3F0D390001AAFE0940090001AAEE0F9
:20EC000094005008900019C9E030E12A90001AAFE02428F090001AAEE03400F0900019BE43
:20EC2000E0FBA3E0FAA3E0240DF9E43AFA74181200812401EE6401ED39900019C9E020E0A8
:20EC40000301EE3F90001AABE0FBA3E0FAA3E0241501EE36D390001AAFE0940090001AAEFD
:20EC6000E09400403D90001AABE0FBA3E0FAA3E02408F9E43AFAC003C002C001120083FA61
:20EC800090001AAEE0FEA3E0FFE4FCFDEB2FFFEA3EFEED39FDEC38FCD001D002D0031200D5
:20ECA00083C2900019BEE0FBA3E0FAA3E0240DF9E43AFA120080D330E049900019C9E090EB
:20ECC000001AAB30E027E0FBA3E0FAA3E02415F9E43AFA74071200812490001AABE0FBA30E
:20ECE000E0FAA3E02416F9E43AFAE4800FE0FBA3E0FAA3E02415F9E43AFA74161200812493
:20ED000001EDCF900019C9E030E01A90001AABE0FBA3E0FAA3E02415F9E43AFA74051200B5
:20ED2000812401EE3FD390001AAFE0940090001AAEE09400400301EE4301EE3FD390001A74
:20ED4000AFE0940090001AAEE09400403D90001AABE0FBA3E0FAA3E02408F9E43AFAC00317
:20ED6000C002C001120083FA90001AAEE0FEA3E0FFE4FCFDEB2FFFEA3EFEED39FDEC38FC6A
:20ED8000D001D002D003120083C2900019BEE0FBA3E0FAA3E0240DF9E43AFA120080D3308D
:20EDA000E05590001AABE0FBA3E0FAA3E02415F9E43AFA74071200812490001AABE0FBA39F
:20EDC000E0FAA3E02416F9E43AFAE41200812490001AABE0FBA3E0FAA3E02408F9E43AFA83
:20EDE000120083A5EF2401FFE43EFEE43DFDE43CFC120083C2804CD390001AAFE094009019
:20EE0000001AAEE09400503B8035900019C9E030E02D90001AABE0FBA3E0FAA3E02415F985
:20EE2000E43AFA74071200812490001AABE0FBA3E0FAA3E02416F9E43AFAE4120081240270
:20EE4000008023900019BEE0FBA3E0FAA3E0240DF9E43AFA74101200812490001AAEE4F024
:20EE6000A37428F0900019BEE0FBA3E0FAA3E0240CF9E43AFA74501200812490001AABE030
:20EE8000FBA3E0FAA3E02408F9E43AFA120083A5900019BEE0FBA3E0FAA3E02408F9E43A7B
:20EEA000FA120083C290001AABE0FBA3E0FAA3E0240CF9E43AFA120083A5900019BEE0FB14
:20EEC000A3E0FAA3E02404F9E43AFA120083C290001AABE0FBA3E0FAA3E0F9120081AEFF39
:20EEE000900019BEE0FBA3E0FAA3E0F9E5F08FF01200822890001AABE0FBA3E0FAA3E02473
:20EF000002F9E43AFA120081AEFF900019BEE0FBA3E0FAA3E02402F9E43AFAE5F08FF012BF
:20EF2000008228900019BEE0FBA3E0FAA3E0240EF9E43AFA740575F078120082287F027E91
:20EF4000001201B58690001AABE0FBA3E0FAA3E02416F9E43AFA74021200812422900019F0
:20EF6000BEE0FBA3E0FAA3E02414F9E43AFA900019BBEBF0A3EAF0A3E9F090001AABE0FB47
:20EF8000A3E0FAA3E02424F9E43AFA9000155FEBF0A3EAF0A3E9F090001AABA3E0FAA3E0EB
:20EFA0002423F9E43AFA900012F4EBF0A3EAF0A3E9F090001AABA3E0FAA3E02418F9E43AE7
:20EFC000FA90001551EBF0A3EAF0A3E9F090001AABA3E0FAA3E0241AF9E43AFA900012F136
:20EFE000EBF0A3EAF0A3E9F090001AABA3E0FAA3E0241CF9E43AFA9000155CEBF0A3EAF03E
:20F00000A3E9F090001AABA3E0FAA3E0241EF9E43AFA90001554EBF0A3EAF0A3E9F090006F
:20F0200019C9E0FD30E6549000155FE0FBA3E0FAA3E0F9E4120081249000155FE0FBA3E0D2
:20F04000FAA3E02402F9E43AFAE4F5F01200822890001551E0FBA3E0FAA3E0F9E475F00163
:20F06000120082289000155CE0FBA3E0FAA3E0F9E475F0011200822801FDAAED30E7030149
:20F08000FDAA900019C9E020E10301FBB99000155FE0FBA3E0FAA3E0F9120080D36003011D
:20F0A000FBB990002D1C7481F0A374DAF0A37456F0A3E4F0A37404F0900019BBE0FBA3E05C
:20F0C000FAA3E0F91202BC20EF600301F15590002651F0900019BBE0FBA3E0FAA3E02405D2
:20F0E000F9E43AFA90002651E0FF7C0029F9EC3AFAA3EBF0A3EAF0A3E9F0120080D3FE641D
:20F10000206004EEB43F1174552FF582E43426F583759300E4F0801990002651E0FF04F005
:20F1200074552FF582E43426F583759300EEF080A27B017A2679551200DDB0EF4E60030178
:20F14000F1F478557C267D017B817ADA795B120086EC01F1F490002B407481F0A374DAF08E
:20F16000A37465F0900019BBE0FBA3E0FAA3E0F912029EF690002652EBF0A3EAF0A3E9F067
:20F1800090002652E0FBA3E0FAA3E04A4B701C90001557E06403700301F566900019BBE015
:20F1A000FBA3E0FAA3E0F90201D709900028B77481F0A374DAF0A37465F0A37481F0A37438
:20F1C000DAF0A3746FF0A37401F0A37426F0A37455F090002652E0FBA3E0FAA3E0F912026E
:20F1E0007AB59000155FE0FBA3E0FAA3E0F974011200812490002D1C7481F0A374DAF0A39A
:20F200007471F0A3E4F0A3740AF07B017A2679551202BC20EF704990001AABE0FBA3E0FA62
:20F22000A3E02404F9E43AFA120083A590001558E0F8A3E0F9A3E0FAA3E0FBC31200836EC6
:20F24000700301F2D6E4FFFEFDFC90001558E0F8A3A3A3E0C31200836E600301F3CD80761A
:20F2600090002D1C7481F0A374DAF0A3747CF0A3E4F0A3740AF07B017A2679551202BC200A
:20F28000EF701078557C267D017B817ADA7987120086EC90002D1C7481F0A374DAF0A37488
:20F2A00094F0A3E4F0A37404F07B017A2679551202BC20EF700301F38C90002C987401F0D3
:20F2C000A37426F0A3744CF07B017A26795512029B85EF4E702078557C267D017B817ADA86
:20F2E0007999120086EC900015577401F0E4FFFEFDFCA301F5149000155FE0FBA3E0FAA391
:20F30000E0F97402120081249000264CE0FBA3E0FAA3E0F9C003C002C0019000155FE0FBEC
:20F32000A3E0FAA3E02404F9E43AFA120084819000264FE0FEA3E0FF9000155FE0FBA3E0B6
:20F34000FAA3E02402F9E43AFAEE8FF0120082281202DAC9C004C005C006C0071202DC2FE4
:20F36000E4FCFD7B587A02F9F812008244D003D002D001D000EB2FFFEA3EFEE93DFDE83CCC
:20F38000FC900012F71200844C01FCDD90001AABE0FBA3E0FAA3E02404F9E43AFA1200831E
:20F3A000A590001558E0F8A3E0F9A3E0FAA3E0FBC31200836E603EE4FFFEFDFC9000155821
:20F3C000E0F8A3A3A3E0C31200836E602890002C6B7481F0A374DAF0A374A9F0A37481F019
:20F3E000A374DAF0A37499F07B817ADA79A31202B0E201FDAA9000155FE0FBA3E0FAA3E0F3
:20F40000F9120080D36401600301F51B90002D1C7481F0A374DAF0A374C1F0A3E4F0A374C0
:20F420000AF07B017A2679551202BC20EF600301F51B900019BBE0FBA3E0FAA3E0F9120249
:20F44000B47FEF4E70751202DB09E4FBFAF9F8C31200836E603D1202DB19EF5402FFE4FE04
:20F46000FDFC7B02FAF9F8C31200836E702590001AABE0FBA3E0FAA3E02404F9E43AFA1255
:20F480000083A590002E131200844C7FEA7E031202A6A890002C6B7481F0A374DAF0A37441
:20F4A000CCF0A37481F0A374DAF0A37499F07B817ADA79A31202B0E201FDAA90001AABE098
:20F4C000FBA3E0FAA3E02404F9E43AFA120083A5900015581200844C900015577402F0126B
:20F4E00002DAC9C004C005C006C0071202DC2FE4FCFD7B587A02F9F812008244D003D00298
:20F50000D001D000EB2FFFEA3EFEE93DFDE83CFC900012F71200844C01FA1A90002D1C74EB
:20F5200081F0A374DAF0A37499F0A3E4F0A37409F07B017A2679551202BC20EF7009900080
:20F54000155704F001FA1A90001557E0B4010F78557C267D017B817ADA799901F9DF9000DE
:20F560001557E0B4033990002C6B7481F0A374DAF0A374DBF0A37481F0A374DAF0A3749967
:20F58000F07B817ADA79A31202B0E2900015577401F0E4FFFEFDFCA31200844C01FDAA9071
:20F5A00000155FE0FBA3E0FAA3E0F9120080D36401600301FA1A90002D1C7481F0A374DA12
:20F5C000F0A374E9F0A3E4F0A37408F07B017A2679551202BC20EF701A900019BBE0FBA390
:20F5E000E0FAA3E0F912022362EF4E600301FA1A01F9CF90002D1C7481F0A374DAF0A374E8
:20F60000F2F0A3E4F0A37407F07B017A2679551202BC20EF7013900019BBE0FBA3E0FAA3D8
:20F62000E0F91202CE4301FA1A90002D1C7481F0A374DAF0A374FAF0A3E4F0A3740AF07B14
:20F64000017A2679551202BC20EF7013900019BBE0FBA3E0FAA3E0F91202891201FA1A904D
:20F66000002D1C7481F0A374DBF0A37405F0A3E4F0A37407F07B017A2679551202BC20EF20
:20F680007013900019BBE0FBA3E0FAA3E0F91202930601FA1A90002D1C7481F0A374DBF04D
:20F6A000A3740DF0A3E4F0A37409F07B017A2679551202BC20EF7013900019BBE0FBA3E0A1
:20F6C000FAA3E0F912028C9101FA1A90002D1C7481F0A374DBF0A37417F0A3E4F0A3740B17
:20F6E000F07B017A2679551202BC20EF7026900019BBE0FBA3E0FAA3E0F9120255C9EF4E14
:20F70000700301F9CF78557C267D017B817ADB792301F9DF90002D1C7481F0A374DBF0A3B7
:20F720007423F0A3E4F0A37408F07B017A2679551202BC20EF701A900019BBE0FBA3E0FAAD
:20F74000A3E0F912023D5DEF4E600301FA1A01F9CF90002D1C7481F0A374DBF0A3742CF02E
:20F76000A3E4F0A37409F07B017A2679551202BC20EF701A900019BBE0FBA3E0FAA3E0F977
:20F780001202750BEF4E600301FA1A01F9CF90002D1C7481F0A374DBF0A37436F0A3E4F003
:20F7A000A3740AF07B017A2679551202BC20EF701A900019BBE0FBA3E0FAA3E0F912026732
:20F7C000C5EF4E600301FA1A01F9CF90002D1C7481F0A374DBF0A37441F0A3E4F0A3740769
:20F7E000F07B017A2679551202BC20EF701A900019BBE0FBA3E0FAA3E0F912019C85EF4E1D
:20F80000600301FA1A01F9CF90002D1C7481F0A374DBF0A37449F0A3E4F0A37408F07B01B5
:20F820007A2679551202BC20EF701A900019BBE0FBA3E0FAA3E0F912025C98EF4E60030110
:20F84000FA1A01F9CF90002D1C7481F0A374DBF0A37452F0A3E4F0A37408F07B017A2679B7
:20F86000551202BC20EF701A900019BBE0FBA3E0FAA3E0F91201DE89EF4E600301FA1A0162
:20F88000F9CF90002D1C7481F0A374DBF0A3745BF0A3E4F0A3740CF07B017A267955120216
:20F8A000BC20EF7026900019BBE0FBA3E0FAA3E0F912028FDEEF4E700301F9CF78557C2646
:20F8C0007D017B817ADB792301F9DF90002D1C7481F0A374DBF0A37468F0A3E4F0A374083F
:20F8E000F07B017A2679551202BC20EF701A900019BBE0FBA3E0FAA3E0F912022830EF4EE4
:20F90000600301FA1A01F9CF90002D1C7481F0A374DBF0A37471F0A3E4F0A3740AF07B018A
:20F920007A2679551202BC20EF7026900019BBE0FBA3E0FAA3E0F9120205DDEF4E70030105
:20F94000F9CF78557C267D017B817ADB797C01F9DF90002D1C7481F0A374DBF0A37484F0A8
:20F96000A3E4F0A3740AF07B017A2679551202BC20EF7024900019BBE0FBA3E0FAA3E0F96A
:20F980001201F90CEF4E7002804578557C267D017B817ADB797C804790002D1C7481F0A380
:20F9A00074DBF0A3748FF0A3E4F0A3740AF07B017A2679551202BC20EF702A900019BBE043
:20F9C000FBA3E0FAA3E0F912025240EF4E7004FE7F012278557C267D017B817ADB797C12F7
:20F9E0000086EC803590002D1C7481F0A374DBF0A3749AF0A3E4F0A37409F07B017A267983
:20FA0000551202BC20EF701290002478F0A304F0900019C97410F001FDAAE490002651F014
:20FA200090002D1C7481F0A374DBF0A374A4F0A3E4F0A3740BF07B017A2679551202BC2018
:20FA4000EF70141202B63678557C267D017B817ADB79B0120086EC90002D1C7481F0A37473
:20FA6000DBF0A374BCF0A3E4F0A3740BF07B017A2679551202BC20EF701A90002E9CF0A32F
:20FA800004F078557C267D017B817ADB79C8120086EC8008E490002E9CF0A3F0E490002E84
:20FAA000FCF0A3F090002D1C7481F0A374DBF0A37471F0A3E4F0A3740AF07B017A2679553D
:20FAC0001202BC20EF7045900025A17481F0A374DBF0A374D4F0A37401F0A3742EF0A37446
:20FAE000FCF07B017A2679551200D58278557C267D017B817ADB797C120086EC90002EFD55
:20FB0000E024FFF090002EFCE034FFF090002651E0FD75F017A424FBF582E5F03412F58308
:20FB2000759300E0FBA3E0FAA3E04A4B700A900019C97410F001FDAAED75F017A424FEF91D
:20FB4000741235F0FA7B011200DDB090002D1FEEF0A3EFF090002651E075F017A424FEF987
:20FB6000741235F0FA90002D1C7401F0A3EAF0A3E9F07B017A2679551202BC20EF703090B0
:20FB800000155FE0FBA3E0FAA3E0F974031200812490002651E0FF9000155FE0FBA3E0FAAD
:20FBA000A3E02401F9E43AFAEF12008124800A90002651E004F001FB0C9000155FE0FBA3F7
:20FBC000E0FAA3E0F9120080D36403600301FCDD90001AAEF0A3F0900019C9E0B4043C9015
:20FBE0000012F1E0FBA3E0FAA3E0F9120081AEFF90001551E0FBA3E0FAA3E0F9E5F08FF0D0
:20FC00001200822890001554E0FBA3E0FAA3E0F9120081AEFF9000155C803A90001551E08A
:20FC2000FBA3E0FAA3E0F9120081AEFF900012F1E0FBA3E0FAA3E0F9E5F08FF01200822819
:20FC40009000155CE0FBA3E0FAA3E0F9120081AEFF90001554E0FBA3E0FAA3E0F9E5F08F5E
:20FC6000F0120082289000155FE0FBA3E0FAA3E02401F9E43AFA120080D375F017A424FB1F
:20FC8000F582E5F03412F583759300E0FBA3E0FAA3E0F912008568EF6007900019C9741033
:20FCA000F01202DAC9C004C005C006C0071202DC2FE4FCFD7B587A02F9F812008244D003A0
:20FCC000D002D001D000EB2FFFEA3EFEE93DFDE83CFC900012F71200844C01FDAA90001963
:20FCE000C9E030E07A9000155FE0FBA3E0FAA3E02402F9E43AFA120081AEC39478E5F09442
:20FD000005402A74FA75F088120081FC9000155FE0FBA3E0FAA3E02404F9E43AFA09E97010
:20FD2000010A740575F078120081FC80329000155FE0FBA3E0FAA3E02402F9E43AFAE4F532
:20FD4000F0120082289000155FE0FBA3E0FAA3E0F9120080D3B40207900019C97410F09087
:20FD600000155FE0FBA3E0FAA3E02402F9E43AFA120081AEFFAEF0D39478EE940590001A0F
:20FD8000AE40097405F0A37478F08005EEF0A3EFF09000155FE0FBA3E0FAA3E02404F9E4BB
:20FDA0003AFA120084641202D72F7E007F0122900028CBECF0A3EDF0900028C8EBF0A3EA14
:20FDC000F0A3E9F01201B9EC900028CBE0FCA3E0FDAE047802CEC313CE13D8F9FF900028E7
:20FDE000D2EEF0A3EFF0ED5403FFA3E4F0A3EFF0E4900028D0F0A3F0900028D2E0FEA3E0BB
:20FE0000FF900028D0E0FCA3E0FDC39FEC9E400301FF2AEDAE047802C333CE33CED8F9FFF8
:20FE2000900028C8E0FBA3E0FAA3E02FF9EA3EFA120083A578181200837F900028CDE0FBDF
:20FE4000A3E0FAA3E02403F9E43AFAEF12008124900028D0E0FEA3E07802C333CE33CED8C4
:20FE6000F9FF900028C8E0FBA3E0FAA3E02FF9EA3EFA120083A578101200837F900028CD8A
:20FE8000E0FBA3E0FAA3E02402F9E43AFAEF12008124900028D0E0FEA3E07802C333CE3350
:20FEA000CED8F9FF900028C8E0FBA3E0FAA3E02FF9EA3EFA120083A578081200837F9000A1
:20FEC00028CDE0FBA3E0FAA3E02401F9E43AFAEF12008124900028D0E0FEA3E07802C3331D
:20FEE000CE33CED8F9FF900028C8E0FBA3E0FAA3E02FF9EA3EFA120083A5900028CDE0FB24
:20FF0000A3E0FAA3E0F9EF12008124900028D1E004F07007900028D0E004F0900028CEE4A8
:20FF200075F0041200818201FDF8900028D4E07002A3E0700301FFDE900028D0E0FEA3E0B2
:20FF40007802C333CE33CED8F9FF900028C8E0FBA3E0FAA3E02FF9EA3EFA120083A5900023
:20FF600028D61200844CE4900028DAF0A3F0900028D4E0FEA3E0FFC3900028DBE09F900057
:20FF800028DAE09E5058900028D6A3A3A3E0FF900028CDE0FBA3E0FAA3E0F9900028DAE018
:20FFA000FCA3E0FDE92DF9EA3CFAEF12008124900028DBE004F07007900028DAE004F0901C
:20FFC0000028D6E0FCA3E0FDA3E0FEA3E0FF78081200837F900028D61200844C8090900020
:20FFE00028C8E0FBA3E0FAA3E0F90202A535AD07AC067B017A007F007E011202B51322FF08
:020000040001F9
:2000000090002875EBF0A3EAF0A3E9F0120083A59000287B1200844CE92404F9E43AFA125C
:200020000083A59000287F1200844C90002875E0FBA3E0FAA3E02408F9E43AFA120083A500
:20004000900028831200844C90002875E0FBA3E0FAA3E0240CF9E43AFA120083A590002848
:20006000871200844C9000287BE0F8A3E0F9A3E0FAA3E0FBC000C001C002C0039000288750
:20008000E0FCA3E0FDA3E0FEA3E0FF90002883E0F8A3E0F9A3E0FAA3E06FFFEA6EFEE96D58
:2000A000FDE86CFC9000287FE0F8A3E0F9A3E0FAA3E05FFFEA5EFEE95DFDE85CFC90002889
:2000C00087E0F8A3E0F9A3E0FAA3E06FFFEA6EFEE96DFDE86CFC90002878E0FBA3E0FAA3B3
:2000E000E0F9120083FAEF2BFFEE3AFEED39FDEC38FCEF2478FFEE34A4FEED346AFDEC3420
:20010000D7FCD003D002D001D000EB2FFFEA3EFEE93DFDE83CFC9000287B1200844C90009F
:20012000287BE0FCA3E0FDA3E0FEA3E0FF780712008392C004C005C006C0079000287BE0EE
:20014000FCA3E0FDA3E0FEA3E0FF78191200837FD003D002D001D000EF4BFFEE4AFEED4990
:20016000FDEC48FC9000287B1200844C9000287BE0FCA3E0FDA3E0FEA3E0FFA3E0F8A3E0AD
:20018000F9A3E0FAA3E0FBEF2BFFEE3AFEED39FDEC38FC9000287B1200844C90002887E0B5
:2001A000F8A3E0F9A3E0FAA3E0FBC000C001C002C00390002883E0FCA3E0FDA3E0FEA3E02F
:2001C000FF9000287FE0F8A3E0F9A3E0FAA3E06FFFEA6EFEE96DFDE86CFC9000287BE0F823
:2001E000A3E0F9A3E0FAA3E05FFFEA5EFEE95DFDE85CFC90002883E0F8A3E0F9A3E0FAA3AD
:20020000E06FFFEA6EFEE96DFDE86CFC90002878E0FBA3E0FAA3E02404F9E43AFA120083BE
:20022000FAEF2BFFEE3AFEED39FDEC38FCEF2456FFEE34B7FEED34C7FDEC34E8FCD003D077
:2002400002D001D000EB2FFFEA3EFEE93DFDE83CFC900028871200844C90002887E0FCA39A
:20026000E0FDA3E0FEA3E0FF780C12008392C004C005C006C00790002887E0FCA3E0FDA39F
:20028000E0FEA3E0FF78141200837FD003D002D001D000EF4BFFEE4AFEED49FDEC48FC90B6
:2002A0000028871200844C90002887E0FCA3E0FDA3E0FEA3E0FF9000287BE0F8A3E0F9A3E5
:2002C000E0FAA3E0FBEF2BFFEE3AFEED39FDEC38FC900028871200844C90002883E0F8A36D
:2002E000E0F9A3E0FAA3E0FBC000C001C002C0039000287FE0FCA3E0FDA3E0FEA3E0FF90FE
:2003000000287BE0F8A3E0F9A3E0FAA3E06FFFEA6EFEE96DFDE86CFC90002887E0F8A3E0E5
:20032000F9A3E0FAA3E05FFFEA5EFEE95DFDE85CFC9000287FE0F8A3E0F9A3E0FAA3E06FA3
:20034000FFEA6EFEE96DFDE86CFC90002878E0FBA3E0FAA3E02408F9E43AFA120083FAEFDF
:200360002BFFEE3AFEED39FDEC38FCEF24DBFFEE3470FEED3420FDEC3424FCD003D002D07A
:2003800001D000EB2FFFEA3EFEE93DFDE83CFC900028831200844C90002883E0FCA3E0FD56
:2003A000A3E0FEA3E0FF781112008392C004C005C006C00790002883E0FCA3E0FDA3E0FE5C
:2003C000A3E0FF780F1200837FD003D002D001D000EF4BFFEE4AFEED49FDEC48FC90002830
:2003E000831200844C90002883E0FCA3E0FDA3E0FEA3E0FFA3E0F8A3E0F9A3E0FAA3E0FB0C
:20040000EF2BFFEE3AFEED39FDEC38FC900028831200844C9000287FE0F8A3E0F9A3E0FA35
:20042000A3E0FBC000C001C002C0039000287BE0FCA3E0FDA3E0FEA3E0FF90002887E0F88F
:20044000A3E0F9A3E0FAA3E06FFFEA6EFEE96DFDE86CFC90002883E0F8A3E0F9A3E0FAA30A
:20046000E05FFFEA5EFEE95DFDE85CFC9000287BE0F8A3E0F9A3E0FAA3E06FFFEA6EFEE941
:200480006DFDE86CFC90002878E0FBA3E0FAA3E0240CF9E43AFA120083FAEF2BFFEE3AFE88
:2004A000ED39FDEC38FCEF24EEFFEE34CEFEED34BDFDEC34C1FCD003D002D001D000EB2FF3
:2004C000FFEA3EFEE93DFDE83CFC9000287F1200844C9000287FE0FCA3E0FDA3E0FEA3E004
:2004E000FF781612008392C004C005C006C0079000287FE0FCA3E0FDA3E0FEA3E0FF780A1A
:200500001200837FD003D002D001D000EF4BFFEE4AFEED49FDEC48FC9000287F1200844C96
:200520009000287FE0FCA3E0FDA3E0FEA3E0FFA3E0F8A3E0F9A3E0FAA3E0FBEF2BFFEE3AF2
:20054000FEED39FDEC38FC9000287F1200844C9000287BE0F8A3E0F9A3E0FAA3E0FBC000FF
:20056000C001C002C00390002887E0FCA3E0FDA3E0FEA3E0FF90002883E0F8A3E0F9A3E085
:20058000FAA3E06FFFEA6EFEE96DFDE86CFC9000287FE0F8A3E0F9A3E0FAA3E05FFFEA5E46
:2005A000FEE95DFDE85CFC90002887E0F8A3E0F9A3E0FAA3E06FFFEA6EFEE96DFDE86CFCC0
:2005C00090002878E0FBA3E0FAA3E02410F9E43AFA120083FAEF2BFFEE3AFEED39FDEC38B6
:2005E000FCEF24AFFFEE340FFEED347CFDEC34F5FCD003D002D001D000EB2FFFEA3EFEE9F6
:200600003DFDE83CFC9000287B1200844C9000287BE0FCA3E0FDA3E0FEA3E0FF7807120048
:200620008392C004C005C006C0079000287BE0FCA3E0FDA3E0FEA3E0FF78191200837FD088
:2006400003D002D001D000EF4BFFEE4AFEED49FDEC48FC9000287B1200844C9000287BE02A
:20066000FCA3E0FDA3E0FEA3E0FFA3E0F8A3E0F9A3E0FAA3E0FBEF2BFFEE3AFEED39FDECBB
:2006800038FC9000287B1200844C90002887E0F8A3E0F9A3E0FAA3E0FBC000C001C002C080
:2006A0000390002883E0FCA3E0FDA3E0FEA3E0FF9000287FE0F8A3E0F9A3E0FAA3E06FFFA4
:2006C000EA6EFEE96DFDE86CFC9000287BE0F8A3E0F9A3E0FAA3E05FFFEA5EFEE95DFDE8CB
:2006E0005CFC90002883E0F8A3E0F9A3E0FAA3E06FFFEA6EFEE96DFDE86CFC90002878E09C
:20070000FBA3E0FAA3E02414F9E43AFA120083FAEF2BFFEE3AFEED39FDEC38FCEF242AFF48
:20072000EE34C6FEED3487FDEC3447FCD003D002D001D000EB2FFFEA3EFEE93DFDE83CFC03
:20074000900028871200844C90002887E0FCA3E0FDA3E0FEA3E0FF780C12008392C004C0AB
:2007600005C006C00790002887E0FCA3E0FDA3E0FEA3E0FF78141200837FD003D002D00133
:20078000D000EF4BFFEE4AFEED49FDEC48FC900028871200844C90002887E0FCA3E0FDA358
:2007A000E0FEA3E0FF9000287BE0F8A3E0F9A3E0FAA3E0FBEF2BFFEE3AFEED39FDEC38FCD5
:2007C000900028871200844C90002883E0F8A3E0F9A3E0FAA3E0FBC000C001C002C00390D8
:2007E00000287FE0FCA3E0FDA3E0FEA3E0FF9000287BE0F8A3E0F9A3E0FAA3E06FFFEA6EA6
:20080000FEE96DFDE86CFC90002887E0F8A3E0F9A3E0FAA3E05FFFEA5EFEE95DFDE85CFC7D
:200820009000287FE0F8A3E0F9A3E0FAA3E06FFFEA6EFEE96DFDE86CFC90002878E0FBA318
:20084000E0FAA3E02418F9E43AFA120083FAEF2BFFEE3AFEED39FDEC38FCEF2413FFEE3496
:2008600046FEED3430FDEC34A8FCD003D002D001D000EB2FFFEA3EFEE93DFDE83CFC9000CA
:2008800028831200844C90002883E0FCA3E0FDA3E0FEA3E0FF781112008392C004C005C038
:2008A00006C00790002883E0FCA3E0FDA3E0FEA3E0FF780F1200837FD003D002D001D000F0
:2008C000EF4BFFEE4AFEED49FDEC48FC900028831200844C90002883E0FCA3E0FDA3E0FE11
:2008E000A3E0FFA3E0F8A3E0F9A3E0FAA3E0FBEF2BFFEE3AFEED39FDEC38FC9000288312B5
:2009000000844C9000287FE0F8A3E0F9A3E0FAA3E0FBC000C001C002C0039000287BE0FC6C
:20092000A3E0FDA3E0FEA3E0FF90002887E0F8A3E0F9A3E0FAA3E06FFFEA6EFEE96DFDE8A2
:200940006CFC90002883E0F8A3E0F9A3E0FAA3E05FFFEA5EFEE95DFDE85CFC9000287BE066
:20096000F8A3E0F9A3E0FAA3E06FFFEA6EFEE96DFDE86CFC90002878E0FBA3E0FAA3E0246D
:200980001CF9E43AFA120083FAEF2BFFEE3AFEED39FDEC38FCEF2401FFEE3495FEED3446EA
:2009A000FDEC34FDFCD003D002D001D000EB2FFFEA3EFEE93DFDE83CFC9000287F1200848C
:2009C0004C9000287FE0FCA3E0FDA3E0FEA3E0FF781612008392C004C005C006C0079000DA
:2009E000287FE0FCA3E0FDA3E0FEA3E0FF780A1200837FD003D002D001D000EF4BFFEE4AA4
:200A0000FEED49FDEC48FC9000287F1200844C9000287FE0FCA3E0FDA3E0FEA3E0FFA3E043
:200A2000F8A3E0F9A3E0FAA3E0FBEF2BFFEE3AFEED39FDEC38FC9000287F1200844C90001C
:200A4000287BE0F8A3E0F9A3E0FAA3E0FBC000C001C002C00390002887E0FCA3E0FDA3E080
:200A6000FEA3E0FF90002883E0F8A3E0F9A3E0FAA3E06FFFEA6EFEE96DFDE86CFC90002848
:200A80007FE0F8A3E0F9A3E0FAA3E05FFFEA5EFEE95DFDE85CFC90002887E0F8A3E0F9A326
:200AA000E0FAA3E06FFFEA6EFEE96DFDE86CFC90002878E0FBA3E0FAA3E02420F9E43AFA12
:200AC000120083FAEF2BFFEE3AFEED39FDEC38FCEF24D8FFEE3498FEED3480FDEC3469FC40
:200AE000D003D002D001D000EB2FFFEA3EFEE93DFDE83CFC9000287B1200844C9000287BE6
:200B0000E0FCA3E0FDA3E0FEA3E0FF780712008392C004C005C006C0079000287BE0FCA308
:200B2000E0FDA3E0FEA3E0FF78191200837FD003D002D001D000EF4BFFEE4AFEED49FDEC5C
:200B400048FC9000287B1200844C9000287BE0FCA3E0FDA3E0FEA3E0FFA3E0F8A3E0F9A310
:200B6000E0FAA3E0FBEF2BFFEE3AFEED39FDEC38FC9000287B1200844C90002887E0F8A3CC
:200B8000E0F9A3E0FAA3E0FBC000C001C002C00390002883E0FCA3E0FDA3E0FEA3E0FF9051
:200BA00000287FE0F8A3E0F9A3E0FAA3E06FFFEA6EFEE96DFDE86CFC9000287BE0F8A3E045
:200BC000F9A3E0FAA3E05FFFEA5EFEE95DFDE85CFC90002883E0F8A3E0F9A3E0FAA3E06FF7
:200BE000FFEA6EFEE96DFDE86CFC90002878E0FBA3E0FAA3E02424F9E43AFA120083FAEF1B
:200C00002BFFEE3AFEED39FDEC38FCEF24AFFFEE34F7FEED3444FDEC348BFCD003D002D0EB
:200C200001D000EB2FFFEA3EFEE93DFDE83CFC900028871200844C90002887E0FCA3E0FDA5
:200C4000A3E0FEA3E0FF780C12008392C004C005C006C00790002887E0FCA3E0FDA3E0FEB4
:200C6000A3E0FF78141200837FD003D002D001D000EF4BFFEE4AFEED49FDEC48FC90002882
:200C8000871200844C90002887E0FCA3E0FDA3E0FEA3E0FF9000287BE0F8A3E0F9A3E0FA49
:200CA000A3E0FBEF2BFFEE3AFEED39FDEC38FC900028871200844C90002883E0F8A3E0F984
:200CC000A3E0FAA3E0FBC000C001C002C0039000287FE0FCA3E0FDA3E0FEA3E0FF900028C5
:200CE0007BE0F8A3E0F9A3E0FAA3E06FFFEA6EFEE96DFDE86CFC90002887E0F8A3E0F9A388
:200D0000E0FAA3E05FFFEA5EFEE95DFDE85CFC9000287FE0F8A3E0F9A3E0FAA3E06FFFEA6C
:200D20006EFEE96DFDE86CFC90002878E0FBA3E0FAA3E02428F9E43AFA120083FAEF2BFF94
:200D4000EE3AFEED39FDEC38FCEF24B1FFEE345BFEED34FFFDEC34FFFCD003D002D001D06E
:200D600000EB2FFFEA3EFEE93DFDE83CFC900028831200844C90002883E0FCA3E0FDA3E0BA
:200D8000FEA3E0FF781112008392C004C005C006C00790002883E0FCA3E0FDA3E0FEA3E072
:200DA000FF780F1200837FD003D002D001D000EF4BFFEE4AFEED49FDEC48FC900028831234
:200DC00000844C90002883E0FCA3E0FDA3E0FEA3E0FFA3E0F8A3E0F9A3E0FAA3E0FBEF2B9D
:200DE000FFEE3AFEED39FDEC38FC900028831200844C9000287FE0F8A3E0F9A3E0FAA3E0E3
:200E0000FBC000C001C002C0039000287BE0FCA3E0FDA3E0FEA3E0FF90002887E0F8A3E0A5
:200E2000F9A3E0FAA3E06FFFEA6EFEE96DFDE86CFC90002883E0F8A3E0F9A3E0FAA3E05F64
:200E4000FFEA5EFEE95DFDE85CFC9000287BE0F8A3E0F9A3E0FAA3E06FFFEA6EFEE96DFD2C
:200E6000E86CFC90002878E0FBA3E0FAA3E0242CF9E43AFA120083FAEF2BFFEE3AFEED39C2
:200E8000FDEC38FCEF24BEFFEE34D7FEED345CFDEC3489FCD003D002D001D000EB2FFFEA06
:200EA0003EFEE93DFDE83CFC9000287F1200844C9000287FE0FCA3E0FDA3E0FEA3E0FF788C
:200EC0001612008392C004C005C006C0079000287FE0FCA3E0FDA3E0FEA3E0FF780A120095
:200EE000837FD003D002D001D000EF4BFFEE4AFEED49FDEC48FC9000287F1200844C90002F
:200F0000287FE0FCA3E0FDA3E0FEA3E0FFA3E0F8A3E0F9A3E0FAA3E0FBEF2BFFEE3AFEEDAD
:200F200039FDEC38FC9000287F1200844C9000287BE0F8A3E0F9A3E0FAA3E0FBC000C0013F
:200F4000C002C00390002887E0FCA3E0FDA3E0FEA3E0FF90002883E0F8A3E0F9A3E0FAA3BF
:200F6000E06FFFEA6EFEE96DFDE86CFC9000287FE0F8A3E0F9A3E0FAA3E05FFFEA5EFEE912
:200F80005DFDE85CFC90002887E0F8A3E0F9A3E0FAA3E06FFFEA6EFEE96DFDE86CFC90002D
:200FA0002878E0FBA3E0FAA3E02430F9E43AFA120083FAEF2BFFEE3AFEED39FDEC38FCEF51
:200FC0002422FFEE3411FEED3490FDEC346BFCD003D002D001D000EB2FFFEA3EFEE93DFDBE
:200FE000E83CFC9000287B1200844C9000287BE0FCA3E0FDA3E0FEA3E0FF78071200839284
:20100000C004C005C006C0079000287BE0FCA3E0FDA3E0FEA3E0FF78191200837FD003D0E0
:2010200002D001D000EF4BFFEE4AFEED49FDEC48FC9000287B1200844C9000287BE0FCA374
:20104000E0FDA3E0FEA3E0FFA3E0F8A3E0F9A3E0FAA3E0FBEF2BFFEE3AFEED39FDEC38FC3C
:201060009000287B1200844C90002887E0F8A3E0F9A3E0FAA3E0FBC000C001C002C0039037
:20108000002883E0FCA3E0FDA3E0FEA3E0FF9000287FE0F8A3E0F9A3E0FAA3E06FFFEA6EF5
:2010A000FEE96DFDE86CFC9000287BE0F8A3E0F9A3E0FAA3E05FFFEA5EFEE95DFDE85CFCE1
:2010C00090002883E0F8A3E0F9A3E0FAA3E06FFFEA6EFEE96DFDE86CFC90002878E0FBA36C
:2010E000E0FAA3E02434F9E43AFA120083FAEF2BFFEE3AFEED39FDEC38FCEF2493FFEE3452
:2011000071FEED3498FDEC34FDFCD003D002D001D000EB2FFFEA3EFEE93DFDE83CFC900039
:2011200028871200844C90002887E0FCA3E0FDA3E0FEA3E0FF780C12008392C004C005C08C
:2011400006C00790002887E0FCA3E0FDA3E0FEA3E0FF78141200837FD003D002D001D0003E
:20116000EF4BFFEE4AFEED49FDEC48FC900028871200844C90002887E0FCA3E0FDA3E0FE60
:20118000A3E0FF9000287BE0F8A3E0F9A3E0FAA3E0FBEF2BFFEE3AFEED39FDEC38FC900039
:2011A00028871200844C90002883E0F8A3E0F9A3E0FAA3E0FBC000C001C002C00390002856
:2011C0007FE0FCA3E0FDA3E0FEA3E0FF9000287BE0F8A3E0F9A3E0FAA3E06FFFEA6EFEE9FD
:2011E0006DFDE86CFC90002887E0F8A3E0F9A3E0FAA3E05FFFEA5EFEE95DFDE85CFC9000EB
:20120000287FE0F8A3E0F9A3E0FAA3E06FFFEA6EFEE96DFDE86CFC90002878E0FBA3E0FAE4
:20122000A3E02438F9E43AFA120083FAEF2BFFEE3AFEED39FDEC38FCEF248EFFEE3443FEAA
:20124000ED3479FDEC34A6FCD003D002D001D000EB2FFFEA3EFEE93DFDE83CFC9000288332
:201260001200844C90002883E0FCA3E0FDA3E0FEA3E0FF781112008392C004C005C006C033
:201280000790002883E0FCA3E0FDA3E0FEA3E0FF780F1200837FD003D002D001D000EF4B92
:2012A000FFEE4AFEED49FDEC48FC900028831200844C90002883E0FCA3E0FDA3E0FEA3E0DE
:2012C000FFA3E0F8A3E0F9A3E0FAA3E0FBEF2BFFEE3AFEED39FDEC38FC90002883120084CA
:2012E0004C9000287FE0F8A3E0F9A3E0FAA3E0FBC000C001C002C0039000287BE0FCA3E084
:20130000FDA3E0FEA3E0FF90002887E0F8A3E0F9A3E0FAA3E06FFFEA6EFEE96DFDE86CFCD3
:2013200090002883E0F8A3E0F9A3E0FAA3E05FFFEA5EFEE95DFDE85CFC9000287BE0F8A349
:20134000E0F9A3E0FAA3E06FFFEA6EFEE96DFDE86CFC90002878E0FBA3E0FAA3E0243CF9E9
:20136000E43AFA120083FAEF2BFFEE3AFEED39FDEC38FCEF2421FFEE3408FEED34B4FDEC2B
:201380003449FCD003D002D001D000EB2FFFEA3EFEE93DFDE83CFC9000287F1200844C9063
:2013A00000287FE0FCA3E0FDA3E0FEA3E0FF781612008392C004C005C006C0079000287F25
:2013C000E0FCA3E0FDA3E0FEA3E0FF780A1200837FD003D002D001D000EF4BFFEE4AFEED76
:2013E00049FDEC48FC9000287F1200844C9000287FE0FCA3E0FDA3E0FEA3E0FFA3E0F8A3AA
:20140000E0F9A3E0FAA3E0FBEF2BFFEE3AFEED39FDEC38FC9000287F1200844C9000287B2A
:20142000E0F8A3E0F9A3E0FAA3E0FBC000C001C002C00390002883E0FCA3E0FDA3E0FEA39C
:20144000E0FF9000287FE0F8A3E0F9A3E0FAA3E06FFFEA6EFEE96DFDE86CFC90002887E09C
:20146000F8A3E0F9A3E0FAA3E05FFFEA5EFEE95DFDE85CFC90002883E0F8A3E0F9A3E0FAC5
:20148000A3E06FFFEA6EFEE96DFDE86CFC90002878E0FBA3E0FAA3E02404F9E43AFA12000C
:2014A00083FAEF2BFFEE3AFEED39FDEC38FCEF2462FFEE3425FEED341EFDEC34F6FCD00353
:2014C000D002D001D000EB2FFFEA3EFEE93DFDE83CFC9000287B1200844C9000287BE0FCF3
:2014E000A3E0FDA3E0FEA3E0FF780512008392C004C005C006C0079000287BE0FCA3E0FD20
:20150000A3E0FEA3E0FF781B1200837FD003D002D001D000EF4BFFEE4AFEED49FDEC48FC09
:201520009000287B1200844C9000287BE0FCA3E0FDA3E0FEA3E0FFA3E0F8A3E0F9A3E0FA90
:20154000A3E0FBEF2BFFEE3AFEED39FDEC38FC9000287B1200844C90002887E0F8A3E0F9E3
:20156000A3E0FAA3E0FBC000C001C002C0039000287FE0FCA3E0FDA3E0FEA3E0FF9000281C
:201580007BE0F8A3E0F9A3E0FAA3E06FFFEA6EFEE96DFDE86CFC90002883E0F8A3E0F9A3E3
:2015A000E0FAA3E05FFFEA5EFEE95DFDE85CFC9000287FE0F8A3E0F9A3E0FAA3E06FFFEAC4
:2015C0006EFEE96DFDE86CFC90002878E0FBA3E0FAA3E02418F9E43AFA120083FAEF2BFFFC
:2015E000EE3AFEED39FDEC38FCEF2440FFEE34B3FEED3440FDEC34C0FCD003D002D001D0DD
:2016000000EB2FFFEA3EFEE93DFDE83CFC900028871200844C90002887E0FCA3E0FDA3E009
:20162000FEA3E0FF780912008392C004C005C006C00790002887E0FCA3E0FDA3E0FEA3E0CD
:20164000FF78171200837FD003D002D001D000EF4BFFEE4AFEED49FDEC48FC90002887127F
:2016600000844C90002887E0FCA3E0FDA3E0FEA3E0FF9000287BE0F8A3E0F9A3E0FAA3E075
:20168000FBEF2BFFEE3AFEED39FDEC38FC900028871200844C90002883E0F8A3E0F9A3E09A
:2016A000FAA3E0FBC000C001C002C0039000287BE0FCA3E0FDA3E0FEA3E0FF90002887E0FB
:2016C000F8A3E0F9A3E0FAA3E06FFFEA6EFEE96DFDE86CFC9000287FE0F8A3E0F9A3E0FA27
:2016E000A3E05FFFEA5EFEE95DFDE85CFC9000287BE0F8A3E0F9A3E0FAA3E06FFFEA6EFEF5
:20170000E96DFDE86CFC90002878E0FBA3E0FAA3E0242CF9E43AFA120083FAEF2BFFEE3AEA
:20172000FEED39FDEC38FCEF2451FFEE345AFEED345EFDEC3426FCD003D002D001D000EB9C
:201740002FFFEA3EFEE93DFDE83CFC900028831200844C90002883E0FCA3E0FDA3E0FEA31A
:20176000E0FF780E12008392C004C005C006C00790002883E0FCA3E0FDA3E0FEA3E0FF78B5
:20178000121200837FD003D002D001D000EF4BFFEE4AFEED49FDEC48FC900028831200843A
:2017A0004C90002883E0FCA3E0FDA3E0FEA3E0FFA3E0F8A3E0F9A3E0FAA3E0FBEF2BFFEE4A
:2017C0003AFEED39FDEC38FC900028831200844C9000287FE0F8A3E0F9A3E0FAA3E0FBC02B
:2017E00000C001C002C00390002887E0FCA3E0FDA3E0FEA3E0FF90002883E0F8A3E0F9A3D3
:20180000E0FAA3E06FFFEA6EFEE96DFDE86CFC9000287BE0F8A3E0F9A3E0FAA3E05FFFEA35
:201820005EFEE95DFDE85CFC90002887E0F8A3E0F9A3E0FAA3E06FFFEA6EFEE96DFDE86CCB
:20184000FC90002878E0FBA3E0FAA3E0F9120083FAEF2BFFEE3AFEED39FDEC38FCEF24AABA
:20186000FFEE34C7FEED34B6FDEC34E9FCD003D002D001D000EB2FFFEA3EFEE93DFDE83CDD
:20188000FC9000287F1200844C9000287FE0FCA3E0FDA3E0FEA3E0FF781412008392C00426
:2018A000C005C006C0079000287FE0FCA3E0FDA3E0FEA3E0FF780C1200837FD003D002D033
:2018C00001D000EF4BFFEE4AFEED49FDEC48FC9000287F1200844C9000287FE0FCA3E0FDB9
:2018E000A3E0FEA3E0FFA3E0F8A3E0F9A3E0FAA3E0FBEF2BFFEE3AFEED39FDEC38FC9000E1
:20190000287F1200844C9000287BE0F8A3E0F9A3E0FAA3E0FBC000C001C002C003900028FE
:2019200083E0FCA3E0FDA3E0FEA3E0FF9000287FE0F8A3E0F9A3E0FAA3E06FFFEA6EFEE98D
:201940006DFDE86CFC90002887E0F8A3E0F9A3E0FAA3E05FFFEA5EFEE95DFDE85CFC900083
:201960002883E0F8A3E0F9A3E0FAA3E06FFFEA6EFEE96DFDE86CFC90002878E0FBA3E0FA79
:20198000A3E02414F9E43AFA120083FAEF2BFFEE3AFEED39FDEC38FCEF245DFFEE3410FECB
:2019A000ED342FFDEC34D6FCD003D002D001D000EB2FFFEA3EFEE93DFDE83CFC9000287BED
:2019C0001200844C9000287BE0FCA3E0FDA3E0FEA3E0FF780512008392C004C005C006C0E0
:2019E000079000287BE0FCA3E0FDA3E0FEA3E0FF781B1200837FD003D002D001D000EF4B27
:201A0000FFEE4AFEED49FDEC48FC9000287B1200844C9000287BE0FCA3E0FDA3E0FEA3E086
:201A2000FFA3E0F8A3E0F9A3E0FAA3E0FBEF2BFFEE3AFEED39FDEC38FC9000287B1200846A
:201A40004C90002887E0F8A3E0F9A3E0FAA3E0FBC000C001C002C0039000287FE0FCA3E010
:201A6000FDA3E0FEA3E0FF9000287BE0F8A3E0F9A3E0FAA3E06FFFEA6EFEE96DFDE86CFC78
:201A800090002883E0F8A3E0F9A3E0FAA3E05FFFEA5EFEE95DFDE85CFC9000287FE0F8A3DE
:201AA000E0F9A3E0FAA3E06FFFEA6EFEE96DFDE86CFC90002878E0FBA3E0FAA3E02428F996
:201AC000E43AFA120083FAEF2BFFEE3AFEED39FDEC38FCEF2453FFEE3414FEED3444FDECF6
:201AE0003402FCD003D002D001D000EB2FFFEA3EFEE93DFDE83CFC900028871200844C903B
:201B0000002887E0FCA3E0FDA3E0FEA3E0FF780912008392C004C005C006C00790002887BA
:201B2000E0FCA3E0FDA3E0FEA3E0FF78171200837FD003D002D001D000EF4BFFEE4AFEED01
:201B400049FDEC48FC900028871200844C90002887E0FCA3E0FDA3E0FEA3E0FF9000287B1D
:201B6000E0F8A3E0F9A3E0FAA3E0FBEF2BFFEE3AFEED39FDEC38FC900028871200844C90E3
:201B8000002883E0F8A3E0F9A3E0FAA3E0FBC000C001C002C0039000287BE0FCA3E0FDA313
:201BA000E0FEA3E0FF90002887E0F8A3E0F9A3E0FAA3E06FFFEA6EFEE96DFDE86CFC90003B
:201BC000287FE0F8A3E0F9A3E0FAA3E05FFFEA5EFEE95DFDE85CFC9000287BE0F8A3E0F95C
:201BE000A3E0FAA3E06FFFEA6EFEE96DFDE86CFC90002878E0FBA3E0FAA3E0243CF9E43AFC
:201C0000FA120083FAEF2BFFEE3AFEED39FDEC38FCEF2481FFEE34E6FEED34A1FDEC34D869
:201C2000FCD003D002D001D000EB2FFFEA3EFEE93DFDE83CFC900028831200844C9000280B
:201C400083E0FCA3E0FDA3E0FEA3E0FF780E12008392C004C005C006C00790002883E0FCC8
:201C6000A3E0FDA3E0FEA3E0FF78121200837FD003D002D001D000EF4BFFEE4AFEED49FD5B
:201C8000EC48FC900028831200844C90002883E0FCA3E0FDA3E0FEA3E0FFA3E0F8A3E0F966
:201CA000A3E0FAA3E0FBEF2BFFEE3AFEED39FDEC38FC900028831200844C9000287FE0F87B
:201CC000A3E0F9A3E0FAA3E0FBC000C001C002C00390002887E0FCA3E0FDA3E0FEA3E0FFE9
:201CE00090002883E0F8A3E0F9A3E0FAA3E06FFFEA6EFEE96DFDE86CFC9000287BE0F8A340
:201D0000E0F9A3E0FAA3E05FFFEA5EFEE95DFDE85CFC90002887E0F8A3E0F9A3E0FAA3E030
:201D20006FFFEA6EFEE96DFDE86CFC90002878E0FBA3E0FAA3E02410F9E43AFA120083FA5D
:201D4000EF2BFFEE3AFEED39FDEC38FCEF24C8FFEE34FBFEED34D3FDEC34E7FCD003D00273
:201D6000D001D000EB2FFFEA3EFEE93DFDE83CFC9000287F1200844C9000287FE0FCA3E091
:201D8000FDA3E0FEA3E0FF781412008392C004C005C006C0079000287FE0FCA3E0FDA3E064
:201DA000FEA3E0FF780C1200837FD003D002D001D000EF4BFFEE4AFEED49FDEC48FC900063
:201DC000287F1200844C9000287FE0FCA3E0FDA3E0FEA3E0FFA3E0F8A3E0F9A3E0FAA3E0ED
:201DE000FBEF2BFFEE3AFEED39FDEC38FC9000287F1200844C9000287BE0F8A3E0F9A3E043
:201E0000FAA3E0FBC000C001C002C00390002883E0FCA3E0FDA3E0FEA3E0FF9000287FE093
:201E2000F8A3E0F9A3E0FAA3E06FFFEA6EFEE96DFDE86CFC90002887E0F8A3E0F9A3E0FAB7
:201E4000A3E05FFFEA5EFEE95DFDE85CFC90002883E0F8A3E0F9A3E0FAA3E06FFFEA6EFE85
:201E6000E96DFDE86CFC90002878E0FBA3E0FAA3E02424F9E43AFA120083FAEF2BFFEE3A8B
:201E8000FEED39FDEC38FCEF24E6FFEE34CDFEED34E1FDEC3421FCD003D002D001D000EBAF
:201EA0002FFFEA3EFEE93DFDE83CFC9000287B1200844C9000287BE0FCA3E0FDA3E0FEA3C3
:201EC000E0FF780512008392C004C005C006C0079000287BE0FCA3E0FDA3E0FEA3E0FF785F
:201EE0001B1200837FD003D002D001D000EF4BFFEE4AFEED49FDEC48FC9000287B120084D2
:201F00004C9000287BE0FCA3E0FDA3E0FEA3E0FFA3E0F8A3E0F9A3E0FAA3E0FBEF2BFFEEEA
:201F20003AFEED39FDEC38FC9000287B1200844C90002887E0F8A3E0F9A3E0FAA3E0FBC0C3
:201F400000C001C002C0039000287FE0FCA3E0FDA3E0FEA3E0FF9000287BE0F8A3E0F9A37B
:201F6000E0FAA3E06FFFEA6EFEE96DFDE86CFC90002883E0F8A3E0F9A3E0FAA3E05FFFEAC6
:201F80005EFEE95DFDE85CFC9000287FE0F8A3E0F9A3E0FAA3E06FFFEA6EFEE96DFDE86C6C
:201FA000FC90002878E0FBA3E0FAA3E02438F9E43AFA120083FAEF2BFFEE3AFEED39FDECD0
:201FC00038FCEF24D6FFEE3407FEED3437FDEC34C3FCD003D002D001D000EB2FFFEA3EFE05
:201FE000E93DFDE83CFC900028871200844C90002887E0FCA3E0FDA3E0FEA3E0FF7809124C
:20200000008392C004C005C006C00790002887E0FCA3E0FDA3E0FEA3E0FF78171200837F54
:20202000D003D002D001D000EF4BFFEE4AFEED49FDEC48FC900028871200844C9000288728
:20204000E0FCA3E0FDA3E0FEA3E0FF9000287BE0F8A3E0F9A3E0FAA3E0FBEF2BFFEE3AFE60
:20206000ED39FDEC38FC900028871200844C90002883E0F8A3E0F9A3E0FAA3E0FBC000C0F2
:2020800001C002C0039000287BE0FCA3E0FDA3E0FEA3E0FF90002887E0F8A3E0F9A3E0FA18
:2020A000A3E06FFFEA6EFEE96DFDE86CFC9000287FE0F8A3E0F9A3E0FAA3E05FFFEA5EFE07
:2020C000E95DFDE85CFC9000287BE0F8A3E0F9A3E0FAA3E06FFFEA6EFEE96DFDE86CFC90FF
:2020E000002878E0FBA3E0FAA3E0240CF9E43AFA120083FAEF2BFFEE3AFEED39FDEC38FC13
:20210000EF2487FFEE340DFEED34D5FDEC34F4FCD003D002D001D000EB2FFFEA3EFEE93D4B
:20212000FDE83CFC900028831200844C90002883E0FCA3E0FDA3E0FEA3E0FF780E120083B0
:2021400092C004C005C006C00790002883E0FCA3E0FDA3E0FEA3E0FF78121200837FD003CC
:20216000D002D001D000EF4BFFEE4AFEED49FDEC48FC900028831200844C90002883E0FCE6
:20218000A3E0FDA3E0FEA3E0FFA3E0F8A3E0F9A3E0FAA3E0FBEF2BFFEE3AFEED39FDEC3844
:2021A000FC900028831200844C9000287FE0F8A3E0F9A3E0FAA3E0FBC000C001C002C0037A
:2021C00090002887E0FCA3E0FDA3E0FEA3E0FF90002883E0F8A3E0F9A3E0FAA3E06FFFEA7A
:2021E0006EFEE96DFDE86CFC9000287BE0F8A3E0F9A3E0FAA3E05FFFEA5EFEE95DFDE85C1E
:20220000FC90002887E0F8A3E0F9A3E0FAA3E06FFFEA6EFEE96DFDE86CFC90002878E0FBBD
:20222000A3E0FAA3E02420F9E43AFA120083FAEF2BFFEE3AFEED39FDEC38FCEF24EDFFEE4B
:202240003414FEED345AFDEC3445FCD003D002D001D000EB2FFFEA3EFEE93DFDE83CFC9007
:2022600000287F1200844C9000287FE0FCA3E0FDA3E0FEA3E0FF781412008392C004C00503
:20228000C006C0079000287FE0FCA3E0FDA3E0FEA3E0FF780C1200837FD003D002D001D03D
:2022A00000EF4BFFEE4AFEED49FDEC48FC9000287F1200844C9000287FE0FCA3E0FDA3E01D
:2022C000FEA3E0FFA3E0F8A3E0F9A3E0FAA3E0FBEF2BFFEE3AFEED39FDEC38FC9000287FD3
:2022E0001200844C9000287BE0F8A3E0F9A3E0FAA3E0FBC000C001C002C00390002883E059
:20230000FCA3E0FDA3E0FEA3E0FF9000287FE0F8A3E0F9A3E0FAA3E06FFFEA6EFEE96DFD9C
:20232000E86CFC90002887E0F8A3E0F9A3E0FAA3E05FFFEA5EFEE95DFDE85CFC9000288358
:20234000E0F8A3E0F9A3E0FAA3E06FFFEA6EFEE96DFDE86CFC90002878E0FBA3E0FAA3E0B7
:202360002434F9E43AFA120083FAEF2BFFEE3AFEED39FDEC38FCEF2405FFEE34E9FEED34A2
:20238000E3FDEC34A9FCD003D002D001D000EB2FFFEA3EFEE93DFDE83CFC9000287B12008B
:2023A000844C9000287BE0FCA3E0FDA3E0FEA3E0FF780512008392C004C005C006C0079071
:2023C00000287BE0FCA3E0FDA3E0FEA3E0FF781B1200837FD003D002D001D000EF4BFFEEE7
:2023E0004AFEED49FDEC48FC9000287B1200844C9000287BE0FCA3E0FDA3E0FEA3E0FFA3E8
:20240000E0F8A3E0F9A3E0FAA3E0FBEF2BFFEE3AFEED39FDEC38FC9000287B1200844C9046
:20242000002887E0F8A3E0F9A3E0FAA3E0FBC000C001C002C0039000287FE0FCA3E0FDA362
:20244000E0FEA3E0FF9000287BE0F8A3E0F9A3E0FAA3E06FFFEA6EFEE96DFDE86CFC90009E
:202460002883E0F8A3E0F9A3E0FAA3E05FFFEA5EFEE95DFDE85CFC9000287FE0F8A3E0F9AB
:20248000A3E0FAA3E06FFFEA6EFEE96DFDE86CFC90002878E0FBA3E0FAA3E02408F9E43A87
:2024A000FA120083FAEF2BFFEE3AFEED39FDEC38FCEF24F8FFEE34A3FEED34EFFDEC34FC1B
:2024C000FCD003D002D001D000EB2FFFEA3EFEE93DFDE83CFC900028871200844C9000285F
:2024E00087E0FCA3E0FDA3E0FEA3E0FF780912008392C004C005C006C00790002887E0FC1D
:20250000A3E0FDA3E0FEA3E0FF78171200837FD003D002D001D000EF4BFFEE4AFEED49FDAD
:20252000EC48FC900028871200844C90002887E0FCA3E0FDA3E0FEA3E0FF9000287BE0F8A1
:20254000A3E0F9A3E0FAA3E0FBEF2BFFEE3AFEED39FDEC38FC900028871200844C900028A9
:2025600083E0F8A3E0F9A3E0FAA3E0FBC000C001C002C0039000287BE0FCA3E0FDA3E0FE73
:20258000A3E0FF90002887E0F8A3E0F9A3E0FAA3E06FFFEA6EFEE96DFDE86CFC9000287F88
:2025A000E0F8A3E0F9A3E0FAA3E05FFFEA5EFEE95DFDE85CFC9000287BE0F8A3E0F9A3E096
:2025C000FAA3E06FFFEA6EFEE96DFDE86CFC90002878E0FBA3E0FAA3E0241CF9E43AFA12A9
:2025E0000083FAEF2BFFEE3AFEED39FDEC38FCEF24D9FFEE3402FEED346FFDEC3467FCD0EF
:2026000003D002D001D000EB2FFFEA3EFEE93DFDE83CFC900028831200844C90002883E08A
:20262000FCA3E0FDA3E0FEA3E0FF780E12008392C004C005C006C00790002883E0FCA3E0BE
:20264000FDA3E0FEA3E0FF78121200837FD003D002D001D000EF4BFFEE4AFEED49FDEC48C0
:20266000FC900028831200844C90002883E0FCA3E0FDA3E0FEA3E0FFA3E0F8A3E0F9A3E02D
:20268000FAA3E0FBEF2BFFEE3AFEED39FDEC38FC900028831200844C9000287FE0F8A3E091
:2026A000F9A3E0FAA3E0FBC000C001C002C00390002887E0FCA3E0FDA3E0FEA3E0FF9000F2
:2026C0002883E0F8A3E0F9A3E0FAA3E06FFFEA6EFEE96DFDE86CFC9000287BE0F8A3E0F90D
:2026E000A3E0FAA3E05FFFEA5EFEE95DFDE85CFC90002887E0F8A3E0F9A3E0FAA3E06FFFB2
:20270000EA6EFEE96DFDE86CFC90002878E0FBA3E0FAA3E02430F9E43AFA120083FAEF2BA7
:20272000FFEE3AFEED39FDEC38FCEF248AFFEE344CFEED342AFDEC348DFCD003D002D001C2
:20274000D000EB2FFFEA3EFEE93DFDE83CFC9000287F1200844C9000287FE0FCA3E0FDA3D8
:20276000E0FEA3E0FF781412008392C004C005C006C0079000287FE0FCA3E0FDA3E0FEA379
:20278000E0FF780C1200837FD003D002D001D000EF4BFFEE4AFEED49FDEC48FC9000287F73
:2027A0001200844C9000287FE0FCA3E0FDA3E0FEA3E0FFA3E0F8A3E0F9A3E0FAA3E0FBEFC0
:2027C0002BFFEE3AFEED39FDEC38FC9000287F1200844C9000287BE0F8A3E0F9A3E0FAA3A6
:2027E000E0FBC000C001C002C00390002878E0FBA3E0FAA3E02414F9E43AFA120083FAC055
:2028000000C001C00290002883E0FCA3E0FDA3E0FEA3E0FF9000287FE0F8A3E0F9A3E0FA93
:20282000A3E06FFFEA6EFEE96DFDE86CFC90002887E0F8A3E0F9A3E0FAA3E06FFFEA6EFE57
:20284000E96DFDE86CFCD002D001D000EF2BFFEE3AFEED39FDEC38FCEF2442FFEE3439FE33
:20286000ED34FAFDEC34FFFCD003D002D001D000EB2FFFEA3EFEE93DFDE83CFC9000287B2A
:202880001200844C9000287BE0FCA3E0FDA3E0FEA3E0FF780412008392C004C005C006C012
:2028A000079000287BE0FCA3E0FDA3E0FEA3E0FF781C1200837FD003D002D001D000EF4B57
:2028C000FFEE4AFEED49FDEC48FC9000287B1200844C9000287BE0FCA3E0FDA3E0FEA3E0B8
:2028E000FFA3E0F8A3E0F9A3E0FAA3E0FBEF2BFFEE3AFEED39FDEC38FC9000287B1200849C
:202900004C90002887E0F8A3E0F9A3E0FAA3E0FBC000C001C002C00390002878E0FBA3E049
:20292000FAA3E02420F9E43AFA120083FAC000C001C0029000287FE0FCA3E0FDA3E0FEA33C
:20294000E0FF9000287BE0F8A3E0F9A3E0FAA3E06FFFEA6EFEE96DFDE86CFC90002883E08F
:20296000F8A3E0F9A3E0FAA3E06FFFEA6EFEE96DFDE86CFCD002D001D000EF2BFFEE3AFECA
:20298000ED39FDEC38FCEF2481FFEE34F6FEED3471FDEC3487FCD003D002D001D000EB2FB9
:2029A000FFEA3EFEE93DFDE83CFCA31200844C90002887E0FCA3E0FDA3E0FEA3E0FF780B09
:2029C00012008392C004C005C006C00790002887E0FCA3E0FDA3E0FEA3E0FF7815120083FA
:2029E0007FD003D002D001D000EF4BFFEE4AFEED49FDEC48FC900028871200844C90002867
:202A000087E0FCA3E0FDA3E0FEA3E0FF9000287BE0F8A3E0F9A3E0FAA3E0FBEF2BFFEE3A0D
:202A2000FEED39FDEC38FC900028871200844C90002883E0F8A3E0F9A3E0FAA3E0FBC000EA
:202A4000C001C002C00390002878E0FBA3E0FAA3E0242CF9E43AFA120083FAC000C001C0F4
:202A6000029000287BE0FCA3E0FDA3E0FEA3E0FF90002887E0F8A3E0F9A3E0FAA3E06FFFC1
:202A8000EA6EFEE96DFDE86CFC9000287FE0F8A3E0F9A3E0FAA3E06FFFEA6EFEE96DFDE8B3
:202AA0006CFCD002D001D000EF2BFFEE3AFEED39FDEC38FCEF2422FFEE3461FEED349DFD49
:202AC000EC346DFCD003D002D001D000EB2FFFEA3EFEE93DFDE83CFCA31200844C90002868
:202AE00083E0FCA3E0FDA3E0FEA3E0FF781012008392C004C005C006C00790002883E0FC18
:202B0000A3E0FDA3E0FEA3E0FF78101200837FD003D002D001D000EF4BFFEE4AFEED49FDAE
:202B2000EC48FC900028831200844C90002883E0FCA3E0FDA3E0FEA3E0FFA3E0F8A3E0F9B7
:202B4000A3E0FAA3E0FBEF2BFFEE3AFEED39FDEC38FC900028831200844C9000287FE0F8CC
:202B6000A3E0F9A3E0FAA3E0FBC000C001C002C00390002878E0FBA3E0FAA3E02438F9E494
:202B80003AFA120083FAC000C001C00290002887E0FCA3E0FDA3E0FEA3E0FF90002883E076
:202BA000F8A3E0F9A3E0FAA3E06FFFEA6EFEE96DFDE86CFC9000287BE0F8A3E0F9A3E0FA36
:202BC000A3E06FFFEA6EFEE96DFDE86CFCD002D001D000EF2BFFEE3AFEED39FDEC38FCEF27
:202BE000240CFFEE3438FEED34E5FDEC34FDFCD003D002D001D000EB2FFFEA3EFEE93DFD8A
:202C0000E83CFCA31200844C9000287FE0FCA3E0FDA3E0FEA3E0FF781712008392C004C03F
:202C200005C006C0079000287FE0FCA3E0FDA3E0FEA3E0FF78091200837FD003D002D00161
:202C4000D000EF4BFFEE4AFEED49FDEC48FC9000287F1200844C9000287FE0FCA3E0FDA383
:202C6000E0FEA3E0FFA3E0F8A3E0F9A3E0FAA3E0FBEF2BFFEE3AFEED39FDEC38FC900028C8
:202C80007F1200844C9000287BE0F8A3E0F9A3E0FAA3E0FBC000C001C002C003900028781B
:202CA000E0FBA3E0FAA3E02404F9E43AFA120083FAC000C001C00290002883E0FCA3E0FD97
:202CC000A3E0FEA3E0FF9000287FE0F8A3E0F9A3E0FAA3E06FFFEA6EFEE96DFDE86CFC906F
:202CE000002887E0F8A3E0F9A3E0FAA3E06FFFEA6EFEE96DFDE86CFCD002D001D000EF2BDD
:202D0000FFEE3AFEED39FDEC38FCEF2444FFEE34EAFEED34BEFDEC34A4FCD003D002D001D9
:202D2000D000EB2FFFEA3EFEE93DFDE83CFC9000287B1200844C9000287BE0FCA3E0FDA3FA
:202D4000E0FEA3E0FF780412008392C004C005C006C0079000287BE0FCA3E0FDA3E0FEA3A7
:202D6000E0FF781C1200837FD003D002D001D000EF4BFFEE4AFEED49FDEC48FC9000287B81
:202D80001200844C9000287BE0FCA3E0FDA3E0FEA3E0FFA3E0F8A3E0F9A3E0FAA3E0FBEFDE
:202DA0002BFFEE3AFEED39FDEC38FC9000287B1200844C90002887E0F8A3E0F9A3E0FAA3B8
:202DC000E0FBC000C001C002C00390002878E0FBA3E0FAA3E02410F9E43AFA120083FAC073
:202DE00000C001C0029000287FE0FCA3E0FDA3E0FEA3E0FF9000287BE0F8A3E0F9A3E0FAB6
:202E0000A3E06FFFEA6EFEE96DFDE86CFC90002883E0F8A3E0F9A3E0FAA3E06FFFEA6EFE75
:202E2000E96DFDE86CFCD002D001D000EF2BFFEE3AFEED39FDEC38FCEF24A9FFEE34CFFE50
:202E4000ED34DEFDEC344BFCD003D002D001D000EB2FFFEA3EFEE93DFDE83CFCA31200840E
:202E60004C90002887E0FCA3E0FDA3E0FEA3E0FF780B12008392C004C005C006C007900018
:202E80002887E0FCA3E0FDA3E0FEA3E0FF78151200837FD003D002D001D000EF4BFFEE4ACC
:202EA000FEED49FDEC48FC900028871200844C90002887E0FCA3E0FDA3E0FEA3E0FF900062
:202EC000287BE0F8A3E0F9A3E0FAA3E0FBEF2BFFEE3AFEED39FDEC38FC90002887120084A9
:202EE0004C90002883E0F8A3E0F9A3E0FAA3E0FBC000C001C002C00390002878E0FBA3E068
:202F0000FAA3E0241CF9E43AFA120083FAC000C001C0029000287BE0FCA3E0FDA3E0FEA35E
:202F2000E0FF90002887E0F8A3E0F9A3E0FAA3E06FFFEA6EFEE96DFDE86CFC9000287FE0A1
:202F4000F8A3E0F9A3E0FAA3E06FFFEA6EFEE96DFDE86CFCD002D001D000EF2BFFEE3AFEE4
:202F6000ED39FDEC38FCEF2460FFEE344BFEED34BBFDEC34F6FCD003D002D001D000EB2FE6
:202F8000FFEA3EFEE93DFDE83CFCA31200844C90002883E0FCA3E0FDA3E0FEA3E0FF781022
:202FA00012008392C004C005C006C00790002883E0FCA3E0FDA3E0FEA3E0FF78101200831D
:202FC0007FD003D002D001D000EF4BFFEE4AFEED49FDEC48FC900028831200844C90002885
:202FE00083E0FCA3E0FDA3E0FEA3E0FFA3E0F8A3E0F9A3E0FAA3E0FBEF2BFFEE3AFEED3998
:20300000FDEC38FC900028831200844C9000287FE0F8A3E0F9A3E0FAA3E0FBC000C001C0AF
:2030200002C00390002878E0FBA3E0FAA3E02428F9E43AFA120083FAC000C001C002900001
:203040002887E0FCA3E0FDA3E0FEA3E0FF90002883E0F8A3E0F9A3E0FAA3E06FFFEA6EFE0F
:20306000E96DFDE86CFC9000287BE0F8A3E0F9A3E0FAA3E06FFFEA6EFEE96DFDE86CFCD0EF
:2030800002D001D000EF2BFFEE3AFEED39FDEC38FCEF2470FFEE34BCFEED34BFFDEC34BEF2
:2030A000FCD003D002D001D000EB2FFFEA3EFEE93DFDE83CFCA31200844C9000287FE0FCB4
:2030C000A3E0FDA3E0FEA3E0FF781712008392C004C005C006C0079000287FE0FCA3E0FD0E
:2030E000A3E0FEA3E0FF78091200837FD003D002D001D000EF4BFFEE4AFEED49FDEC48FC20
:203100009000287F1200844C9000287FE0FCA3E0FDA3E0FEA3E0FFA3E0F8A3E0F9A3E0FA8C
:20312000A3E0FBEF2BFFEE3AFEED39FDEC38FC9000287F1200844C9000287BE0F8A3E0F9EF
:20314000A3E0FAA3E0FBC000C001C002C00390002878E0FBA3E0FAA3E02434F9E43AFA12E8
:203160000083FAC000C001C00290002883E0FCA3E0FDA3E0FEA3E0FF9000287FE0F8A3E063
:20318000F9A3E0FAA3E06FFFEA6EFEE96DFDE86CFC90002887E0F8A3E0F9A3E0FAA3E06FCD
:2031A000FFEA6EFEE96DFDE86CFCD002D001D000EF2BFFEE3AFEED39FDEC38FCEF24C6FF4A
:2031C000EE347EFEED349BFDEC3428FCD003D002D001D000EB2FFFEA3EFEE93DFDE83CFC8C
:2031E0009000287B1200844C9000287BE0FCA3E0FDA3E0FEA3E0FF780412008392C004C001
:2032000005C006C0079000287BE0FCA3E0FDA3E0FEA3E0FF781C1200837FD003D002D0016C
:20322000D000EF4BFFEE4AFEED49FDEC48FC9000287B1200844C9000287BE0FCA3E0FDA3A5
:20324000E0FEA3E0FFA3E0F8A3E0F9A3E0FAA3E0FBEF2BFFEE3AFEED39FDEC38FC900028E2
:203260007B1200844C90002887E0F8A3E0F9A3E0FAA3E0FBC000C001C002C0039000287F26
:20328000E0FCA3E0FDA3E0FEA3E0FF9000287BE0F8A3E0F9A3E0FAA3E06FFFEA6EFEE96D2E
:2032A000FDE86CFC90002883E0F8A3E0F9A3E0FAA3E06FFFEA6EFEE96DFDE86CFC90002813
:2032C00078E0FBA3E0FAA3E0F9120083FAEF2BFFEE3AFEED39FDEC38FCEF24FAFFEE34273C
:2032E000FEED34A1FDEC34EAFCD003D002D001D000EB2FFFEA3EFEE93DFDE83CFC9000288B
:20330000871200844C90002887E0FCA3E0FDA3E0FEA3E0FF780B12008392C004C005C006AD
:20332000C00790002887E0FCA3E0FDA3E0FEA3E0FF78151200837FD003D002D001D000EF52
:203340004BFFEE4AFEED49FDEC48FC900028871200844C90002887E0FCA3E0FDA3E0FEA3AA
:20336000E0FF9000287BE0F8A3E0F9A3E0FAA3E0FBEF2BFFEE3AFEED39FDEC38FC900028B2
:20338000871200844C90002883E0F8A3E0F9A3E0FAA3E0FBC000C001C002C0039000287804
:2033A000E0FBA3E0FAA3E0240CF9E43AFA120083FAC000C001C0029000287BE0FCA3E0FD90
:2033C000A3E0FEA3E0FF90002887E0F8A3E0F9A3E0FAA3E06FFFEA6EFEE96DFDE86CFC9060
:2033E00000287FE0F8A3E0F9A3E0FAA3E06FFFEA6EFEE96DFDE86CFCD002D001D000EF2BDE
:20340000FFEE3AFEED39FDEC38FCEF2485FFEE3430FEED34EFFDEC34D4FCD003D002D001EA
:20342000D000EB2FFFEA3EFEE93DFDE83CFCA31200844C90002883E0FCA3E0FDA3E0FEA3FA
:20344000E0FF781012008392C004C005C006C00790002883E0FCA3E0FDA3E0FEA3E0FF78B6
:20346000101200837FD003D002D001D000EF4BFFEE4AFEED49FDEC48FC900028831200843F
:203480004C90002883E0FCA3E0FDA3E0FEA3E0FFA3E0F8A3E0F9A3E0FAA3E0FBEF2BFFEE4D
:2034A0003AFEED39FDEC38FC900028831200844C9000287FE0F8A3E0F9A3E0FAA3E0FBC02E
:2034C00000C001C002C00390002878E0FBA3E0FAA3E02418F9E43AFA120083FAC000C0013E
:2034E000C00290002887E0FCA3E0FDA3E0FEA3E0FF90002883E0F8A3E0F9A3E0FAA3E06F6E
:20350000FFEA6EFEE96DFDE86CFC9000287BE0F8A3E0F9A3E0FAA3E06FFFEA6EFEE96DFD15
:20352000E86CFCD002D001D000EF2BFFEE3AFEED39FDEC38FCEF2405FFEE341DFEED348849
:20354000FDEC3404FCD003D002D001D000EB2FFFEA3EFEE93DFDE83CFCA31200844C900071
:20356000287FE0FCA3E0FDA3E0FEA3E0FF781712008392C004C005C006C0079000287FE062
:20358000FCA3E0FDA3E0FEA3E0FF78091200837FD003D002D001D000EF4BFFEE4AFEED492C
:2035A000FDEC48FC9000287F1200844C9000287FE0FCA3E0FDA3E0FEA3E0FFA3E0F8A3E031
:2035C000F9A3E0FAA3E0FBEF2BFFEE3AFEED39FDEC38FC9000287F1200844C9000287BE049
:2035E000F8A3E0F9A3E0FAA3E0FBC000C001C002C00390002878E0FBA3E0FAA3E02424F90A
:20360000E43AFA120083FAC000C001C00290002883E0FCA3E0FDA3E0FEA3E0FF9000287FEF
:20362000E0F8A3E0F9A3E0FAA3E06FFFEA6EFEE96DFDE86CFC90002887E0F8A3E0F9A3E0B9
:20364000FAA3E06FFFEA6EFEE96DFDE86CFCD002D001D000EF2BFFEE3AFEED39FDEC38FC91
:20366000EF2439FFEE34D0FEED34D4FDEC34D9FCD003D002D001D000EB2FFFEA3EFEE93D7D
:20368000FDE83CFC9000287B1200844C9000287BE0FCA3E0FDA3E0FEA3E0FF780412008355
:2036A00092C004C005C006C0079000287BE0FCA3E0FDA3E0FEA3E0FF781C1200837FD00355
:2036C000D002D001D000EF4BFFEE4AFEED49FDEC48FC9000287B1200844C9000287BE0FC81
:2036E000A3E0FDA3E0FEA3E0FFA3E0F8A3E0F9A3E0FAA3E0FBEF2BFFEE3AFEED39FDEC38CF
:20370000FC9000287B1200844C90002887E0F8A3E0F9A3E0FAA3E0FBC000C001C002C00304
:2037200090002878E0FBA3E0FAA3E02430F9E43AFA120083FAC000C001C0029000287FE030
:20374000FCA3E0FDA3E0FEA3E0FF9000287BE0F8A3E0F9A3E0FAA3E06FFFEA6EFEE96DFD4C
:20376000E86CFC90002883E0F8A3E0F9A3E0FAA3E06FFFEA6EFEE96DFDE86CFCD002D00160
:20378000D000EF2BFFEE3AFEED39FDEC38FCEF24E5FFEE3499FEED34DBFDEC34E6FCD00359
:2037A000D002D001D000EB2FFFEA3EFEE93DFDE83CFCA31200844C90002887E0FCA3E0FDF4
:2037C000A3E0FEA3E0FF780B12008392C004C005C006C00790002887E0FCA3E0FDA3E0FE0A
:2037E000A3E0FF78151200837FD003D002D001D000EF4BFFEE4AFEED49FDEC48FC900028D6
:20380000871200844C90002887E0FCA3E0FDA3E0FEA3E0FF9000287BE0F8A3E0F9A3E0FA9D
:20382000A3E0FBEF2BFFEE3AFEED39FDEC38FC900028871200844C90002883E0F8A3E0F9D8
:20384000A3E0FAA3E0FBC000C001C002C00390002878E0FBA3E0FAA3E0243CF9E43AFA12D9
:203860000083FAC000C001C0029000287BE0FCA3E0FDA3E0FEA3E0FF90002887E0F8A3E05C
:20388000F9A3E0FAA3E06FFFEA6EFEE96DFDE86CFC9000287FE0F8A3E0F9A3E0FAA3E06FCE
:2038A000FFEA6EFEE96DFDE86CFCD002D001D000EF2BFFEE3AFEED39FDEC38FCEF24F8FF11
:2038C000EE347CFEED34A2FDEC341FFCD003D002D001D000EB2FFFEA3EFEE93DFDE83CFC89
:2038E000A31200844C90002883E0FCA3E0FDA3E0FEA3E0FF781012008392C004C005C006AB
:20390000C00790002883E0FCA3E0FDA3E0FEA3E0FF78101200837FD003D002D001D000EF75
:203920004BFFEE4AFEED49FDEC48FC900028831200844C90002883E0FCA3E0FDA3E0FEA3CC
:20394000E0FFA3E0F8A3E0F9A3E0FAA3E0FBEF2BFFEE3AFEED39FDEC38FC900028831200C7
:20396000844C9000287FE0F8A3E0F9A3E0FAA3E0FBC000C001C002C00390002878E0FBA33D
:20398000E0FAA3E02408F9E43AFA120083FAC000C001C00290002887E0FCA3E0FDA3E0FE9F
:2039A000A3E0FF90002883E0F8A3E0F9A3E0FAA3E06FFFEA6EFEE96DFDE86CFC9000287B5C
:2039C000E0F8A3E0F9A3E0FAA3E06FFFEA6EFEE96DFDE86CFCD002D001D000EF2BFFEE3A78
:2039E000FEED39FDEC38FCEF2465FFEE3456FEED34ACFDEC34C4FCD003D002D001D000EBBE
:203A00002FFFEA3EFEE93DFDE83CFCA31200844C9000287FE0FCA3E0FDA3E0FEA3E0FF787C
:203A20001712008392C004C005C006C0079000287FE0FCA3E0FDA3E0FEA3E0FF7809120009
:203A4000837FD003D002D001D000EF4BFFEE4AFEED49FDEC48FC9000287F1200844C9000A3
:203A6000287FE0FCA3E0FDA3E0FEA3E0FFA3E0F8A3E0F9A3E0FAA3E0FBEF2BFFEE3AFEED22
:203A800039FDEC38FC9000287F1200844C9000287BE0F8A3E0F9A3E0FAA3E0FBC000C001B4
:203AA000C002C00390002887E0FCA3E0FDA3E0FEA3E0FF120083619000287FE0F8A3E0F962
:203AC000A3E0FAA3E04FFFEA4EFEE94DFDE84CFCA3E0F8A3E0F9A3E0FAA3E06FFFEA6EFE44
:203AE000E96DFDE86CFC90002878E0FBA3E0FAA3E0F9120083FAEF2BFFEE3AFEED39FDEC42
:203B000038FCEF2444FFEE3422FEED3429FDEC34F4FCD003D002D001D000EB2FFFEA3EFEFD
:203B2000E93DFDE83CFC9000287B1200844C9000287BE0FCA3E0FDA3E0FEA3E0FF7806120B
:203B4000008392C004C005C006C0079000287BE0FCA3E0FDA3E0FEA3E0FF781A1200837F02
:203B6000D003D002D001D000EF4BFFEE4AFEED49FDEC48FC9000287B1200844C9000287BE5
:203B8000E0FCA3E0FDA3E0FEA3E0FFA3E0F8A3E0F9A3E0FAA3E0FBEF2BFFEE3AFEED39FD72
:203BA000EC38FC9000287B1200844C90002887E0F8A3E0F9A3E0FAA3E0FBC000C001C002FF
:203BC000C00390002883E0FCA3E0FDA3E0FEA3E0FF120083619000287BE0F8A3E0F9A3E088
:203BE000FAA3E04FFFEA4EFEE94DFDE84CFCA3E0F8A3E0F9A3E0FAA3E06FFFEA6EFEE96D50
:203C0000FDE86CFC90002878E0FBA3E0FAA3E0241CF9E43AFA120083FAEF2BFFEE3AFEED40
:203C200039FDEC38FCEF2497FFEE34FFFEED342AFDEC3443FCD003D002D001D000EB2FFF60
:203C4000EA3EFEE93DFDE83CFC900028871200844C90002887E0FCA3E0FDA3E0FEA3E0FF3C
:203C6000780A12008392C004C005C006C00790002887E0FCA3E0FDA3E0FEA3E0FF78161247
:203C800000837FD003D002D001D000EF4BFFEE4AFEED49FDEC48FC900028871200844C9059
:203CA000002887E0FCA3E0FDA3E0FEA3E0FF9000287BE0F8A3E0F9A3E0FAA3E0FBEF2BFF5B
:203CC000EE3AFEED39FDEC38FC900028871200844C90002883E0F8A3E0F9A3E0FAA3E0FBD0
:203CE000C000C001C002C0039000287FE0FCA3E0FDA3E0FEA3E0FF1200836190002887E013
:203D0000F8A3E0F9A3E0FAA3E04FFFEA4EFEE94DFDE84CFC9000287BE0F8A3E0F9A3E0FA44
:203D2000A3E06FFFEA6EFEE96DFDE86CFC90002878E0FBA3E0FAA3E02438F9E43AFA12000F
:203D400083FAEF2BFFEE3AFEED39FDEC38FCEF24A7FFEE3423FEED3494FDEC34ABFCD0031C
:203D6000D002D001D000EB2FFFEA3EFEE93DFDE83CFC900028831200844C90002883E0FC1A
:203D8000A3E0FDA3E0FEA3E0FF780F12008392C004C005C006C00790002883E0FCA3E0FD45
:203DA000A3E0FEA3E0FF78111200837FD003D002D001D000EF4BFFEE4AFEED49FDEC48FC4B
:203DC000900028831200844C90002883E0FCA3E0FDA3E0FEA3E0FFA3E0F8A3E0F9A3E0FAB8
:203DE000A3E0FBEF2BFFEE3AFEED39FDEC38FC900028831200844C9000287FE0F8A3E0F91B
:203E0000A3E0FAA3E0FBC000C001C002C0039000287BE0FCA3E0FDA3E0FEA3E0FF1200837A
:203E20006190002883E0F8A3E0F9A3E0FAA3E04FFFEA4EFEE94DFDE84CFCA3E0F8A3E0F9B4
:203E4000A3E0FAA3E06FFFEA6EFEE96DFDE86CFC90002878E0FBA3E0FAA3E02414F9E43AA1
:203E6000FA120083FAEF2BFFEE3AFEED39FDEC38FCEF2439FFEE34A0FEED3493FDEC34FC5F
:203E8000FCD003D002D001D000EB2FFFEA3EFEE93DFDE83CFC9000287F1200844C9000288D
:203EA0007FE0FCA3E0FDA3E0FEA3E0FF781512008392C004C005C006C0079000287FE0FC47
:203EC000A3E0FDA3E0FEA3E0FF780B1200837FD003D002D001D000EF4BFFEE4AFEED49FDE0
:203EE000EC48FC9000287F1200844C9000287FE0FCA3E0FDA3E0FEA3E0FFA3E0F8A3E0F9EC
:203F0000A3E0FAA3E0FBEF2BFFEE3AFEED39FDEC38FC9000287F1200844C9000287BE0F800
:203F2000A3E0F9A3E0FAA3E0FBC000C001C002C00390002887E0FCA3E0FDA3E0FEA3E0FF66
:203F4000120083619000287FE0F8A3E0F9A3E0FAA3E04FFFEA4EFEE94DFDE84CFCA3E0F87E
:203F6000A3E0F9A3E0FAA3E06FFFEA6EFEE96DFDE86CFC90002878E0FBA3E0FAA3E02430FF
:203F8000F9E43AFA120083FAEF2BFFEE3AFEED39FDEC38FCEF24C3FFEE3459FEED345BFD38
:203FA000EC3465FCD003D002D001D000EB2FFFEA3EFEE93DFDE83CFC9000287B1200844CA3
:203FC0009000287BE0FCA3E0FDA3E0FEA3E0FF780612008392C004C005C006C007900028DC
:203FE0007BE0FCA3E0FDA3E0FEA3E0FF781A1200837FD003D002D001D000EF4BFFEE4AFE8C
:20400000ED49FDEC48FC9000287B1200844C9000287BE0FCA3E0FDA3E0FEA3E0FFA3E0F81B
:20402000A3E0F9A3E0FAA3E0FBEF2BFFEE3AFEED39FDEC38FC9000287B1200844C900028BA
:2040400087E0F8A3E0F9A3E0FAA3E0FBC000C001C002C00390002883E0FCA3E0FDA3E0FE6C
:20406000A3E0FF120083619000287BE0F8A3E0F9A3E0FAA3E04FFFEA4EFEE94DFDE84CFC5A
:20408000A3E0F8A3E0F9A3E0FAA3E06FFFEA6EFEE96DFDE86CFC90002878E0FBA3E0FAA397
:2040A000E0240CF9E43AFA120083FAEF2BFFEE3AFEED39FDEC38FCEF2492FFEE34CCFEED51
:2040C000340CFDEC348FFCD003D002D001D000EB2FFFEA3EFEE93DFDE83CFC9000288712DF
:2040E00000844C90002887E0FCA3E0FDA3E0FEA3E0FF780A12008392C004C005C006C00793
:2041000090002887E0FCA3E0FDA3E0FEA3E0FF78161200837FD003D002D001D000EF4BFFE0
:20412000EE4AFEED49FDEC48FC900028871200844C90002887E0FCA3E0FDA3E0FEA3E0FF27
:204140009000287BE0F8A3E0F9A3E0FAA3E0FBEF2BFFEE3AFEED39FDEC38FC90002887120A
:2041600000844C90002883E0F8A3E0F9A3E0FAA3E0FBC000C001C002C0039000287FE0FCCC
:20418000A3E0FDA3E0FEA3E0FF1200836190002887E0F8A3E0F9A3E0FAA3E04FFFEA4EFE8F
:2041A000E94DFDE84CFC9000287BE0F8A3E0F9A3E0FAA3E06FFFEA6EFEE96DFDE86CFC901E
:2041C000002878E0FBA3E0FAA3E02428F9E43AFA120083FAEF2BFFEE3AFEED39FDEC38FCF6
:2041E000EF247DFFEE34F4FEED34EFFDEC34FFFCD003D002D001D000EB2FFFEA3EFEE93D49
:20420000FDE83CFC900028831200844C90002883E0FCA3E0FDA3E0FEA3E0FF780F120083AE
:2042200092C004C005C006C00790002883E0FCA3E0FDA3E0FEA3E0FF78111200837FD003CC
:20424000D002D001D000EF4BFFEE4AFEED49FDEC48FC900028831200844C90002883E0FCE5
:20426000A3E0FDA3E0FEA3E0FFA3E0F8A3E0F9A3E0FAA3E0FBEF2BFFEE3AFEED39FDEC3843
:20428000FC900028831200844C9000287FE0F8A3E0F9A3E0FAA3E0FBC000C001C002C00379
:2042A0009000287BE0FCA3E0FDA3E0FEA3E0FF1200836190002883E0F8A3E0F9A3E0FAA3C7
:2042C000E04FFFEA4EFEE94DFDE84CFCA3E0F8A3E0F9A3E0FAA3E06FFFEA6EFEE96DFDE821
:2042E0006CFC90002878E0FBA3E0FAA3E02404F9E43AFA120083FAEF2BFFEE3AFEED39FD21
:20430000EC38FCEF24D1FFEE345DFEED3484FDEC3485FCD003D002D001D000EB2FFFEA3E53
:20432000FEE93DFDE83CFC9000287F1200844C9000287FE0FCA3E0FDA3E0FEA3E0FF781500
:2043400012008392C004C005C006C0079000287FE0FCA3E0FDA3E0FEA3E0FF780B12008372
:204360007FD003D002D001D000EF4BFFEE4AFEED49FDEC48FC9000287F1200844C900028D5
:204380007FE0FCA3E0FDA3E0FEA3E0FFA3E0F8A3E0F9A3E0FAA3E0FBEF2BFFEE3AFEED39E8
:2043A000FDEC38FC9000287F1200844C9000287BE0F8A3E0F9A3E0FAA3E0FBC000C001C004
:2043C00002C00390002887E0FCA3E0FDA3E0FEA3E0FF120083619000287FE0F8A3E0F9A356
:2043E000E0FAA3E04FFFEA4EFEE94DFDE84CFCA3E0F8A3E0F9A3E0FAA3E06FFFEA6EFEE9D5
:204400006DFDE86CFC90002878E0FBA3E0FAA3E02420F9E43AFA120083FAEF2BFFEE3AFEB4
:20442000ED39FDEC38FCEF244FFFEE347EFEED34A8FDEC346FFCD003D002D001D000EB2F89
:20444000FFEA3EFEE93DFDE83CFC9000287B1200844C9000287BE0FCA3E0FDA3E0FEA3E04C
:20446000FF780612008392C004C005C006C0079000287BE0FCA3E0FDA3E0FEA3E0FF781A5E
:204480001200837FD003D002D001D000EF4BFFEE4AFEED49FDEC48FC9000287B1200844CDB
:2044A0009000287BE0FCA3E0FDA3E0FEA3E0FFA3E0F8A3E0F9A3E0FAA3E0FBEF2BFFEE3A37
:2044C000FEED39FDEC38FC9000287B1200844C90002887E0F8A3E0F9A3E0FAA3E0FBC00038
:2044E000C001C002C00390002883E0FCA3E0FDA3E0FEA3E0FF120083619000287BE0F8A338
:20450000E0F9A3E0FAA3E04FFFEA4EFEE94DFDE84CFCA3E0F8A3E0F9A3E0FAA3E06FFFEA8C
:204520006EFEE96DFDE86CFC90002878E0FBA3E0FAA3E0243CF9E43AFA120083FAEF2BFF48
:20454000EE3AFEED39FDEC38FCEF24E0FFEE34E6FEED342CFDEC34FEFCD003D002D001D050
:2045600000EB2FFFEA3EFEE93DFDE83CFC900028871200844C90002887E0FCA3E0FDA3E07A
:20458000FEA3E0FF780A12008392C004C005C006C00790002887E0FCA3E0FDA3E0FEA3E03D
:2045A000FF78161200837FD003D002D001D000EF4BFFEE4AFEED49FDEC48FC9000288712F1
:2045C00000844C90002887E0FCA3E0FDA3E0FEA3E0FF9000287BE0F8A3E0F9A3E0FAA3E0E6
:2045E000FBEF2BFFEE3AFEED39FDEC38FC900028871200844C90002883E0F8A3E0F9A3E00B
:20460000FAA3E0FBC000C001C002C0039000287FE0FCA3E0FDA3E0FEA3E0FF120083619000
:20462000002887E0F8A3E0F9A3E0FAA3E04FFFEA4EFEE94DFDE84CFC9000287BE0F8A3E002
:20464000F9A3E0FAA3E06FFFEA6EFEE96DFDE86CFC90002878E0FBA3E0FAA3E02418F9E4D6
:204660003AFA120083FAEF2BFFEE3AFEED39FDEC38FCEF2414FFEE3443FEED3401FDEC342D
:20468000A3FCD003D002D001D000EB2FFFEA3EFEE93DFDE83CFC900028831200844C900006
:2046A0002883E0FCA3E0FDA3E0FEA3E0FF780F12008392C004C005C006C00790002883E011
:2046C000FCA3E0FDA3E0FEA3E0FF78111200837FD003D002D001D000EF4BFFEE4AFEED49D3
:2046E000FDEC48FC900028831200844C90002883E0FCA3E0FDA3E0FEA3E0FFA3E0F8A3E0D8
:20470000F9A3E0FAA3E0FBEF2BFFEE3AFEED39FDEC38FC900028831200844C9000287FE0EF
:20472000F8A3E0F9A3E0FAA3E0FBC000C001C002C0039000287BE0FCA3E0FDA3E0FEA3E071
:20474000FF1200836190002883E0F8A3E0F9A3E0FAA3E04FFFEA4EFEE94DFDE84CFCA3E06B
:20476000F8A3E0F9A3E0FAA3E06FFFEA6EFEE96DFDE86CFC90002878E0FBA3E0FAA3E0242F
:2047800034F9E43AFA120083FAEF2BFFEE3AFEED39FDEC38FCEF24A1FFEE3411FEED3408B6
:2047A000FDEC344EFCD003D002D001D000EB2FFFEA3EFEE93DFDE83CFC9000287F120084FD
:2047C0004C9000287FE0FCA3E0FDA3E0FEA3E0FF781512008392C004C005C006C00790009D
:2047E000287FE0FCA3E0FDA3E0FEA3E0FF780B1200837FD003D002D001D000EF4BFFEE4A65
:20480000FEED49FDEC48FC9000287F1200844C9000287FE0FCA3E0FDA3E0FEA3E0FFA3E005
:20482000F8A3E0F9A3E0FAA3E0FBEF2BFFEE3AFEED39FDEC38FC9000287F1200844C9000DE
:20484000287BE0F8A3E0F9A3E0FAA3E0FBC000C001C002C00390002887E0FCA3E0FDA3E042
:20486000FEA3E0FF120083619000287FE0F8A3E0F9A3E0FAA3E04FFFEA4EFEE94DFDE84C4C
:20488000FCA3E0F8A3E0F9A3E0FAA3E06FFFEA6EFEE96DFDE86CFC90002878E0FBA3E0FA36
:2048A000A3E02410F9E43AFA120083FAEF2BFFEE3AFEED39FDEC38FCEF2482FFEE347EFEED
:2048C000ED3453FDEC34F7FCD003D002D001D000EB2FFFEA3EFEE93DFDE83CFC9000287B59
:2048E0001200844C9000287BE0FCA3E0FDA3E0FEA3E0FF780612008392C004C005C006C090
:20490000079000287BE0FCA3E0FDA3E0FEA3E0FF781A1200837FD003D002D001D000EF4BD8
:20492000FFEE4AFEED49FDEC48FC9000287B1200844C9000287BE0FCA3E0FDA3E0FEA3E037
:20494000FFA3E0F8A3E0F9A3E0FAA3E0FBEF2BFFEE3AFEED39FDEC38FC9000287B1200841B
:204960004C90002887E0F8A3E0F9A3E0FAA3E0FBC000C001C002C00390002883E0FCA3E0BD
:20498000FDA3E0FEA3E0FF120083619000287BE0F8A3E0F9A3E0FAA3E04FFFEA4EFEE94DE0
:2049A000FDE84CFCA3E0F8A3E0F9A3E0FAA3E06FFFEA6EFEE96DFDE86CFC90002878E0FB61
:2049C000A3E0FAA3E0242CF9E43AFA120083FAEF2BFFEE3AFEED39FDEC38FCEF2435FFEE30
:2049E00034F2FEED343AFDEC34BDFCD003D002D001D000EB2FFFEA3EFEE93DFDE83CFC900A
:204A00000028871200844C90002887E0FCA3E0FDA3E0FEA3E0FF780A12008392C004C00535
:204A2000C006C00790002887E0FCA3E0FDA3E0FEA3E0FF78161200837FD003D002D001D063
:204A400000EF4BFFEE4AFEED49FDEC48FC900028871200844C90002887E0FCA3E0FDA3E045
:204A6000FEA3E0FF9000287BE0F8A3E0F9A3E0FAA3E0FBEF2BFFEE3AFEED39FDEC38FC9022
:204A80000028871200844C90002883E0F8A3E0F9A3E0FAA3E0FBC000C001C002C003900065
:204AA000287FE0FCA3E0FDA3E0FEA3E0FF1200836190002887E0F8A3E0F9A3E0FAA3E04F18
:204AC000FFEA4EFEE94DFDE84CFC9000287BE0F8A3E0F9A3E0FAA3E06FFFEA6EFEE96DFDA0
:204AE000E86CFC90002878E0FBA3E0FAA3E02408F9E43AFA120083FAEF2BFFEE3AFEED392A
:204B0000FDEC38FCEF24BBFFEE34D2FEED34D7FDEC342AFCD003D002D001D000EB2FFFEA35
:204B20003EFEE93DFDE83CFC900028831200844C90002883E0FCA3E0FDA3E0FEA3E0FF78C7
:204B40000F12008392C004C005C006C00790002883E0FCA3E0FDA3E0FEA3E0FF78111200D4
:204B6000837FD003D002D001D000EF4BFFEE4AFEED49FDEC48FC900028831200844C90006E
:204B80002883E0FCA3E0FDA3E0FEA3E0FFA3E0F8A3E0F9A3E0FAA3E0FBEF2BFFEE3AFEEDED
:204BA00039FDEC38FC900028831200844C9000287FE0F8A3E0F9A3E0FAA3E0FBC000C0017B
:204BC000C002C0039000287BE0FCA3E0FDA3E0FEA3E0FF1200836190002883E0F8A3E0F939
:204BE000A3E0FAA3E04FFFEA4EFEE94DFDE84CFCA3E0F8A3E0F9A3E0FAA3E06FFFEA6EFE13
:204C0000E96DFDE86CFC90002878E0FBA3E0FAA3E02424F9E43AFA120083FAEF2BFFEE3ABD
:204C2000FEED39FDEC38FCEF2491FFEE34D3FEED3486FDEC34EBFCD003D002D001D000EBC1
:204C40002FFFEA3EFEE93DFDE83CFC9000287F1200844C9000287FE0FCA3E0FDA3E0FEA3ED
:204C6000E0FF781512008392C004C005C006C0079000287FE0FCA3E0FDA3E0FEA3E0FF787D
:204C80000B1200837FD003D002D001D000EF4BFFEE4AFEED49FDEC48FC9000287F12008410
:204CA0004C9000287FE0FCA3E0FDA3E0FEA3E0FFA3E0F8A3E0F9A3E0FAA3E0FBEF2BFFEE19
:204CC0003AFEED39FDEC38FC9000287F1200844C90002875E0FBA3E0FAA3E0F9C002C001BC
:204CE000120083A59000287BE0F8A3E0F9A3E0FAA3E02FFFEA3EFEE93DFDE83CFCD001D0BB
:204D000002120083C290002875E0FBA3E0FAA3E02404F9E43AFAC002C001120083A59000AC
:204D2000287FE0F8A3E0F9A3E0FAA3E02FFFEA3EFEE93DFDE83CFCD001D002120083C29057
:204D4000002875E0FBA3E0FAA3E02408F9E43AFAC002C001120083A590002883E0F8A3E04B
:204D6000F9A3E0FAA3E02FFFEA3EFEE93DFDE83CFCD001D002120083C290002875E0FBA3FE
:204D8000E0FAA3E0240CF9E43AFAC002C001120083A590002887E0F8A3E0F9A3E0FAA3E025
:204DA0002FFFEA3EFEE93DFDE83CFCD001D002020083C290001551E0FBA3E0FAA3E0F9E4C4
:204DC00075F001120081D2AFF0FE6003215AA1EF24FE7003214EBA1470032152431470037B
:204DE00021549C14700321580A24046003215AA190002B407484F0A37419F0A3747BF090DC
:204E00000019BBE0FBA3E0FAA3E0F912029EF690001DD1EBF0A3EAF0A3E9F090001DD1E092
:204E2000FBA3E0FAA3E04A4B70037F0122900025A17484F0A37419F0A37483F0A37401F0DD
:204E4000A3741DF0A374D4F090001DD1E0FBA3E0FAA3E0F91200D582900026A17484F0A3B6
:204E60007419F0A3748DF090001DD4E0FEA3E0FF900026A4EEF0A3EFF02401FFE43EA3F0AD
:204E8000A3EFF0900019BBE0FBA3E0FAA3E0F91200D1A390001AAEEEF0A3EFF090001DD499
:204EA000E0F9A3E0FF9000155CE0FBA3E0FAA3E0C98FF012008228215AA49000155CE0FBBC
:204EC000A3E0FAA3E0F9120081AEFF1202DA56EF64044E701B9000155CE0FBA3E0FAA3E049
:204EE000F9120081AEFF1202D4D3EF4E700280349000155CE0FBA3E0FAA3E0F9120081AE45
:204F0000FF1202DA56EF64054E70299000155CE0FBA3E0FAA3E0F9120081AEFF1202D4D33F
:204F2000EF4E7010FE7F9CFD7B017A1D7935120088AA80767E007F9C7D007B017A1D7935CC
:204F4000120088AA9000155CE0FBA3E0FAA3E0F9120081AEFF7B017A1D793590002E2F74D6
:204F600001F01202DBA69000155CE0FBA3E0FAA3E0F9120081AEFF7B017A1D793590002E17
:204F80002F7405F01202DBA69000155CE0FBA3E0FAA3E0F9120081AEFF7B017A1D7935907E
:204FA000002E2F7406F01202DBA6900026A17481F0A37490F0A37406F0A37484F0A3741AF9
:204FC000F0A374A5F090001DADE0FCA3E0FDA3E0FEA3E0FF900026A71200844C900019BBD9
:204FE000E0FBA3E0FAA3E0F91200D1A390001AAEEEF0A3EFF0900019BBE0FBA3E0FAA3E060
:20500000F990001AAEE0FEA3E0FFE92FF9EA3EFAC003900026A17484F0A3741AF0A374A8CA
:20502000F090001D51E0FCA3E0FDA3E0FEA3E0FF900026A41200844C90001DBDE0FCA3E01E
:20504000FDA3E0FEA3E0FF900026A81200844CD0031200D1A390001AAFE02FF090001AAE07
:20506000E03EF090001DD4E4F0A304F090001DD4E0FEA3E0FFD39403EE64809480400321A1
:205080005AA4EE600321518CEF24FE606D1470032151402402600321518C90001DD67484AA
:2050A000F0A3741BF0A37413F090001D59E0FCA3E0FDA3E0FEA3E0FF90001DDC1200844CF4
:2050C00090001DD97484F0A3741BF0A37421F090001DC5E0FCA3E0FDA3E0FEA3E0FF9000B7
:2050E0001DC1E0F8A3E0F9A3E0FAA3E02FFFEA3EFEE93DFDE83CFC21518490001DD6748476
:20510000F0A3741BF0A3742FF090001D55E0FCA3E0FDA3E0FEA3E0FF90001DDC1200844C7B
:2051200090001DD97484F0A3741BF0A3743DF090001DCDE0FCA3E0FDA3E0FEA3E0FF8044FE
:2051400090001DD67484F0A3741BF0A3744BF090001D5DE0FCA3E0FDA3E0FEA3E0FF900077
:205160001DDC1200844C90001DD97484F0A3741BF0A37460F090001DC9E0FCA3E0FDA3E008
:20518000FEA3E0FF90001DE01200844C900019BBE0FBA3E0FAA3E0F990001AAEE0FEA3E02F
:2051A000FFE92FF9EA3EFAC003C002C001900026A17481F0A37490F0A37443F090001DD6D7
:2051C000E0F9A3E0FAA3E0900026A4C9F0A3EAF0A3E9F090001DDCE0FCA3E0FDA3E0FEA3E1
:2051E000E0FF900026A71200844C90001DD9E0F9A3E0FAA3E0900026ABC9F0A3EAF0A3E90F
:20520000F090001DE0E0FCA3E0FDA3E0FEA3E0FF900026AE1200844CD001D002D0031200E4
:20522000D1A390001AAFE02FF090001AAEE03EF090001DD5E004F0700790001DD4E004F01A
:2052400021506C9000155CE0FBA3E0FAA3E0F9120081AEFF1202DA56EF64044E701B900058
:20526000155CE0FBA3E0FAA3E0F9120081AEFF1202D4D3EF4E700280349000155CE0FBA30C
:20528000E0FAA3E0F9120081AEFF1202DA56EF64054E70299000155CE0FBA3E0FAA3E0F920
:2052A000120081AEFF1202D4D3EF4E7010FE7F9CFD7B017A1D7935120088AA80327E007F6C
:2052C0009C7D007B017A1D7935120088AA9000155CE0FBA3E0FAA3E0F9120081AEFF7B011F
:2052E0007A1D793590002E2F7403F01202DBA690001DD4E4F0A304F090001DD4E0FEA3E0B2
:20530000FFD39403EE648094804003215AA4EE60032153E5EF24FE604514607D2402600302
:205320002153E590001DD67484F0A3741BF0A37473F090001D8DE0FCA3E0FDA3E0FEA3E073
:20534000FF90001DDC1200844C90001DD97484F0A3741BF0A3747FF090001D91807490000B
:205360001DD67484F0A3741BF0A37492F090001D95E0FCA3E0FDA3E0FEA3E0FF90001DDC6D
:205380001200844C90001DD97484F0A3741BF0A374A6F090001D99803990001DD67484F084
:2053A000A3741BF0A374BAF090001D9DE0FCA3E0FDA3E0FEA3E0FF90001DDC1200844C9066
:2053C000001DD97484F0A3741BF0A374CFF090001DA1E0FCA3E0FDA3E0FEA3E0FF90001D9D
:2053E000E01200844C900019BBE0FBA3E0FAA3E0F990001AAEE0FEA3E0FFE92FF9EA3EFAC8
:20540000C003C002C001900026A17481F0A37490F0A37443F090001DD6E0F9A3E0FAA3E0CD
:20542000900026A4C9F0A3EAF0A3E9F090001DDCE0FCA3E0FDA3E0FEA3E0FF900026A71209
:2054400000844C90001DD9E0F9A3E0FAA3E0900026ABC9F0A3EAF0A3E9F090001DE0E0FCA1
:20546000A3E0FDA3E0FEA3E0FF900026AE1200844CD001D002D0031200D1A390001AAFE02E
:205480002FF090001AAEE03EF090001DD5E004F0700790001DD4E004F02152F89000155CF9
:2054A000E0FBA3E0FAA3E0F9120081AEFF1202DA56EF64044E701B9000155CE0FBA3E0FA0B
:2054C000A3E0F9120081AEFF1202D4D3EF4E700280349000155CE0FBA3E0FAA3E0F912000B
:2054E00081AEFF1202DA56EF64054E70299000155CE0FBA3E0FAA3E0F9120081AEFF1202D2
:20550000D4D3EF4E7010FE7F9CFD7B017A1D7935120088AA80757E007F9C7D007B017A1DEE
:205520007935120088AA9000155CE0FBA3E0FAA3E0F9120081AEFF7B017A1D7935E490002F
:205540002E2FF01202DBA69000155CE0FBA3E0FAA3E0F9120081AEFF7B017A1D7935900003
:205560002E2F7402F01202DBA69000155CE0FBA3E0FAA3E0F9120081AEFF7B017A1D7935FD
:2055800090002E2F7405F01202DBA6900026A17481F0A37490F0A37406F0A37484F0A3749E
:2055A0001BF0A374E5F090001DB5E0FCA3E0FDA3E0FEA3E0FF900026A71200844C9000194B
:2055C000BBE0FBA3E0FAA3E0F91200D1A390001AAEEEF0A3EFF090001DD4E4F0A304F09082
:2055E000001DD4E0FEA3E0FFD39405EE648094804003215AA4EE6003215753EF24FE6055C4
:205600001470032156911470032156CC1470032157072404600321575390001DD67484F06A
:20562000A3741BF0A374E8F090001D35E0FCA3E0FDA3E0FEA3E0FF90001DDC1200844C901D
:20564000001DD97484F0A3741BF0A374F4F090001D7D21574090001DD67484F0A3741BF0E0
:20566000A37413F090001D3DE0FCA3E0FDA3E0FEA3E0FF90001DDC1200844C90001DD97462
:2056800084F0A3741CF0A37402F090001D8121574090001DD67484F0A3741BF0A3742FF0C1
:2056A00090001D39E0FCA3E0FDA3E0FEA3E0FF90001DDC1200844C90001DD97484F0A374B5
:2056C0001CF0A3740FF090001D85807490001DD67484F0A3741BF0A3744BF090001D41E0D5
:2056E000FCA3E0FDA3E0FEA3E0FF90001DDC1200844C90001DD97484F0A3741CF0A3741FF9
:20570000F090001D89803990001DD67484F0A3741CF0A3742EF090001D45E0FCA3E0FDA3F6
:20572000E0FEA3E0FF90001DDC1200844C90001DD97484F0A3741CF0A37438F090001D49D8
:20574000E0FCA3E0FDA3E0FEA3E0FF90001DE01200844C900019BBE0FBA3E0FAA3E0F990B3
:20576000001AAEE0FEA3E0FFE92FF9EA3EFAC003C002C001900026A17481F0A37490F0A312
:205780007443F090001DD6E0F9A3E0FAA3E0900026A4C9F0A3EAF0A3E9F090001DDCE0FC95
:2057A000A3E0FDA3E0FEA3E0FF900026A71200844C90001DD9E0F9A3E0FAA3E0900026AB67
:2057C000C9F0A3EAF0A3E9F090001DE0E0FCA3E0FDA3E0FEA3E0FF900026AE1200844CD015
:2057E00001D002D0031200D1A390001AAFE02FF090001AAEE03EF090001DD5E004F07007F2
:2058000090001DD4E004F02155DF9000155CE0FBA3E0FAA3E0F9120081AEFF1202DA56EF96
:2058200064044E701B9000155CE0FBA3E0FAA3E0F9120081AEFF1202D4D3EF4E70028034F4
:205840009000155CE0FBA3E0FAA3E0F9120081AEFF1202DA56EF64054E70299000155CE0CF
:20586000FBA3E0FAA3E0F9120081AEFF1202D4D3EF4E7010FE7F9CFD7B017A1D7935120093
:2058800088AA80327E007F9C7D007B017A1D7935120088AA9000155CE0FBA3E0FAA3E0F934
:2058A000120081AEFF7B017A1D793590002E2F7402F01202DBA690001DD4E4F0A304F09083
:2058C000001DD4E0FEA3E0FFD39403EE648094804003215A63EE60032159ACEF24FE6045D9
:2058E00014607D240260032159AC90001DD67484F0A3741BF0A37473F090001D61E0FCA374
:20590000E0FDA3E0FEA3E0FF90001DDC1200844C90001DD97484F0A3741BF0A3747FF09096
:20592000001D65807490001DD67484F0A3741BF0A37492F090001D69E0FCA3E0FDA3E0FED8
:20594000A3E0FF90001DDC1200844C90001DD97484F0A3741BF0A374A6F090001D6D80394A
:2059600090001DD67484F0A3741BF0A374BAF090001D71E0FCA3E0FDA3E0FEA3E0FF9000CC
:205980001DDC1200844C90001DD97484F0A3741BF0A374CFF090001D75E0FCA3E0FDA3E0C5
:2059A000FEA3E0FF90001DE01200844C900019BBE0FBA3E0FAA3E0F990001AAEE0FEA3E007
:2059C000FFE92FF9EA3EFAC003C002C001900026A17481F0A37490F0A37443F090001DD6AF
:2059E000E0F9A3E0FAA3E0900026A4C9F0A3EAF0A3E9F090001DDCE0FCA3E0FDA3E0FEA3B9
:205A0000E0FF900026A71200844C90001DD9E0F9A3E0FAA3E0900026ABC9F0A3EAF0A3E9E6
:205A2000F090001DE0E0FCA3E0FDA3E0FEA3E0FF900026AE1200844CD001D002D0031200BC
:205A4000D1A390001AAFE02FF090001AAEE03EF090001DD5E004F0700790001DD4E004F0F2
:205A60002158BF900019BBE0FBA3E0FAA3E0F990001AAEE0FEA3E0FFE92FF9EA3EFA90003B
:205A800026A17484F0A3741CF0A37448F01200D1A390001AAFE02FF090001AAEE03EF08021
:205AA000037F01227F002290001551E0FBA3E0FAA3E0F9120081AEFFAEF0E5F0600321653A
:205AC00033EF120084D55AFA015F32025F99035FBA0760250860320960360D60860E6230E5
:205AE0000F640410640412647013647D1664D51764E21864E21A00006533900026A17484D2
:205B0000F0A37400F0A37468F0900019BBE0FBA3E0FAA3E0F91200D1A390001AAEEEF0A388
:205B2000EFF0E4900022FDF0A3F0900022FDE475F00112008182AFF0FE6003215E0EEF14D2
:205B4000B40E004003215E0E90015B5775F004A4C58325F0C5837302015B8F02015BAD0251
:205B6000015BCB02015BFE02015C0E02015C1E02015C3302015C4802015C5D02015C7B02E7
:205B8000015D1102015D2C02015D4C02015D79900023077484F0A37401F0A374A2F0780AB0
:205BA0007C237D017B847A0179AF215D45900023077484F0A37401F0A374B9F0780A7C23D8
:205BC0007D017B847A0179CA215D45900023077484F0A37401F0A374D2F0900026A17484F5
:205BE000F0A37401F0A374E3F0A3E4F0A37402F0A3E4F0A304F0A3E4F0A304215E9F900069
:205C000022FEE004F07007900022FDE004F0900022FEE004F07007900022FDE004F0900088
:205C200023077484F0A37401F0A374F0F01202DAD9803D900023077484F0A37401F0A3740E
:205C4000FBF01202DAE98028900023077484F0A37402F0A37407F01202DAF98013900023F4
:205C6000077484F0A37402F0A37417F01202DB09900023321200844C215E21900023077481
:205C800084F0A37402F0A3741FF07B017A23790A1202D616900026A17484F0A37402F0A3DA
:205CA000742BF09000230AE0FF3395E0900026A4E4F0A3EFF09000230BE0FF3395E090008C
:205CC00026A6E4F0A3EFF09000230CE0FF3395E0900026A8E4F0A3EFF09000230DE0FF33D6
:205CE00095E0900026AAE4F0A3EFF09000230EE0FF3395E0900026ACE4F0A3EFF0900023C6
:205D00000FE0FF3395E0900026AEE4F0A3EF215E9F900023077484F0A37402F0A37449F00A
:205D20001202DCBB780A7C237D018019900023077484F0A37402F0A37455F01202DCC2784F
:205D40000A7C237D01120086EC215EAA900023077484F0A37402F0A37463F01202DC2F90AB
:205D60000026A4EEF0A3EFF0900026A17484F0A37402F0A3747B215E9F900023077484F05F
:205D8000A37402F0A3747EF090002B047401F0A37423F0A37438F0A37401F0A37423F0A313
:205DA000743AF0A37401F0A37423F0A3743CF07B017A2379361202C8FF900026A17484F0EE
:205DC000A37402F0A3748CF090002336E0FFA3E0900026A4CFF0A3EFF090002338E0FFA3D4
:205DE000E0900026A6CFF0A3EFF09000233AE0FFA3E0900026A8CFF0A3EFF09000233CE069
:205E0000FFA3E0900026AACFF0A3EF215E9F90001551E0FBA3E0FAA3E0F9E475F00221609B
:205E2000C1900026A17484F0A37402F0A374B0F090002332E0FCA3E0FDA3E0FEA3E0FF78E6
:205E4000181200837FE4900026A4F0A3EFF090002332E0FCA3E0FDA3E0FEA3E0FF78101288
:205E600000837FE4900026A6F0A3EFF090002332E0FCA3E0FDA3E0FEA3E0FF780812008315
:205E80007FE4900026A8F0A3EFF090002332E0FCA3E0FDA3A3E0FEE4900026AAF0A3CEF0D5
:205EA0007B017A23790A1200D1A37B017A23790A1200DDB0EF4E7010780A7C237D017B842A
:205EC0007A0279BC120086EC900019BBE0FBA3E0FAA3E0F990001AAEE0FEA3E0FFE92FF98C
:205EE000EA3EFAC002C001900026A17484F0A37402F0A374C3F090002307E0F9A3E0FAA338
:205F0000E0900026A4C9F0A3EAF0A3E9F0A37401F0A37423F0A3740AF0D001D0021200D1CC
:205F2000A390001AAFE02FF090001AAEE03EF0215B2A900019BBE0FBA3E0FAA3E0F9900092
:205F40001AAEE0FEA3E0FFE92FF9EA3EFA900026A17484F0A37402F0A374DDF01200D1A334
:205F600090001AAFE02FF090001AAEE03EF012027EC690001551E0FBA3E0FAA3E0F9E475E8
:205F8000F003120082289000155CE0FBA3E0FAA3E0F9E475F0012160C1E4FFFE1201AC133E
:205FA000EF4E7002FF2290001551E0FBA3E0FAA3E0F9E475F007120082281202DC38EF4ED6
:205FC0006070900019BBE0FBA3E0FAA3E0F990001AAEE0FEA3E0FFE92FF9EA3EFA90002618
:205FE000A17484F0A37403F0A37404F01200D1A390001AAFE02FF090001AAEE03EF090002F
:206000001551E0FBA3E0FAA3E0F9E475F008120082289000155CE0FBA3E0FAA3E0F9E4F58B
:20602000F012008228E4FFFE12020000EF4E7002FF221202DC38900026A17484F0A374036E
:20604000F0A37439F0900019BBE0FBA3E0FAA3E0F91200D1A390001AAEEEF0A3EFF090000A
:20606000155CE0FBA3E0FAA3E0F9E475F0011200822890001551E0FBA3E0FAA3E0F9E475B2
:20608000F00E120082289000155CE0FBA3E0FAA3E0F9120081AEC39401FFE5F09400FE90E2
:2060A000002301F0A3EFF0C39403EE64809480401790001551E0FBA3E0FAA3E0F9E475F0A0
:2060C0000F120082287F002290002302E0FF7B017A2379031202D263E4900022FDF0A3F0CC
:2060E000900022FDE0FCA3E0FDC39402EC64809480400321618B90002301E0FEA3E0780279
:20610000C333CE33CED8F92DFFEC3E900022FFF0A3EFF0900022FFE0FEA3E07802C333CE20
:2061200033CED8F924C2F974233EFA7B0178037C237D017E007F0412008820EF703A9000E7
:2061400022FFE0FEA3E09000254075F00312008458EE75F003A42583F583759300E0FBA3D2
:20616000E0FAA3E02401F9E43AFA90002307EBF0A3EAF0A3E9F08013900022FEE004F07077
:2061800007900022FDE004F02160E0900022FDE07004A3E06402700F900023077484F0A364
:2061A0007403F0A374B2F0900019BBE0FBA3E0FAA3E0F990001AAEE0FEA3E0FFE92FF9EAD4
:2061C0003EFAC002C001900026A17484F0A37403F0A374BAF090002302E02401FE9000238F
:2061E00001E03400900026A4F0A3CEF090002307E0F9A3E0FAA3E0900026A6C9F0A3EAF0BA
:20620000A3E9F0D001D0021200D1A390001AAFE02FF090001AAEE03EF09000155CE0FBA39C
:20622000E0FAA3E0F9E475F001120081FC21608678357C237D017B817A9079727E007F0C64
:206240001200805590002BB97401F0A37423F0A37434F0A37401F0A37423F0A37432F07B33
:20626000017A237933E4FF1202C89E900019BBE0FBA3E0FAA3E0F990001AAEE0FEA3E0FF87
:20628000E92FF9EA3EFAC002C001900026A17484F0A37403F0A374F6F090002332E075F0D8
:2062A00003A42435F582E43423F583759300E0F9A3E0FAA3E0900026A4C9F0A3EAF0A3E9B7
:2062C000F0D001D0021200D1A390001AAFE02FF090001AAEE03EF090002332E07012780A1E
:2062E0007C237D017B847A0279BC120086EC802A900026A17484F0A37404F0A374A8F0901A
:20630000002333E004FFF0900026A4E4F0A3EFF07B017A23790A1200D1A3900019BBE0FB43
:20632000A3E0FAA3E0F990001AAEE0FEA3E0FFE92FF9EA3EFA900026A17484F0A37404F02F
:20634000A374ADF0A37401F0A37423F0A3740AF01200D1A390001AAFE02FF090001AAEE030
:206360003EF090002332E07012780A7C237D017B847A0279BC120086EC802A900026A17460
:2063800084F0A37404F0A374A8F090002334E004FFF0900026A4E4F0A3EFF07B017A2379D3
:2063A0000A1200D1A3900019BBE0FBA3E0FAA3E0F990001AAEE0FEA3E0FFE92FF9EA3EFA2A
:2063C000900026A17484F0A37404F0A374DEF0A37401F0A37423F0A3740AF01200D1A39035
:2063E000001AAFE02FF090001AAEE03EF090001551E0FBA3E0FAA3E0F9E475F001120081C8
:20640000FC2165361202DC98EF64017070900019BBE0FBA3E0FAA3E0F990001AAEE0FEA3F7
:20642000E0FFE92FF9EA3EFA900026A17484F0A37405F0A3740EF01200D1A390001AAFE02B
:206440002FF090001AAEE03EF09000155CE0FBA3E0FAA3E0F9E4F5F0120082289000155167
:20646000E0FBA3E0FAA3E0F9E475F01312008228E4FFFE12023950EF4E7067FF221202DC8D
:2064800098EF6402705C900026A17484F0A37405F0A37441F0900019BBE0FBA3E0FAA3E071
:2064A000F91200D1A390001AAEEEF0A3EFF09000155CE0FBA3E0FAA3E0F9E4F5F012008273
:2064C0002890001551E0FBA3E0FAA3E0F9E475F01712008228E4FFFE120183CEEF4E7002BA
:2064E000FF22900019BBE0FBA3E0FAA3E0F990001AAEE0FEA3E0FFE92FF9EA3EFA900026A2
:20650000A17484F0A37405F0A37476F01200D1A390001AAFE02FF090001AAEE03EF0900095
:206520001551E0FBA3E0FAA3E0F9E4F5F01200822880037F01227F002290002C57EBF0A345
:20654000EAF0A3E9F07E0090002CBE7401F0A3742CF0A3745DF07B017A2C795B1202C63CE5
:2065600090002C5AE0FD1470032166DC1470032167C0147003216A1824FE7003216B781498
:206580007003216C5C24066003216D9190002C5CE0FF90002C5EE0FBE490002D40F09000A6
:2065A0002C57E0F9A3E0FAA3E090002D41C9F0A3EAF0A3E9F01202B7E390002C5CE0FF909A
:2065C000002C5AE0FD90002C5EE0FBC00390002D407401F090002C57E0FBA3E0FAA3E0242C
:2065E00004F9E43AFA90002D41EBF0A3EAF0A3E9F0D0031202B7E390002C5CE0FF90002C80
:206600005AE0FD90002C5EE0FBC00390002D407402F090002C57E0FBA3E0FAA3E02408F915
:20662000E43AFA90002D41EBF0A3EAF0A3E9F0D0031202B7E390002C5CE0FF90002C5AE002
:20664000FD90002C5EE0FBC00390002D407403F090002C57E0FBA3E0FAA3E0240CF9E43AEC
:20666000FA90002D41EBF0A3EAF0A3E9F0D0031202B7E390002C5CE0FF90002C5AE0FD9053
:20668000002C5EE0FBC00390002D407404F090002C57E0FBA3E0FAA3E02410F9E43AFA90AA
:2066A000002D41EBF0A3EAF0A3E9F0D0031202B7E390002C5CE0FF90002C5AE0FD90002C71
:2066C0005EE0FBC00390002D407405F090002C57E0FBA3E0FAA3E02414216D7B90002C5C11
:2066E000E0FF90002C5AE0FD90002C5EE0FBC003E490002D40F090002C57E0FBA3E0FAA331
:20670000E0241CF9E43AFA90002D41EBF0A3EAF0A3E9F0D0031202B7E390002C5CE0FF906E
:20672000002C5AE0FD90002C5EE0FBC00390002D407401F090002C57E0FBA3E0FAA3E024CA
:2067400020F9E43AFA90002D41EBF0A3EAF0A3E9F0D0031202B7E390002C5CE0FF90002C02
:206760005AE0FD90002C5EE0FBC00390002D407402F090002C57E0FBA3E0FAA3E02424F998
:20678000E43AFA90002D41EBF0A3EAF0A3E9F0D0031202B7E390002C5CE0FF90002C5AE0A1
:2067A000FD90002C5EE0FBC00390002D407403F090002C57E0FBA3E0FAA3E02428216D7B7D
:2067C00090002C5CE0FF90002C5AE0FD90002C5EE0FBC003E490002D40F090002C57E0FB58
:2067E000A3E0FAA3E0242CF9E43AFA90002D41EBF0A3EAF0A3E9F0D0031202B7E390002C29
:206800005CE0FF90002C5AE0FD90002C5EE0FBC00390002D407401F090002C57E0FBA3E0BF
:20682000FAA3E02430F9E43AFA90002D41EBF0A3EAF0A3E9F0D0031202B7E390002C5CE02B
:20684000FF90002C5AE0FD90002C5EE0FBC00390002D407402F090002C57E0FBA3E0FAA31D
:20686000E02434F9E43AFA90002D41EBF0A3EAF0A3E9F0D0031202B7E390002C5CE0FF90F5
:20688000002C5AE0FD90002C5EE0FBC00390002D407403F090002C57E0FBA3E0FAA3E02467
:2068A00038F9E43AFA90002D41EBF0A3EAF0A3E9F0D0031202B7E390002C5CE0FF90002C89
:2068C0005AE0FD90002C5EE0FBC00390002D407404F090002C57E0FBA3E0FAA3E0243CF91D
:2068E000E43AFA90002D41EBF0A3EAF0A3E9F0D0031202B7E390002C5CE0FF90002C5AE040
:20690000FD90002C5EE0FBC00390002D407405F090002C57E0FBA3E0FAA3E02440F9E43AF3
:20692000FA90002D41EBF0A3EAF0A3E9F0D0031202B7E390002C5CE0FF90002C5AE0FD9090
:20694000002C5EE0FBC00390002D407408F090002C57E0FBA3E0FAA3E02448F9E43AFA90AB
:20696000002D41EBF0A3EAF0A3E9F0D0031202B7E390002C5CE0FF90002C5AE0FD90002CAE
:206980005EE0FBC00390002D407409F090002C57E0FBA3E0FAA3E0244CF9E43AFA90002D65
:2069A00041EBF0A3EAF0A3E9F0D0031202B7E390002C5CE0FF90002C5AE0FD90002C5EE05D
:2069C000FBC00390002D40740AF090002C57E0FBA3E0FAA3E02450F9E43AFA90002D41EB32
:2069E000F0A3EAF0A3E9F0D0031202B7E390002C5CE0FF90002C5AE0FD90002C5EE0FBC08E
:206A00000390002D40740BF090002C57E0FBA3E0FAA3E02454216D7B90002C5CE0FF900011
:206A20002C5AE0FD90002C5EE0FBC003E490002D40F090002C57E0FBA3E0FAA3E02458F907
:206A4000E43AFA90002D41EBF0A3EAF0A3E9F0D0031202B7E390002C5CE0FF90002C5AE0DE
:206A6000FD90002C5EE0FBC00390002D407401F090002C57E0FBA3E0FAA3E0245CF9E43A7A
:206A8000FA90002D41EBF0A3EAF0A3E9F0D0031202B7E390002C5CE0FF90002C5AE0FD902F
:206AA000002C5EE0FBC00390002D407402F090002C57E0FBA3E0FAA3E02460F9E43AFA9038
:206AC000002D41EBF0A3EAF0A3E9F0D0031202B7E390002C5CE0FF90002C5AE0FD90002C4D
:206AE0005EE0FBC00390002D407403F090002C57E0FBA3E0FAA3E02464F9E43AFA90002DF2
:206B000041EBF0A3EAF0A3E9F0D0031202B7E390002C5CE0FF90002C5AE0FD90002C5EE0FB
:206B2000FBC00390002D407404F090002C57E0FBA3E0FAA3E02468F9E43AFA90002D41EBBE
:206B4000F0A3EAF0A3E9F0D0031202B7E390002C5CE0FF90002C5AE0FD90002C5EE0FBC02C
:206B60000390002D407405F090002C57E0FBA3E0FAA3E0246C216D7B90002C5CE0FF90009E
:206B80002C5AE0FD90002C5EE0FBC003E490002D40F090002C57E0FBA3E0FAA3E02478F986
:206BA000E43AFA90002D41EBF0A3EAF0A3E9F0D0031202B7E390002C5CE0FF90002C5AE07D
:206BC000FD90002C5EE0FBC00390002D407401F090002C57E0FBA3E0FAA3E0247CF9E43AF9
:206BE000FA90002D41EBF0A3EAF0A3E9F0D0031202B7E390002C5CE0FF90002C5AE0FD90CE
:206C0000002C5EE0FBC00390002D407402F090002C57E0FBA3E0FAA3E02480F9E43AFA90B6
:206C2000002D41EBF0A3EAF0A3E9F0D0031202B7E390002C5CE0FF90002C5AE0FD90002CEB
:206C40005EE0FBC00390002D407403F090002C57E0FBA3E0FAA3E02484216D7B90002C5C1D
:206C6000E0FF90002C5AE0FD90002C5EE0FBC003E490002D40F090002C57E0FBA3E0FAA3AB
:206C8000E02488F9E43AFA90002D41EBF0A3EAF0A3E9F0D0031202B7E390002C5CE0FF907D
:206CA000002C5AE0FD90002C5EE0FBC00390002D407401F090002C57E0FBA3E0FAA3E02445
:206CC0008CF9E43AFA90002D41EBF0A3EAF0A3E9F0D0031202B7E390002C5CE0FF90002C11
:206CE0005AE0FD90002C5EE0FBC00390002D407402F090002C57E0FBA3E0FAA3E02490F9A7
:206D0000E43AFA90002D41EBF0A3EAF0A3E9F0D0031202B7E390002C5CE0FF90002C5AE01B
:206D2000FD90002C5EE0FBC00390002D407403F090002C57E0FBA3E0FAA3E02494F9E43A7D
:206D4000FA90002D41EBF0A3EAF0A3E9F0D0031202B7E390002C5CE0FF90002C5AE0FD906C
:206D6000002C5EE0FBC00390002D407404F090002C57E0FBA3E0FAA3E02498F9E43AFA903B
:206D8000002D41EBF0A3EAF0A3E9F0D0031202B7E322E490002BD5F0A3F090002BD3F09009
:206DA000002BD3E0FF04F0EFC3940A5069E47F807E80FDFC90002BD91200844C90002BD618
:206DC000E0FFC00790002BD9E0FCA3E0FDA3E0FEA3E0FF90002D391200844CD0077D147C5E
:206DE000001202C7D890002BD6E0FF7B017A2B79D97D147C001202CD5BE47F807E80FDFCDA
:206E000090002BD9E0F8A3E0F9A3E0FAA3E0FBC31200836E708990002BD3E0B40A0412028C
:206E2000D8E1E47F81FEFDFC90002BD91200844C90002BD6E0FFC00790002BD9E0FCA3E01E
:206E4000FDA3E0FEA3E0FF90002D391200844CD0077D177C001202C7D8E4FF7E04FDFC90D2
:206E6000002BD91200844C90002BD6E0FFC00790002BD9E0FCA3E0FDA3E0FEA3E0FF900072
:206E80002D391200844CD0077D187C001202C7D8E47F747E88FDFC90002BD91200844C9033
:206EA000002BD6E0FFC00790002BD9E0FCA3E0FDA3E0FEA3E0FF90002D391200844CD00789
:206EC0007D1C7C001202C7D8E47F807E19FDFC90002BD91200844C90002BD6E0FFC007903A
:206EE000002BD9E0FCA3E0FDA3E0FEA3E0FF90002D391200844CD0077D1D7C001202C7D8B7
:206F0000E47F2C7E01FDFC90002BD91200844C90002BD6E0FFC00790002BD9E0FCA3E0FDCD
:206F2000A3E0FEA3E0FF90002D391200844CD0077D1E7C001202C7D8E4FFFEFDFC90002B40
:206F4000D91200844C90002BD6E0FFC00790002BD9E0FCA3E0FDA3E0FEA3E0FF90002D3956
:206F60001200844CD0077D267C001202C7D8E47FA07EFCFDFC90002BD91200844C90002BDF
:206F8000D6E0FFC00790002BD9E0FCA3E0FDA3E0FEA3E0FF90002D391200844CD0077D68EE
:206FA0007C001202C7D8E47F417EFAFDFC90002BD91200844CE490002BD3F090002BD3E047
:206FC000FEC39402503D90002BD6E0FFC007EE2469FDE433FCC004C00590002BD9E0FCA36F
:206FE000E0FDA3E0FEA3E0FF90002D391200844CD005D004D0071202C7D890002BD3E00434
:20700000F080B8E47F417EFAFDFC90002BD91200844CE490002BD3F090002BD3E0FEC39498
:2070200002503D90002BD6E0FFC007EE246BFDE433FCC004C00590002BD9E0FCA3E0FDA3E1
:20704000E0FEA3E0FF90002D391200844CD005D004D0071202C7D890002BD3E004F080B82B
:20706000E47F107E20FDFC90002BD91200844C90002BD6E0FFC00790002BD9E0FCA3E0FD69
:20708000A3E0FEA3E0FF90002D391200844CD0077D6D7C001202C7D8E47F047E08FDFC90AF
:2070A000002BD91200844C90002BD6E0FFC00790002BD9E0FCA3E0FDA3E0FEA3E0FF900030
:2070C0002D391200844CD0077D6E7C001202C7D8E47F087E10FDFC90002BD91200844C907F
:2070E000002BD6E0FFC00790002BD9E0FCA3E0FDA3E0FEA3E0FF90002D391200844CD00747
:207100007D6F7C001202C7D8E47F027E04FDFC90002BD91200844C90002BD6E0FFC0079037
:20712000002BD9E0FCA3E0FDA3E0FEA3E0FF90002D391200844CD0077D707C001202C7D821
:20714000E490002BD3F090002BD3E0FBC3940440032171F5E4FF7E01FDFC90002BD912003E
:20716000844CEB75F002A42471FDE435F0FCC004C00590002BD6E0FFC00790002BD9E0FC82
:20718000A3E0FDA3E0FEA3E0FF90002D391200844CD007D005D0041202C7D8E4FFFEFDFC87
:2071A00090002BD91200844C90002BD3E075F002A42471FFE435F0CF2401FDE43FFCC0046F
:2071C000C00590002BD6E0FFC00790002BD9E0FCA3E0FDA3E0FEA3E0FF90002D3912008434
:2071E0004CD007D005D0041202C7D890002BD3E004F0217146E47F087E08FDFC90002BD958
:207200001200844C90002BD6E0FFC00790002BD9E0FCA3E0FDA3E0FEA3E0FF90002D39125A
:2072200000844CD0077D797C001202C7D8E47F1E7E14FDFC90002BD91200844C90002BD66F
:20724000E0FFC00790002BD9E0FCA3E0FDA3E0FEA3E0FF90002D391200844CD0077D7A7C73
:20726000001202C7D8E4FFFEFDFC90002BD91200844C90002BD6E0FFC00790002BD9E0FC64
:20728000A3E0FDA3E0FEA3E0FF90002D391200844CD0077D7B7C001202C7D8E47F207E4054
:2072A000FDFC90002BD91200844C90002BD6E0FFC00790002BD9E0FCA3E0FDA3E0FEA3E034
:2072C000FF90002D391200844CD0077D817C001202C7D8E4FF7E40FDFC90002BD91200840F
:2072E0004C90002BD6E0FFC00790002BD9E0FCA3E0FDA3E0FEA3E0FF90002D391200844C40
:20730000D0077D8C7C001202C7D8E47F11FEFDFC90002BD91200844C90002BD6E0FFC00746
:2073200090002BD9E0FCA3E0FDA3E0FEA3E0FF90002D391200844CD0077D957C001202C742
:20734000D8E47F337E22FDFC90002BD91200844C90002BD6E0FFC00790002BD9E0FCA3E086
:20736000FDA3E0FEA3E0FF90002D391200844CD0077D967C001202C7D8E47F557E44FDFCA9
:2073800090002BD91200844C90002BD6E0FFC00790002BD9E0FCA3E0FDA3E0FEA3E0FF90BD
:2073A000002D391200844CD0077D977C001202C7D8E490002BD4F090002BD4E0FF7E00D349
:2073C00090002489E09F7480F890002488E0648098500321751690002CBE7401F0A3742B4D
:2073E000F0A374D7F07B017A2B79D51202C63C90002BD7E0FAA3E0FB64184A701FFFFEFD01
:20740000FCA31200844C90002BD6E0FFC007EBAE027803C333CE33CED8F98024E47F01FE02
:20742000FDFC90002BD91200844C90002BD6E0FFC007A3E0FEA3E07803C333CE33CED8F991
:207440002403FDEE3401FCC004C00590002BD9E0FCA3E0FDA3E0FEA3E0FF90002D39120065
:20746000844CD005D004D0071202C7D8E4FFFEFDFC90002BD91200844C90002BD6E0FFC089
:2074800007A3E0FEA3E07803C333CE33CED8F92404FDEE3401FCC004C00590002BD9E0FC93
:2074A000A3E0FDA3E0FEA3E0FF90002D391200844CD005D004D0071202C7D8E47F017E104C
:2074C000FDFC90002BD91200844C90002BD6E0FFC007A3E0FEA3E07803C333CE33CED8F9F1
:2074E0002405FDEE3401FCC004C00590002BD9E0FCA3E0FDA3E0FEA3E0FF90002D391200C3
:20750000844CD005D004D0071202C7D890002BD4E004F02173B72290001551E0FBA3E0FA4A
:20752000A3E0F9E475F001120081D2AFF0FE6003217C75EF24FE7003217B60147003217B6B
:20754000DC24026003217C7590002B407483F0A374F5F0A374E6F0900019BBE0FBA3E0FA2D
:20756000A3E0F912029EF690002275EBF0A3EAF0A3E9F0900025A17483F0A374F5F0A3749C
:20758000EFF0A37401F0A37422F0A37478F01200D5829000227AE4F0A374F0F0E02464F0A4
:2075A0009000227AE03400F0900026A17483F0A374F5F0A374FAF090002278E0FEA3E0FFD6
:2075C000900026A4EEF0A3EFF09000227AE0FDA3E0900026A6CDF0A3EDF0EF2401FFE43E97
:2075E000A3F0A3EFF0900019BBE0FBA3E0FAA3E0F91200D1A390001AAEEEF0A3EFF0900070
:207600002278E0F9A3E0FF9000155CE0FBA3E0FAA3E0C98FF01200822890002279E0FF1279
:2076200002DA569000227CEEF0A3EFF090002279E0FF7B017A22799412028B6E7B017A2236
:2076400079981202D5989000227CE07004A3E064046003217731900019BBE0FBA3E0FAA3A0
:20766000E0F990001AAEE0FEA3E0FFE92FF9EA3EFA900026A17483F0A374F7F0A374D0F033
:207680001200D1A390001AAFE02FF090001AAEE03EF090002279E0FF1202D4D3EF4E70082C
:2076A0007B837AF779F9803190002294E0C4F854F0C8A3E0C4540F48540F9000263475F0A6
:2076C0000312008458E475F003A42583F583759300E0FBA3E0FAA3E0F990002275EBF0A328
:2076E000EAF0A3E9F0900019BBE0FBA3E0FAA3E0F990001AAEE0FEA3E0FFE92FF9EA3EFA11
:20770000C002C001900026A17483F0A374F8F0A37406F090002275E0F9A3E0FAA3E090000C
:2077200026A4C9F0A3EAF0A3E9F0D001D00221792B900019BBE0FBA3E0FAA3E0F990001A83
:20774000AEE0FEA3E0FFE92FF9EA3EFA900026A17483F0A374F8F0A3740EF01200D1A39080
:20776000001AAFE02FF090001AAEE03EF09000227CE0FEA3E0FF64024E7003A38071EF643F
:20778000034E6006EF64054E706C900019BBE0FBA3E0FAA3E0F990001AAEE0FEA3E0FFE9D7
:2077A0002FF9EA3EFAC002C001900026A17483F0A374F8F0A37444F0E4A3F0A3F0900026B4
:2077C00034E0F9A3E0FAA3E0900026A6C9F0A3EAF0A3E9F0D001D0021200D1A390001AAF0C
:2077E000E02FF090001AAEE03EF09000227EE4F0A37405F080099000227EE4F0A304F09060
:2078000000227EE0FFA3E090002273CFF0A3EFF090002273E0FEA3E0FFD39406EE648094A8
:207820008040032179017C0090002295E0540FFDEFB5050CECB506087B837AF879598006BB
:207840007B837AF8796290002275EBF0A3EAF0A3E9F0900019BBE0FBA3E0FAA3E0F990001A
:207860001AAEE0FEA3E0FFE92FF9EA3EFAC003C002C001900026A17483F0A374F8F0A37413
:2078800063F090002273E0FEA3E0FF900026A4EEF0A3EFF090002275E0F9A3E0FAA3E090C6
:2078A0000026A6C9F0A3EAF0A3E9F09000263475F003EF12008458EE75F003A42583F58301
:2078C000759300E0F9A3E0FAA3E0900026A9C9F0A3EAF0A3E9F0D001D002D0031200D1A3BA
:2078E00090001AAFE02FF090001AAEE03EF090002274E004F0700790002273E004F02178C7
:2079000010900019BBE0FBA3E0FAA3E0F990001AAEE0FEA3E0FFE92FF9EA3EFA900026A1DD
:207920007483F0A374F8F0A3747CF01200D1A390001AAFE02FF090001AAEE03EF078807C26
:20794000227D017B837AF87988120086EC90002295E0540F6405601990002CB37483F0A32D
:2079600074F8F0A3748DF07B017A2279801202C083900019BBE0FBA3E0FAA3E0F990001ACD
:20798000AEE0FEA3E0FFE92FF9EA3EFAC002C001900026A17481F0A37490F0A37482F0A324
:2079A0007401F0A37422F0A37480F0E4A3F0A3F090002628E0F9A3E0FAA3E0900026A9C9C9
:2079C000F0A3EAF0A3E9F0D001D0021200D1A390001AAFE02FF090001AAEE03EF090002225
:2079E00094E030E0087B837AF8795980067B837AF8796290002275EBF0A3EAF0A3E9F0905D
:207A00000019BBE0FBA3E0FAA3E0F990001AAEE0FEA3E0FFE92FF9EA3EFAC002C0019000C0
:207A200026A17483F0A374F8F0A37497F0A3E4F0A304F090002275E0F9A3E0FAA3E090005D
:207A400026A6C9F0A3EAF0A3E9F09000262BE0F9A3E0FAA3E0900026A9C9F0A3EAF0A3E9CD
:207A6000F0D001D0021200D1A390001AAFE02FF090001AAEE03EF0900019BBE0FBA3E0FA73
:207A8000A3E0F990001AAEE0FEA3E0FFE92FF9EA3EFA900026A17483F0A374F8F0A374BB70
:207AA000F01200D1A390001AAFE02FF090001AAEE03EF090002279E02498F582E43422F525
:207AC00083759300E0B401087B837AF8795980067B837AF8796290002275EBF0A3EAF0A349
:207AE000E9F0900019BBE0FBA3E0FAA3E0F990001AAEE0FEA3E0FFE92FF9EA3EFAC003C007
:207B000002C001900026A17483F0A374F8F0A374D5F090002622E0F9A3E0FAA3E090002622
:207B2000A4C9F0A3EAF0A3E9F090002275E0F9A3E0FAA3E0900026A7C9F0A3EAF0A3E9F0E0
:207B400090002625E0F9A3E0FAA3E0900026AAC9F0A3EAF0A3E9F0D001D002D003217C61EB
:207B60009000155CE0FBA3E0FAA3E0F9120081AEFF90002278E5F0F0A3EFF0A3E4F0A374F1
:207B8000F0F0E02464F09000227AE03400F090002279E0FF7B017A22799412028B6E9000B1
:207BA00019BBE0FBA3E0FAA3E0F990001AAEE0FEA3E0FFE92FF9EA3EFA900026A17483F0F4
:207BC000A374F9F0A3740FF09000227AE0FFA3E0900026A4CFF0A3EFF0217C61900026A111
:207BE0007483F0A374F9F0A374FCF0A3E4F0A37406F09000155CE0FBA3E0FAA3E0F9120030
:207C000081AE2401FEE435F0900026A6F0A3CEF0E4A3F0A3F0A3F0A37405F0900019BBE06F
:207C2000FBA3E0FAA3E0F91200D1A390001AAEEEF0A3EFF0900019BBE0FBA3E0FAA3E02FA4
:207C4000F9EA3EFA900026A17483F0A374FCF0A37495F0A3E4F0A37406F0A3E4F0A3740515
:207C6000F01200D1A390001AAFE02FF090001AAEE03EF080037F01227F002290002A39EB2C
:207C8000F0A3EAF0A3E9F090002A38EFF07E0090002CBE7401F0A3742AF0A3743EF07B01DB
:207CA0007A2A793C1202C63C90002A3FE00490002A46F090002A39E0FBA3E0FAA3E0F912AF
:207CC0000081AE540F64066003217DFB90002A3DE0FFC007A3E0FEA3E07803C333CE33CECB
:207CE000D8F92400FDEE3401FC7B017A2A7940D0071202CD5B90002A40E0FCA3E0FDA3E0AE
:207D0000FEA3E054FCFFEC90002A401200844C90002A3DE0FFC007A3E0FEA3E07803C333B9
:207D2000CE33CED8F92400FDEE3401FCC004C00590002A40E0FCA3E0FDA3E0FEA3E0FF90F1
:207D4000002D391200844CD005D004D0071202C7D890002A38E0FF25E025E02491F582E4BD
:207D6000341EF583759300E064017062EF25E025E02490F582E4341EF583759300E06405F7
:207D8000704C90002A38E07D011202A5F690002A447408F0A3E4F090002A3DE0FF90002AB7
:207DA00046E0FD90002A44E0FBA3E090002E1FCBF0A3EBF0E4FB1202D04890002A38E0FF52
:207DC0007D051202A5F690002A447408800690002A44741AF0A3E4F090002A3DE0FF900019
:207DE0002A46E0FD90002A44E0FBA3E090002E1FCBF0A3EBF0E4FB0202D048E47F837E0461
:207E0000FDFC90002A401200844C90002A3DE0FFC007A3E0FEA3E07803C333CE33CED8F9DB
:207E20002400FDEE3401FCC004C00590002A40E0FCA3E0FDA3E0FEA3E0FF90002D39120018
:207E4000844CD005D004D0071202C7D890002A39E0FBA3E0FAA3E0F9120081AE540F64054B
:207E6000600321805690002A3EE07004A3E064187003217F8D90002A38E025E025E024912C
:207E8000F582E4341EF583759300E0B4013590002A447408F0A3E4F090002A3DE0FF9000A4
:207EA0002A46E0FD90002A44E0FBA3E090002E1FCBF0A3EBF0E4FB1202D0487F017E0012E8
:207EC00002CF2590002A38E025E025E02490F582E4341EF583759300E0640190002A44703C
:207EE000557405F0A374E1F090002A3DE0FF90002A46E0FD90002A44E0FBA3E090002E1FF0
:207F0000CBF0A3EBF07B041202D04890002A447402F0A3E4F090002A3DE0FF90002A46E0EC
:207F2000FD90002A44E0FBA3E090002E1FCBF0A3EBF07B098025E4F0A374A0F090002A3D37
:207F4000E0FF90002A46E0FD90002A44E0FBA3E090002E1FCBF0A3EBF07B041202D04890B8
:207F6000002A447413F0A37440F090002A3DE0FF90002A46E0FD90002A44E0FBA3E0900036
:207F80002E1FCBF0A3EBF0E4FB1202D048E47F017E16FDFC90002A401200844C90002A4089
:207FA000E0FCA3E0FDA3E0FEA3E044F0FFEE4401FEEC90002A401200844C90002A3DE0FF5F
:207FC000C007A3E0FEA3E07803C333CE33CED8F92402FDEE3401FCC004C00590002A40E020
:207FE000FCA3E0FDA3E0FEA3E0FF90002D391200844CD005D004D0071202C7D890002A3D00
:20800000E0FFC007A3E0FEA3E07803C333CE33CED8F92401FDEE3401FC7B017A2A7940D0BB
:20802000071202CD5B90002A40E0FCA3E0FDA3E0FEA3E0FFEE44C0FEEC90002A4012008438
:208040004C90002A40E0FCA3E0FDA3E0FEA3E0FFEE54DF2182A990002A447408F0A3E4F02D
:2080600090002A3DE0FF90002A46E0FD90002A44E0FBA3E090002E1FCBF0A3EBF0E4FB12EA
:2080800002D0487F017E001202CF25E47F017E16FDFC90002A401200844C90002A40E0FC1D
:2080A000A3E0FDA3E0FEA3E0540FFFEE54FEFEEC90002A401200844C90002A39E0FBA3E083
:2080C000FAA3E0F9120081AE540F14603014604A14606414607E2404600321817690002AFD
:2080E000447401F0A37440F090002A40E0FCA3E0FDA3E0FEA3E0FFEE4401FE807090002A5C
:20810000447421F0A3E4F090002A40E0FCA3E0FDA3E0FEA3E04480FF805390002A4474209D
:20812000F0A3E4F090002A40E0FCA3E0FDA3E0FEA3E04440FF803690002A447401F0A3E45B
:20814000F090002A40E0FCA3E0FDA3E0FEA3E04420FF8019E490002A44F0A3F090002A407A
:20816000E0FCA3E0FDA3E0FEA3E04410FFEC90002A401200844C90002A3EE07004A3E06451
:2081800018602390002A3DE0FF90002A46E0FD90002A44E0FBA3E090002E1FCBF0A3EBF01F
:2081A000E4FB1202D04890002A3EE07004A3E06418700321824890002A38E025E025E0240B
:2081C00090F582E4341EF583759300E06401707890002A3DE0FF90002A46E0FD90002DB491
:2081E0007401F0A3742AF0A37444F07B111202CC1E90002A44E020E54F90002A3DE0FF907C
:20820000002A46E0FD90002DB47401F0A3742AF0A37444F07B1E1202CC1E90002A44E0F05A
:20822000A3E04480F090002A3DE0FF90002A46E0FD90002A44E0FBA3E090002E1FCBF0A3BD
:20824000EBF07B1E1202D04890002A3DE0FFC007A3E0FEA3E07803C333CE33CED8F92402A6
:20826000FDEE3401FCC004C00590002A40E0FCA3E0FDA3E0FEA3E0FF90002D391200844C28
:20828000D005D004D0071202C7D8E4FFFEFDFC90002A401200844C90002A40E0FCA3E0FD9F
:2082A000A3E0FEA3E0FFEE4420FEEC90002A401200844C90002A40E0FCA3E0FDA3E0FEA329
:2082C000E054C0FFEE54F7FEEC90002A401200844C90002A39E0FBA3E0FAA3E0F912008152
:2082E000AEE5F090002A4030E012E0FCA3E0FDA3E0FEA3E04480FFEE44168010E0FCA3E085
:20830000FDA3E0FEA3E0547FFFEE54E9FEEC90002A401200844C90002A3EE0FAA3E0FB64E5
:20832000184A7012A3E0FCA3E0FDA3E0FEA3E0FFEE4420FE804E90002A38E0FF25E025E05E
:208340002491F582E4341EF583759300E0B4013DEF25E025E02490F582E4341EF58375938F
:2083600000E090002A40B4050EE0FCA3E0FDA3E0FEA3E04440800CE0FCA3E0FDA3E0FEA36C
:20838000E054BFFFEC90002A401200844C90002A3DE0FFC007EBAE027803C333CE33CED8D3
:2083A000F92401FDEE3401FCC004C00590002A40E0FCA3E0FDA3E0FEA3E0FF90002D391299
:2083C00000844CD005D004D0071202C7D82290002049EEF0A3EFF09000155CE0FBA3E0FAC6
:2083E000A3E0F9120081AE45F060032184A8900019BBE0FBA3E0FAA3E0F990001AAEE0FE6D
:20840000A3E0FFE92FF9EA3EFA900026A17484F0A37416F0A3748EF01200D1A390001AAFD7
:20842000E02FF090001AAEE03EF0E49000204BF0A3F0900019BBE0FBA3E0FAA3E0F99000AD
:208440001AAEE0FEA3E0FFE92FF9EA3EFA900026A17484F0A37416F0A374BCF01200D1A31C
:2084600090001AAFE02FF090001AAEE03EF09000204CE004F070079000204BE004F0C390D5
:2084800000204CE094049000204BE06480948040A19000155CE0FBA3E0FAA3E0F9E475F026
:2084A0000112008228218AA79000155CE0FBA3E0FAA3E0F9120081AEFFAEF0D39408EE9409
:2084C00000400321862CEF64014E703C900019BBE0FBA3E0FAA3E0F990001AAEE0FEA3E047
:2084E000FFE92FF9EA3EFA900026A17484F0A37416F0A374D6F01200D1A390001AAFE02F23
:20850000F090001AAEE03EF07B017A20795D1202D5EC900019BBE0FBA3E0FAA3E0F990007C
:208520001AAEE0FEA3E0FFE92FF9EA3EFA900026A17484F0A37417F0A3740DF01200D1A3E9
:2085400090001AAFE02FF090001AAEE03EF0E49000204BF0A3F01202A478900019BBE0FB8C
:20856000A3E0FAA3E0F990001AAEE0FEA3E0FFE92FF9EA3EFAC003C002C001900026A17406
:2085800084F0A37417F0A37421F09000155CE0FBA3E0FAA3E0F9120081AEFF900026A4E5CD
:2085A000F0F0A3EFF0A37401F0A37420F0A37451F0D001D002D0031200D1A390001AAFE09D
:2085C0002FF090001AAEE03EF09000204FE0FEA3E0FF245DF582E43420F583759300E0FD2A
:2085E0007C0090002049E0FAA3E0FB12024CC89000155CE0FBA3E0FAA3E0F9E475F0011255
:208600000081FC9000204CE004F070079000204BE004F0D39000204CE094039000204BE0A6
:20862000648094805003218556218AA79000155CE0FBA3E0FAA3E0F9120081AEFFAEF0D31B
:208640009414EE940040032187D6EF64094E703C900019BBE0FBA3E0FAA3E0F990001AAE49
:20866000E0FEA3E0FFE92FF9EA3EFA900026A17484F0A37417F0A3743EF01200D1A39000AF
:208680001AAFE02FF090001AAEE03EF07B017A20795D1202D5EC900019BBE0FBA3E0FAA38C
:2086A000E0F990001AAEE0FEA3E0FFE92FF9EA3EFA900026A17484F0A37417F0A3740DF085
:2086C0001200D1A390001AAFE02FF090001AAEE03EF09000155CE0FBA3E0FAA3E0F912006F
:2086E00081AEC39405FFE5F09400FEEF7802CEC313CE13D8F9FF9000204BEEF0A3EFF0A3CD
:20870000E4F0A304F01202A478900019BBE0FBA3E0FAA3E0F990001AAEE0FEA3E0FFE92FB6
:20872000F9EA3EFA900026A17484F0A37417F0A37479F09000204DE0FFA3E0900026A4CFB9
:20874000F0A3EFF09000204BE0FFA3E0900026A6CFF0A3EFF0A37401F0A37420F0A3745116
:20876000F01200D1A390001AAFE02FF090001AAEE03EF09000204FE0FEA3E0FF245DF5826E
:20878000E43420F583759300E0FD7C0090002049E0FAA3E0FB12024CC89000155CE0FBA3D0
:2087A000E0FAA3E0F9E475F001120081FC9000204EE004F070079000204DE004F0D390000D
:2087C000204EE094049000204DE0648094805003218705218AA79000155CE0FBA3E0FAA390
:2087E000E0F9120081AE641545F060032188BE7B017A20795D1202D5EC1202A4789000194D
:20880000BBE0FBA3E0FAA3E0F990001AAEE0FEA3E0FFE92FF9EA3EFA900026A17484F0A3FC
:208820007417F0A37498F0A37401F0A37420F0A37451F01200D1A390001AAFE02FF0900029
:208840001AAEE03EF09000204FE0FEA3E0FF245DF582E43420F583759300E0FD7C0090004A
:208860002049E0FAA3E0FB12024CC8900019BBE0FBA3E0FAA3E0F990001AAEE0FEA3E0FF1F
:20888000E92FF9EA3EFA900026A17484F0A37418F0A37414F01200D1A390001AAFE02FF04E
:2088A00090001AAEE03EF09000155CE0FBA3E0FAA3E0F9E475F001120081FC218AA79000C2
:2088C000155CE0FBA3E0FAA3E0F9120081AEFFAEF0C39440EE94004003218AA2EF64164E15
:2088E000703C900019BBE0FBA3E0FAA3E0F990001AAEE0FEA3E0FFE92FF9EA3EFA900026F3
:20890000A17484F0A37418F0A3742CF01200D1A390001AAFE02FF090001AAEE03EF07B01BC
:208920007A20795D1202D5EC900019BBE0FBA3E0FAA3E0F990001AAEE0FEA3E0FFE92FF9F1
:20894000EA3EFA900026A17484F0A37417F0A3740DF01200D1A390001AAFE02FF090001AFC
:20896000AEE03EF09000204DE4F0A304F01202A478900019BBE0FBA3E0FAA3E0F990001AC1
:20898000AEE0FEA3E0FFE92FF9EA3EFA900026A17484F0A37418F0A37476F09000204FE0DC
:2089A000FFA3E0900026A4CFF0A3EFF0A37401F0A37420F0A37451F01200D1A390001AAF34
:2089C000E02FF090001AAEE03EF09000204FE0FEA3E0FF245DF582E43420F583759300E043
:2089E000FD7C0090002049E0FAA3E0FB12024CC89000155CE0FBA3E0FAA3E0F9E475F00166
:208A0000120081FC9000155CE0FBA3E0FAA3E0F9120081AED39440E5F09400405D9000195B
:208A2000BBE0FBA3E0FAA3E0F990001AAEE0FEA3E0FFE92FF9EA3EFA900026A17484F0A3DA
:208A40007418F0A37490F09000204DE0FEA3E0FFC374049FFFE49EFEEF25E0FFEE339000A9
:208A600026A4F0A3EFF01200D1A390001AAFE02FF090001AAEE03EF0802D9000204EE004E7
:208A8000F070079000204DE004F0D39000204EE094049000204DE064809480500321896D16
:208AA00080057E007F0122E4FEFF2290001551E0FBA3E0FAA3E0F9120081AEFFAEF0E5F091
:208AC0006003219108EF24FE6037146070147003218CC1147003218DE314700321908C24F8
:208AE0000560032191087F017E001202A81390001551E0FBA3E0FAA3E0F9E475F0022191C0
:208B000001900026A17483F0A374EBF0A374CEF0900019BBE0FBA3E0FAA3E0F91200D1A391
:208B200090001AAEEEF0A3EFF090001551E0FBA3E0FAA3E0F9E475F0031200822890001506
:208B40005CE0FBA3E0FAA3E0F9120081AEC39401FFE5F09400FE7B017A2879371202C6A49A
:208B6000EF4E702B90001551E0FBA3E0FAA3E0F9E475F00412008228D390001AAFE09400AA
:208B800090001AAEE094005003218CC17F00229000155CE0FBA3E0FAA3E0F9120081AEC3CE
:208BA0009401FFE5F09400FE90002EFCE0B50616A3E0B50711900028417483F0A374ECF02C
:208BC000A37479F0800F900028417483F0A374ECF0A37482F090002837E0FEA3E0FF640176
:208BE0004E90002844700D7483F0A374ECF0A37483F0800B7483F0A374ECF0A37482F090CC
:208C00000019BBE0FBA3E0FAA3E0F990001AAEE0FCA3E0FDE92DF9EA3CFAC003C002C00183
:208C2000900026A17483F0A374ECF0A37493F09000155CE0FBA3E0FAA3E0F9120081AEFD56
:208C4000900026A4E5F0F0A3EDF090002841E0F9A3E0FAA3E0900026A6C9F0A3EAF0A3E985
:208C6000F0A3EEF0A3EFF090002844E0F9A3E0FAA3E0900026ABC9F0A3EAF0A3E9F0D00148
:208C8000D002D0031200D1A390001AAFE02FF090001AAEE03EF09000155CE0FBA3E0FAA3EF
:208CA000E0F9E475F001120081FCC390001AAFE094B090001AAEE094045003218B3D7F0037
:208CC00022900019BBE0FBA3E0FAA3E0F990001AAEE0FEA3E0FFE92FF9EA3EFA900026A1F8
:208CE0007483F0A374ECF0A374AFF01200D1A390001AAFE02FF090001AAEE03EF0900028E8
:208D000033E4F0A304F0C390002489E09401FF90002488E09400FE90002833E0FCA3E0FD4C
:208D2000D39FEE6480F8EC6480985054900019BBE0FBA3E0FAA3E0F990001AAEE0FEA3E0FA
:208D4000FFE92FF9EA3EFA900026A17483F0A374EDF0A3746DF0A3ECF0A3EDF01200D1A3B6
:208D600090001AAFE02FF090001AAEE03EF090002834E004F0708F90002833E004F08086B1
:208D8000900019BBE0FBA3E0FAA3E0F990001AAEE0FEA3E0FFE92FF9EA3EFA900026A174E5
:208DA00083F0A374EDF0A3747BF01200D1A390001AAFE02FF090001AAEE03EF09000155C85
:208DC000E0FBA3E0FAA3E0F9E475F0011200822890001551E0FBA3E0FAA3E0F9E475F005A1
:208DE00021910190002EFCE0FEA3E0FF7B017A2879371202C6A4EF4E700EFE7F0AFD7B019F
:208E00007A287937120088AA9000155CE0FBA3E0FAA3E0F9120081AEFFC390002489E09433
:208E200001FD90002488E09400FCD3EF9DE5F09C402B90001551E0FBA3E0FAA3E0F9E4752A
:208E4000F00612008228D390001AAFE0940090001AAEE09400500321908C7F00229000151E
:208E60005CE0FBA3E0FAA3E0F9120081AEC39401FEE5F0940090002835F0A3CEF0E4900010
:208E80002847F0A3F090002835E0FEA3E07803CEA2E713CE13D8F82439F58274283EF583D6
:208EA000759300E0FD7C0090002836E05407F974017E00A801088005C333CE33CED8F9FB75
:208EC000AA06EA5CFEEB5D4E601090002848E004F0700790002847E004F090002835E0FEAF
:208EE000A3E07803CEA2E713CE13D8F8243DF58274283EF583759300E0FFEB5F60109000FE
:208F00002848E004F0700790002847E004F0900019BBE0FBA3E0FAA3E0F990001AAEE0FE55
:208F2000A3E0FFE92FF9EA3EFA900026A17483F0A374EDF0A374C3F01200D1A390001AAFA1
:208F4000E02FF090001AAEE03EF090002833E4F0A37402F090002833E0FEA3E0FFC3EE6484
:208F6000809480500321906190002847E0FCA3E0FDEFB50515EEB50411900028417483F047
:208F8000A374EDF0A374CBF0800F900028417483F0A374ECF0A37482F090002833E0FEA3B4
:208FA000E0FF4E90002844600D7483F0A374EDF0A374D3F0800B7483F0A374ECF0A3748268
:208FC000F0900019BBE0FBA3E0FAA3E0F990001AAEE0FCA3E0FDE92DF9EA3CFAC003C00201
:208FE000C001900026A17483F0A374EDF0A374D8F090002835E0FDA3E0900026A4CDF0A398
:20900000EDF0A3EEF0A3EFF090002841E0F9A3E0FAA3E0900026A8C9F0A3EAF0A3E9F090FE
:20902000002844E0F9A3E0FAA3E0900026ABC9F0A3EAF0A3E9F0D001D002D0031200D1A3DC
:2090400090001AAFE02FF090001AAEE03EF090002834E024FFF090002833E034FFF0218FD5
:20906000549000155CE0FBA3E0FAA3E0F9E475F001120081FCC390001AAFE094B090001A04
:20908000AEE094045003218E087F002290002EFCE07002A3E090002841700D7483F0A374FC
:2090A000EEF0A37404F0800B7483F0A374ECF0A37482F0900026A17483F0A374EEF0A3748F
:2090C0000DF090002841E0F9A3E0FAA3E0900026A4C9F0A3EAF0A3E9F0900019BBE0FBA3D3
:2090E000E0FAA3E0F91200D1A390001AAEEEF0A3EFF090001551E0FBA3E0FAA3E0F9E4F539
:20910000F0120082287F00227F012278F97C267D017B817A9079E27E007F0612008055780C
:20912000FF7C267D017B817A9079E87E007F0C1200805590001551E0FBA3E0FAA3E0F912DD
:209140000081AEFFAEF0E5F060032196E8EF24FE700321929114700321929124026003212F
:2091600096E8900026A17484F0A37424F0A37469F0900019BBE0FBA3E0FAA3E0F91200D17C
:20918000A390001AAEEEF0A3EFF0900019BBE0FBA3E0FAA3E0F990001AAEE0FEA3E0FFE99B
:2091A0002FF9EA3EFA900026A17484F0A37424F0A374D9F01200D1A390001AAFE02FF090AD
:2091C000001AAEE03EF01202DB09900026ED1200844C900026F5E4F0A304F0900019BBE0E2
:2091E000FBA3E0FAA3E0F990001AAEE0FEA3E0FFE92FF9EA3EFAC001900026A17484F0A3ED
:209200007425F0A3741CF0900026F6E075F008A4FFC374209FF9900026EDE0FCA3E0FDA375
:20922000E0FEA3E0FFA8011200837FE4900026A4F0A3EFF0D0011200D1A390001AAFE02FA2
:20924000F090001AAEE03EF0900026F6E004F07007900026F5E004F0D3900026F6E094044B
:20926000900026F5E06480948050032191DB90001AAFE024FEF090001AAEE034FFF0900055
:209280001551E0FBA3E0FAA3E0F9E475F0022196E2900019BBE0FBA3E0FAA3E0F990001ACE
:2092A000AEE0FEA3E0FFE92FF9EA3EFA900026A17481F0A37490F0A374B0F0A37484F0A3B5
